:020000040800F2
:1000000000800020D90B0008A14A0008A54A00087A
:10001000A94A0008AD4A0008B14A000800000000E3
:10002000000000000000000000000000B94A0008C5
:10003000B54A000800000000BD4A0008C14A000897
:10004000914C0008954C0008994C0008A14C000800
:10005000214F0008254F0008294F00082D4F0008A8
:10006000314F0008354F0008394F000800000000EC
:100070000000000000000000000000000000000080
:100080000000000000000000000000003D4F0008DC
:10009000414F0008454F0008494F00084D4F0008E8
:1000A000514F0008554F0008594F00085D4F000898
:1000B000614F000859500008715000088550000831
:1000C000895000088D500008915000089550000894
:1000D000995000089D500008A1500008A550000844
:1000E000F1500008FD500008015100080000000018
:1000F0000000000000000000000000000000000000
:1001000000000000000000000000000000000000EF
:10011000A9500008000000000000000000000000DE
:1001200000000000000000000000000000000000CF
:1001300000000000000000000000000000000000BF
:1001400000000000000000000000000000000000AF
:10015000000000000000000000000000000000009F
:10016000000000000000000000000000000000008F
:10017000000000000000000000000000000000007F
:10018000000000000000000000000000000000006F
:10019000000000000000000000000000000000005F
:1001A000000000000000000000000000000000004F
:1001B000000000000000000000000000000000003F
:1001C000000000000000000000000000000000002F
:1001D000000000000000000000000000000000001F
:0401E0005FF8E0F1F3
:1001E80081F0004102E000BF83F0004330B54FEAE0
:1001F80041044FEA430594EA050F08BF90EA020F4D
:100208001FBF54EA000C55EA020C7FEA645C7FEADF
:10021800655C00F0E2804FEA5454D4EB5555B8BF02
:100228006D420CDD2C4480EA020281EA030382EA73
:10023800000083EA010180EA020281EA0303362D05
:1002480088BF30BD11F0004F4FEA01314FF4801CD8
:100258004CEA113102D0404261EB410113F0004FEA
:100268004FEA03334CEA133302D0524263EB4303A1
:1002780094EA050F00F0A780A4F10104D5F1200E3F
:100288000DDB02FA0EFC22FA05F2801841F100019A
:1002980003FA0EF2801843FA05F359410EE0A5F16E
:1002A80020050EF1200E012A03FA0EFC28BF4CF09F
:1002B800020C43FA05F3C01851EBE37101F0004555
:1002C80007D54FF0000EDCF1000C7EEB00006EEB62
:1002D8000101B1F5801F1BD3B1F5001F0CD34908EC
:1002E8005FEA30004FEA3C0C04F101044FEA445243
:1002F80012F5800F80F09A80BCF1004F08BF5FEACA
:10030800500C50F1000041EB045141EA050130BDA9
:100318005FEA4C0C404141EB010111F4801FA4F14C
:100328000104E9D191F0000F04BF01460020B1FAA1
:1003380081F308BF2033A3F10B03B3F120020CDAD9
:100348000C3208DD02F1140CC2F10C0201FA0CF0B7
:1003580021FA02F10CE002F11402D8BFC2F1200C1C
:1003680001FA02F120FA0CFCDCBF41EA0C019040D2
:10037800E41AA2BF01EB0451294330BD6FEA04041B
:100388001F3C1CDA0C340EDC04F11404C4F1200206
:1003980020FA04F001FA02F340EA030021FA04F318
:1003A80045EA030130BDC4F10C04C4F1200220FA6F
:1003B80002F001FA04F340EA0300294630BD21FAAD
:1003C80004F0294630BD94F0000F83F4801306BF73
:1003D80081F480110134013D4EE77FEA645C18BF67
:1003E8007FEA655C29D094EA050F08BF90EA020FFE
:1003F80005D054EA000C04BF1946104630BD91EAF6
:10040800030F1EBF0021002030BD5FEA545C05D1F8
:100418004000494128BF41F0004130BD14F5800437
:100428003CBF01F5801130BD01F0004545F0FE41AB
:1004380041F470014FF0000030BD7FEA645C1ABFE0
:10044800194610467FEA655C1CBF0B46024650EA17
:10045800013406BF52EA033591EA030F41F4002143
:1004680030BD00BF90F0000F04BF0021704730B5C9
:100478004FF4806404F132044FF000054FF000019E
:1004880050E700BF90F0000F04BF0021704730B55F
:100498004FF4806404F1320410F0004548BF404234
:1004A8004FF000013EE700BF42004FEAE2014FEA89
:1004B80031014FEA02701FBF12F07F4393F07F4F64
:1004C80081F06051704792F0000F14BF93F07F4F96
:1004D800704730B54FF4607401F0004521F00041D9
:1004E80020E700BF50EA010208BF704730B54FF05F
:1004F80000050AE050EA010208BF704730B511F064
:10050800004502D5404261EB41014FF4806404F19B
:1005180032045FEA915C3FF4DCAE4FF003025FEA1D
:10052800DC0C18BF03325FEADC0C18BF033202EBA5
:10053800DC02C2F1200300FA03FC20FA02F001FAFF
:1005480003FE40EA0E0021FA02F11444C1E600BF9E
:1005580070B54FF0FF0C4CF4E06C1CEA11541DBF51
:100568001CEA135594EA0C0F95EA0C0F00F0DEF81C
:100578002C4481EA030621EA4C5123EA4C5350EA01
:10058800013518BF52EA033541F4801143F4801352
:1005980038D0A0FB02CE4FF00005E1FB02E506F0E3
:1005A8000042E0FB03E54FF00006E1FB03569CF038
:1005B800000F18BF4EF0010EA4F1FF04B6F5007F3E
:1005C80064F5407404D25FEA4E0E6D4146EB0606B0
:1005D80042EAC62141EA55514FEAC52040EA5E5039
:1005E8004FEACE2EB4F1FD0C88BFBCF5E06F1ED8E3
:1005F800BEF1004F08BF5FEA500E50F1000041EB1A
:10060800045170BD06F0004646EA010140EA0200C6
:1006180081EA0301B4EB5C04C2BFD4EB0C0541EAE8
:10062800045170BD41F480114FF0000E013C00F3FD
:10063800AB8014F1360FDEBF002001F0004170BD21
:10064800C4F10004203C35DA0C341BDC04F114043A
:10065800C4F1200500FA05F320FA04F001FA05F2C6
:1006680040EA020001F0004221F0004110EBD37093
:1006780021FA04F642EB06015EEA430E08BF20EABF
:10068800D37070BDC4F10C04C4F1200500FA04F362
:1006980020FA05F001FA04F240EA020001F00041F4
:1006A80010EBD37041F100015EEA430E08BF20EA67
:1006B800D37070BDC4F1200500FA05F24EEA020EAF
:1006C80020FA04F301FA05F243EA020321FA04F0DE
:1006D80001F0004121FA04F220EA020000EBD37095
:1006E8005EEA430E08BF20EAD37070BD94F0000F95
:1006F8000FD101F00046400041EB010111F4801FC9
:1007080008BF013CF7D041EA060195F0000F18BF79
:10071800704703F00046520043EB030313F4801FB5
:1007280008BF013DF7D043EA0603704794EA0C0F6F
:100738000CEA135518BF95EA0C0F0CD050EA410685
:1007480018BF52EA4306D1D181EA030101F0004102
:100758004FF0000070BD50EA410606BF104619462A
:1007680052EA430619D094EA0C0F02D150EA013636
:1007780013D195EA0C0F05D152EA03361CBF104677
:1007880019460AD181EA030101F0004141F0FE4116
:1007980041F470014FF0000070BD41F0FE4141F49A
:1007A800780170BD70B54FF0FF0C4CF4E06C1CEA9A
:1007B80011541DBF1CEA135594EA0C0F95EA0C0F4F
:1007C80000F0A7F8A4EB050481EA030E52EA03350A
:1007D8004FEA013100F088804FEA03334FF080552B
:1007E80045EA131343EA12634FEA022245EA111558
:1007F80045EA10654FEA00260EF000419D4208BF09
:10080800964244F1FD0404F5407402D25B084FEAB5
:100818003202B61A65EB03055B084FEA32024FF461
:1008280080104FF4002CB6EB020E75EB030E22BFBE
:10083800B61A754640EA0C005B084FEA3202B6EB7E
:10084800020E75EB030E22BFB61A754640EA5C002D
:100858005B084FEA3202B6EB020E75EB030E22BFBD
:10086800B61A754640EA9C005B084FEA3202B6EBBE
:10087800020E75EB030E22BFB61A754640EADC007D
:1008880055EA060E18D04FEA051545EA16754FEADF
:1008980006164FEAC30343EA52734FEAC2025FEAFD
:1008A8001C1CC0D111F4801F0BD141EA00014FF08C
:1008B80000004FF0004CB6E711F4801F04BF01435D
:1008C8000020B4F1FD0C88BFBCF5E06F3FF6AFAE79
:1008D800B5EB030C04BFB6EB020C5FEA500C50F109
:1008E800000041EB045170BD0EF0004E4EEA11318C
:1008F80014EB5C04C2BFD4EB0C0541EA045170BD93
:1009080041F480114FF0000E013C90E645EA060ED6
:100918008DE60CEA135594EA0C0F08BF95EA0C0F04
:100928003FF43BAF94EA0C0F0AD150EA01347FF44C
:1009380034AF95EA0C0F7FF425AF104619462CE723
:1009480095EA0C0F06D152EA03353FF4FDAE104686
:10095800194622E750EA410618BF52EA43067FF4D7
:10096800C5AE50EA41047FF40DAF52EA43057FF467
:10097800EBAE12E74A0011D212F5001211D20DD5D2
:100988006FF47873B3EB62520ED44FEAC12343F08D
:10099800004343EA505323FA02F070474FF0000037
:1009A800704750EA013002D14FF0FF3070474FF0E6
:1009B8000000704780F0004002E000BF81F0004175
:1009C80042001FBF5FEA410392EA030F7FEA226CED
:1009D8007FEA236C6AD04FEA1262D2EB1363C1BF7D
:1009E800D218414048404140B8BF5B42192B88BFEC
:1009F800704710F0004F40F4000020F07F4018BF0F
:100A0800404211F0004F41F4000121F07F4118BF2E
:100A1800494292EA030F3FD0A2F1010241FA03FCD6
:100A280010EB0C00C3F1200301FA03F100F00043BE
:100A380002D5494260EB4000B0F5000F13D3B0F186
:100A4800807F06D340084FEA310102F10102FE2AF5
:100A580051D2B1F1004F40EBC25008BF20F0010065
:100A680040EA03007047490040EB000010F4000F13
:100A7800A2F10102EDD1B0FA80FCACF1080CB2EBA6
:100A88000C0200FA0CF0AABF00EBC2505242184305
:100A9800BCBFD0401843704792F0000F81F40001AA
:100AA80006BF80F400000132013BB5E74FEA41037D
:100AB8007FEA226C18BF7FEA236C21D092EA030FE9
:100AC80004D092F0000F08BF0846704790EA010F63
:100AD8001CBF0020704712F07F4F04D1400028BF90
:100AE80040F00040704712F100723CBF00F5000072
:100AF800704700F0004343F0FE4040F400007047A8
:100B08007FEA226216BF08467FEA23630146420253
:100B180006BF5FEA412390EA010F40F48000704766
:100B28004FF0000304E000BF10F0004348BF40420C
:100B38005FEA000C08BF704743F0964301464FF048
:100B480000001CE050EA010208BF70474FF00003A4
:100B58000AE000BF50EA010208BF704711F00043E5
:100B680002D5404261EB41015FEA010C02BF8446B5
:100B78000146002043F0B64308BFA3F18053A3F514
:100B88000003BCFA8CF2083AA3EBC25310DB01FA5B
:100B980002FC634400FA02FCC2F12002BCF1004FDF
:100BA80020FA02F243EB020008BF20F00100704770
:100BB80002F1200201FA02FCC2F1200250EA4C00C4
:100BC80021FA02F243EB020008BF20EADC7070470A
:100BD800684620F007018D4601B540F20002C2F2D6
:100BE800000240F28813C2F200039A4211D245F281
:100BF8008C12C0F6010240F20003C2F2000340F278
:100C08008810C2F2000052F8041B43F8041B834208
:100C1800F9D340F28812C2F2000241F6AC33C2F2B4
:100C280000039A420AD213464FF0000141F6AC3253
:100C3800C2F2000243F8041B9342FBD301F0CEF842
:100C4800BDE8014085467047F0B583B001A806F0BD
:100C5800DDFE4FF48060C0F230004FF0010106F075
:100C680035FF4FF0C103ADF804304FF002048DF8A2
:100C780006404FF028068DF807604FF40060C4F274
:100C8800010001A906F0E2FD4FF40063ADF804305D
:100C98008DF806408DF807604FF44065C4F20105F1
:100CA800284601A906F0D2FD4FF4A053ADF8043050
:100CB8008DF806404FF010078DF80770284601A9F7
:100CC80006F0C4FD4EF20003ADF804308DF806407E
:100CD8004FF018038DF80730284601A906F0B6FD35
:100CE80042F2D033ADF804308DF806408DF8077025
:100CF8004FF48055C4F20105284601A906F0A6FD67
:100D080028464FF4005106F0D3FE4FF47053ADF867
:100D180004308DF806408DF807604FF4A055C4F2F2
:100D28000105284601A906F091FD4CF29933ADF86A
:100D380004308DF806408DF80770284601A906F0A2
:100D480085FD4FF44073ADF804308DF806408DF8FA
:100D580007604FF4C055C4F20105284601A906F002
:100D680075FD4FF48043ADF804308DF806404FF020
:100D780004038DF8073028460DEB030106F066FDE5
:100D88004BF69D43ADF804308DF806408DF807709A
:100D9800284601A906F05AFD03B0F0BD08B54FF08A
:100DA800040006F025FF48F6A04006F047FF4FF084
:100DB800010006F085FF4FF0010006F04FFF08BD67
:100DC80030B583B04FF000604FF0000107F036FFF8
:100DD8004FF4A06007F0A8FE4FF46D43CEF2000375
:100DE800DA68C2F30222C2F10703042B28BF0423E6
:100DF80002F1040106298CBF033A00224FF00104D6
:100E080004FA03F303F1FF3303F0020303FA02F2D7
:100E18004FEA0212D2B24FF46D43CEF2000383F8C8
:100E280023204FF01C038DF804308DF805404FF057
:100E380000058DF806508DF8074001A807F088FED8
:100E48004FF01D038DF804304FF002038DF8053084
:100E58008DF806508DF8074001A807F079FE4FF08D
:100E680003038DF804308DF805308DF8065001A87D
:100E780007F06EFE03B030BD00B589B005A808F0D4
:100E8800F7F901A808F0FDF94FF00A02ADF81420AF
:100E98004FF00003ADF8163047F6BC72ADF81820D5
:100EA800ADF81A304FF0804005A908F08BF94FF0E3
:100EB80080404FF001010A4608F0FAF94FF08040EF
:100EC8004FF0010108F0E7F909B000BD10B588B08E
:100ED80005A808F0CDF901A808F0D3F948F6A04212
:100EE800ADF814204FF00003ADF816304FF064024F
:100EF800ADF81820ADF81A304FF48064C4F200043D
:100F0800204605A908F05EF920464FF001010A467F
:100F180008F0CEF920464FF0010108F0BCF908B0FE
:100F280010BD00BF30B587B04FF41054C4F20104AF
:100F3800204608F0CDF94FF0000301938DF80830F2
:100F48004FF001058DF809504FF460220392049385
:100F58008DF81450204601A908F0FEF920464FF0FC
:100F680010012A464FF0070308F0E6FA284608F071
:100F7800D9FB2046294608F04FFA204608F068FABF
:100F88004FF41054C4F20104204608F071FA002806
:100F9800FAD14FF41050C4F2010008F085FA4FF46A
:100FA8001054C4F20104204608F08EFA0028FAD141
:100FB8004FF41050C4F201004FF0010108F0A0FAFC
:100FC80007B030BD30B587B04FF4164302934FF0E9
:100FD8000004ADF80C40ADF80E40ADF81040ADF887
:100FE80014404FF00C03ADF812304FF49045C4F2A2
:100FF8000005284602A906F089FE4FF40063ADF803
:101008000030ADF802404FF40073ADF804304FF4EF
:101018008073ADF806302846694606F057FF284623
:101028004FF0010106F082FF07B030BD30B587B040
:101038004FF00003ADF804304FF48272ADF806208B
:10104800ADF808304FF00202ADF80A204FF0010564
:10105800ADF80C504FF40072ADF80E204FF030028E
:10106800ADF81020ADF812304FF00703ADF814308A
:101078004FF46054C4F20004204601A907F014FE9E
:101088002046294607F0B0FE2046294607F058FEBC
:1010980007B030BD70B58CB005460E464FF0580409
:1010A800C4F20204204607F0CFFE43F60C03C4F254
:1010B8000003019302954FF01003039304964FF039
:1010C800000305934FF08002069207930893099353
:1010D8000A930B93204601A907F0C8FF4FF460500C
:1010E800C4F200004FF002014FF0010207F048FE81
:1010F80020464FF0010107F0FBFF0CB070BD00BFA8
:1011080010B54FF0C0504FF0010107F0E9FA07F0B1
:10111800C9FC4FF0010007F047F94FF041042046A1
:1011280007F04AFB0028FAD04FF4807007F06AF9FC
:101138004FF0010007F07EF907F048FC07F036FC95
:101148004FF00100014607F07FFB07F02FFC4FF43A
:10115800004007F00DFC07F029FC10BD38B54FF032
:10116800010007F091FD06F089FF4FF4803006F08A
:10117800D5FF07F017F840F26813C2F200031870A1
:101188001B78012B2CD14FF010000CF001FC4FF014
:1011980002000CF0F1FB4FF0000007F09DF84FF053
:1011A800000007F0DDF84FF0000007F0B7F84FF443
:1011B80040304FF4E01107F027F84FF0010007F036
:1011C80049F84FF03904204607F0F6FA0028FAD01B
:1011D8004FF0020007F04EF807F06EF80828FBD130
:1011E8004FF07D004FF0010107F04CFA4FF001007D
:1011F800014607F019FA4FF480404FF0010107F05B
:101208006FFA4FF007004FF0010107F069FA4FF449
:1012180000704FF0010107F035FA4FF0C0504FF061
:10122800010107F05DFA4FF400604FF0010107F08B
:1012380057FA4FF480204FF0010107F051FAFFF7F9
:1012480003FDFFF7BDFDFFF7A9FDFFF7BBFEFFF7A5
:1012580069FEFFF711FEFFF739FE4FF0010007F0B6
:1012680003FD4FF0B80007F045FCC0B240F2F82388
:10127800C2F2000318704FF0B40007F03BFCC0B294
:1012880040F2CB23C2F2000318704FF0B00007F011
:1012980031FCC0B240F21043C2F2000318704FF0A4
:1012A800A80007F027FCC0B240F2E813C2F200031E
:1012B80018704FF0A40007F01DFCC0B240F21443B0
:1012C800C2F2000318704FF0BC0007F013FC4AF29A
:1012D800A953984208D0FFF713FF4FF0BC004AF219
:1012E800A95107F0EBFB3BE007F070FB4FF0010062
:1012F800014607F0A9FA07F059FB40F28A13C2F237
:1013080000034FF000021A7007F0F8FA45F27F1355
:10131800C0F20103984282BF002444F20755CCF280
:101328002E2504D81CE00DF02DFE04F1010407F071
:10133800E5FAA5FB0020B4EB104FF4D307F0DEFA72
:1013480044F20753CCF22E23A3FB00234FEA1342A7
:101358004FF4A343C0F2010303FB120007F0ECFAB9
:1013680040F28A13C2F200034FF001021A704FF4E0
:10137800C07009F04FFB4FF0500009F057FB4FF0D9
:101388007F0009F071FB09F077FB38BD2DE9F043C8
:1013980085B04FF004038DF80C304FF000058DF840
:1013A8000D5041F6EF23C2F200034FF0FF021A700E
:1013B8004FF0010637461C4640F2B528C2F2000835
:1013C80040F69909C2F2000923780A2B02BFFF23CD
:1013D800237000272378122B0BD11DB105F1FF359F
:1013E800EDB201E04FF003054FF0FF0323704FF01B
:1013F800010623780F2B0AD105F10105EDB2032D63
:1014080088BF00254FF0FF0323704FF00106022D1F
:101418000FD123780E2B01BF012388F80030FF235A
:1014280023702378132B01BF002388F80030FF2393
:10143800237023780B2B02D023780D2B1FD1237810
:101448000B2B14BF00230123032D18D8DFE805F068
:1014580002080E1440F2CE22C2F20002137017E006
:1014680040F2BB12C2F200021370CEE040F2B23278
:10147800C2F200021370E5E089F800302DE1032D77
:1014880000F24481DFE815F00400C100DE00290104
:1014980040F2CE23C2F200031B784BB14FF002009A
:1014A8004FF00D0103AA4FF000030EF013FA0BE002
:1014B8004FF002004FF00D0144F6B052C0F60102A1
:1014C8004FF000030EF006FA41F27413C2F2000363
:1014D8001B684FF0010200924FF03C004FF01801DA
:1014E8004EF66022B2FBF3F24FF005030EF064FAF9
:1014F80040F2C623C2F200031B784BB14FF0020042
:101508004FF0220103AA4FF000030EF0E3F90BE0BD
:101518004FF002004FF0220144F6B052C0F601022B
:101528004FF000030EF0D6F940F6C403C2F20003F0
:101538001B784BB14FF01B004FF0220103AA4FF06C
:1015480000030EF0C7F90BE04FF01B004FF022012B
:1015580044F6B052C0F601024FF000030EF0BAF99B
:1015680040F2E133C2F200031B784BB14FF0330075
:101578004FF0220103AA4FF000030EF0ABF90BE085
:101588004FF033004FF0220144F6B052C0F601028A
:101598004FF000030EF09EF940F2BD23C2F20003A3
:1015A8001B784BB14FF04B004FF0220103AA4FF0CC
:1015B80000030EF08FF90BE04FF04B004FF02201C3
:1015C80044F6B052C0F601024FF000030EF082F963
:1015D80040F66A03C2F200031B784BB14FF0630078
:1015E8004FF0220103AA4FF000030EF073F98DE0CB
:1015F8004FF063004FF0220144F6B052C0F60102EA
:101608004FF000030EF066F980E040F2BB13C2F21F
:1016180000031B784BB14FF002004FF00D0103AAF5
:101628004FF000030EF056F970E04FF002004FF053
:101638000D0144F6B052C0F601024FF000030EF05F
:1016480049F963E040F2B233C2F200031B784BB1B0
:101658004FF002004FF00D0103AA4FF000030EF007
:1016680039F90BE04FF002004FF00D0144F6B0528B
:10167800C0F601024FF000030EF02CF998F8003084
:10168800ABB14FF002004FF0210103AA4FF0000365
:101698000EF020F94FF002004FF0170144F6B05257
:1016A800C0F601024FF000030EF014F92EE04FF0DF
:1016B80002004FF0170103AA4FF000030EF00AF9D9
:1016C8004FF002004FF0210144F6B052C0F601027B
:1016D8004FF000030EF0FEF818E099F800304BB117
:1016E8004FF002004FF00D0103AA4FF000030EF077
:1016F800F1F80BE04FF002004FF00D0144F6B05244
:10170800C0F601024FF000030EF0E4F8002E00F0DE
:101718007D810EF0D3FF40F29C23C2F200039B6848
:10172800012B10D013B1022B26D119E04FF0140071
:101738004FF0010143F2CC72C0F601024FF00003F2
:101748000EF0C8F818E04FF014004FF0010143F212
:10175800D472C0F601024FF000030EF0BBF80BE0A4
:101768004FF014004FF0010143F2DC72C0F60102A1
:101778004FF000030EF0AEF84FF0000000904FF06D
:101788000A014FF07F020B460EF0BCFD032D00F25C
:101798003B81DFE815F0040074008F001E014FF054
:1017A80064004FF0010143F2E872C0F601024FF005
:1017B80000030EF08FF840F29C23C2F200039B68EE
:1017C800012B1CD013B1022B4AD131E04FF00A0093
:1017D8004FF00E0143F2EC72C0F601024FF0000325
:1017E8000EF078F84FF00A004FF0180143F2F47247
:1017F800C0F601024FF000030EF06CF830E04FF035
:101808000A004FF00E0143F60802C0F601024FF03D
:1018180000030EF05FF84FF00A004FF0180143F68E
:101828001402C0F601024FF000030EF053F817E05F
:101838004FF00A004FF00E0143F62802C0F60102ED
:101848004FF000030EF046F84FF00A004FF0180171
:1018580043F63002C0F601024FF000030EF03AF8EA
:101868004FF00A004FF0220143F64402C0F601028D
:101878004FF000030EF02EF84FF00006C6E04FF0D0
:1018880064004FF0010143F65802C0F601024FF020
:1018980000030EF01FF84FF00A004FF00E0143F658
:1018A8005C02C0F601024FF000030EF013F84FF08F
:1018B8000006ABE04FF064004FF0010143F664020C
:1018C800C0F601024FF000030EF004F840F29C232A
:1018D800C2F200039B68012B2DD02BB1022B18BF3D
:1018E800002640F093804DE04FF00A004FF00E01C3
:1018F80043F66802C0F601024FF000030DF0EAFF5C
:101908004FF00A004FF0180143F67002C0F60102CA
:101918004FF000030DF0DEFF4FF00A004FF02201F8
:1019280043F67C02C0F601024FF000030DF0D2FF2F
:101938004FF000066AE04FF00A004FF00E0143F640
:101948008802C0F601024FF000030DF0C3FF4FF00C
:101958000A004FF0180143F69002C0F601024FF05A
:1019680000030DF0B7FF4FF00A004FF0220143F6D5
:101978009C02C0F601024FF000030DF0ABFF4FF0E0
:10198800000643E04FF00A004FF00E0143F6A802AC
:10199800C0F601024FF000030DF09CFF4FF00A0063
:1019A8004FF0180143F6B002C0F601024FF00003F1
:1019B8000DF090FF4FF00A004FF0220143F6BC02F1
:1019C800C0F601024FF000030DF084FF4FF000064F
:1019D8001CE04FF064004FF0010143F6C802C0F666
:1019E80001024FF000030DF075FF4FF00A004FF0B1
:1019F8000E0143F6CC02C0F601024FF000030DF0D1
:101A080069FF4FF0000601E04FF000064FF01400A8
:101A18004FF0010103F02AF8002F7FF4D5AC05B090
:101A2800BDE8F08370B582B004460E4600F10C00A4
:101A380044F65055C0F60105C0B22A464FF00003DF
:101A48000DF048FF04F11E00C0B231462A464FF09F
:101A580000030DF03FFF41F61533C2F200031A7878
:101A680004F124004FF001050095C0B231464FF053
:101A780002030DF0A1FF41F61733C2F200031A78F2
:101A880004F112000095C0B231464FF002030DF088
:101A980093FF41F60733C2F200031A7800952046F7
:101AA80031464FF002030DF087FF02B070BD00BF52
:101AB80010B582B00EF002FE4FF0000400942046EC
:101AC80021464FF07F024FF03F030EF01BFC4FF012
:101AD80032004FF0020143F6D402C0F60102234659
:101AE8000DF0F8FE4FF0010200924FF072004FF037
:101AF80002010B460DF060FF009420464FF00A01EA
:101B08004FF07F020B460EF0FDFB4FF002004FF046
:101B1800370143F6E002C0F6010223460DF0DAFE73
:101B280002B010BD10B582B00EF0C8FD4FF0000431
:101B38000094204621464FF07F024FF03F030EF0FD
:101B4800E1FB4FF00200014643F6EC02C0F6010249
:101B580023460DF0BFFE009420464FF00A014FF0D7
:101B68007F020B460EF0CEFB02B010BD10B582B05E
:101B78000EF0A4FD4FF000040094204621464FF0DB
:101B88007F024FF03F030EF0BDFB4FF0020001460D
:101B980043F6FC02C0F6010223460DF09BFE0094BA
:101BA80020464FF00A014FF07F020B460EF0AAFBC9
:101BB80002B010BD00B583B00EF080FD4FF00001FB
:101BC800009108464FF07F024FF03F030EF09AFB5A
:101BD80040F29C23C2F200039B68012B0FD013B183
:101BE800022B23D117E04FF00200014643F60C12F6
:101BF800C0F601024FF000030DF06CFE16E04FF046
:101C08000200014643F61C12C0F601024FF0000321
:101C18000DF060FE0AE04FF00200014643F62C1278
:101C2800C0F601024FF000030DF054FE4FF0000023
:101C380000904FF00A014FF07F020B460EF062FB56
:101C480003B000BD10B582B00EF038FD4FF00001B2
:101C5800009108464FF07F024FF03F030EF052FB11
:101C680040F29C23C2F200039B68012B10D013B1F1
:101C7800022B26D119E04FF014004FF0020143F671
:101C88003C12C0F601024FF000030DF023FE18E0ED
:101C98004FF014004FF0020143F65012C0F6010253
:101CA8004FF000030DF016FE0BE04FF014004FF05C
:101CB800020143F66412C0F601024FF000030DF072
:101CC80009FE4FF00004009420464FF00A014FF03F
:101CD8007F020B460EF016FB4FF002004FF0370163
:101CE80043F67812C0F6010223460DF0F3FD02B068
:101CF80010BD00BF10B54FF0040006F0FBFED8B1D0
:101D080041F28813C2F200034FF001041C704FF037
:101D1800040006F0EFFE01464FF0080006F0CEFE84
:101D280041F29813C2F200034FF0C8021A7040F251
:101D38008813C2F200031C704FF00C0006F0DAFEA4
:101D4800B8B141F28913C2F200034FF001021A70D0
:101D58004FF00C0006F0CEFEC0B241F29913C2F269
:101D68000003187040F28813C2F200034FF0020219
:101D78001A704FF0140006F0BDFEB8B141F27813A6
:101D8800C2F200034FF001021A704FF0140006F07F
:101D9800B1FEC0B241F28013C2F20003187040F2E3
:101DA8008813C2F200034FF003021A704FF01C00B0
:101DB80006F0A0FE80B141F27913C2F200034FF0A1
:101DC80001021A704FF01C0006F094FEC0B241F2F6
:101DD8005413C2F20003187010BD00BF2DE9F04F74
:101DE80083B007F01FFDFFF7B9F90DF073FF00F09E
:101DF8003FFD4FF00000014602F0C4F940F6B8304C
:101E08004FF0010102F032FE40F29C23C2F20003BF
:101E1800DB684BB14FF00003009301934FF01900BA
:101E280019461A4607F0C8FC40F29C23C2F2000388
:101E38009B68022B08D900F04FFD40F29C23C2F2A8
:101E480000034FF000029A6041F6EF23C2F200034C
:101E58004FF0FF021A70FFF72BFEFFF74BFF40F21F
:101E68006C13C2F200034FF001021A7040F2A4177B
:101E7800C2F200079146154640F28E18C2F20008D9
:101E88009A4603F104063D7088F8005041F6EF23A6
:101E9800C2F200031B780C2B11D140F64313C2F297
:101EA80000034FF000021A700BF02AFA41F6EF23F4
:101EB800C2F200034FF0FF021A708AF8009041F650
:101EC800EF23C2F200031B780A2B40F0068141F68B
:101ED800EF23C2F200034FF0FF021A700EF0EEFB80
:101EE800FFF7B0FE4FF010004FF0220143F68412C6
:101EF800C0F601024FF000030DF0ECFC41F6EF24B0
:101F0800C2F20004DCE040F64013C2F200031B7882
:101F1800002B00F0AB8040F64013C2F200034FF0F4
:101F280000021A7041F25413C2F200031B788BB3FB
:101F380040F29C23C2F200039B68012B10D013B11E
:101F4800022B33D119E04FF014004FF00D0143F686
:101F58009812C0F601024FF000030DF0BBFC25E01B
:101F68004FF014004FF00D0143F6A412C0F6010221
:101F78004FF000030DF0AEFC18E04FF014004FF0E6
:101F88000D0143F6B012C0F601024FF000030DF048
:101F9800A1FC0BE04FF014004FF00D0143F6BC120A
:101FA800C0F601024FF000030DF094FC4FF004005E
:101FB8004FF0170141F25C12C2F200024FF0000329
:101FC8000DF088FC40F26343C2F200031B784BB16A
:101FD8004FF021004FF0220132464FF000030DF080
:101FE80079FC0BE04FF021004FF0220144F6B0528B
:101FF800C0F601024FF000030DF06CFC40F2B41380
:10200800C2F200031B784BB14FF03F004FF02201A2
:1020180032464FF000030DF05DFC0BE04FF03F003F
:102028004FF0220144F6B052C0F601024FF000030F
:102038000DF050FC40F26043C2F200031B784BB134
:102048004FF05D004FF0220132464FF000030DF0D3
:1020580041FC0BE04FF05D004FF0220144F6B05216
:10206800C0F601024FF000030DF034FC41F25413A6
:10207800C2F200031B781BB323780D2B20D140F24A
:10208800CE23C2F200034FF0000B83F800B04FF0EC
:102098001C00594606F012FD41F25413C2F2000327
:1020A80083F800B04FF014004FF00D0143F6C8124A
:1020B800C0F601025B460DF00DFC4FF0FF032370E4
:1020C80023780A2B7FF41FAF41F6EF23C2F20003F7
:1020D8004FF0FF021A708AF8009041F6EF23C2F21F
:1020E80000031B780B2B40F0178140F28813C2F2D3
:1020F80000031B78002B40F00F8108F099FD0028A1
:1021080041D00EF0DBFA40F29C23C2F200039B6838
:10211800012B10D013B1022B26D119E04FF0140077
:102128004FF01E0143F6D412C0F601024FF000032F
:102138000DF0D0FB18E04FF014004FF01E0143F6ED
:10214800E412C0F601024FF000030DF0C3FB0BE0F0
:102158004FF014004FF01E0143F6F412C0F60102CE
:102168004FF000030DF0B6FB4FF4FA60494602F059
:102178007DFC40F28813C2F200034FF000021A708F
:10218800FFF796FCBFE040F29C23C2F200039B6875
:10219800012B13D013B1022B2FD11FE04FF00000F9
:1021A80043F60821C0F601014FF00A0209F0C0F811
:1021B80040F63C13C2F2000318601EE04FF0000026
:1021C80043F61C21C0F601014FF00A0209F0B0F8ED
:1021D80040F63C13C2F2000318600EE04FF0000016
:1021E80043F63021C0F601014FF00A0209F0A0F8C9
:1021F80040F63C13C2F20003186040F63C13C2F2EA
:1022080000031B68042B6ED8DFE803F0030B233CA4
:10221800550040F28813C2F200034FF000021A7012
:102228006AE04FF00400494606F048FC41F2981372
:10223800C2F2000383F8009040F28813C2F2000350
:1022480083F8009040F29613C2F2000383F80090DE
:1022580052E04FF00C00494606F030FC41F2991369
:10226800C2F2000383F8009040F28813C2F2000320
:102278004FF002021A7040F29613C2F2000383F87C
:10228800009039E04FF01400494606F017FC41F27F
:102298008013C2F2000383F8009040F28813C2F260
:1022A80000034FF003021A7040F29613C2F20003C3
:1022B80083F8009020E041F25413C2F200031B7827
:1022C800D3B94FF01C00494606F0F8FB41F254130D
:1022D800C2F2000383F8009040F29613C2F20003A2
:1022E80083F8009008E040F28813C2F200034FF030
:1022F80000021A70FFF7DCFB41F62233C2F200033A
:102308004FF0FF021A7041F6EF23C2F200034FF0BC
:10231800FF021A708AF8009040F64013C2F20003D8
:102328001B78002B3FF4AFAD40F64013C2F2000318
:102338004FF000021A7040F28813C2F200031B78B3
:10234800042B00F28882DFE813F005005600F20043
:10235800780100029AF800302BB14FF000038AF898
:102368000030FFF7A5FB08F041F888B340F29C2342
:10237800C2F200039B68012B10D013B1022B33D19A
:1023880019E04FF028004FF01E0143F64022C0F636
:1023980001024FF000030DF09DFA25E04FF02800F0
:1023A8004FF01E0143F64822C0F601024FF0000329
:1023B8000DF090FA18E04FF028004FF01E0143F698
:1023C8005422C0F601024FF000030DF083FA0BE02F
:1023D8004FF032004FF01E0143F66422C0F60102AE
:1023E8004FF000030DF076FA4FF04D004FF0370133
:1023F800FFF718FB47E59AF800302BB14FF00003C0
:102408008AF80030FFF78EFB40F64313C2F2000350
:1024180083F800904FF004004FF00D0141F64C3264
:10242800C2F200024FF000030DF054FA4FF004001E
:102438004FF0170141F63432C2F200024FF00003A8
:102448000DF048FA4FF004004FF0210141F69432A4
:10245800C2F200024FF000030DF03CFA4FF0040006
:102468004FF02B0141F67C32C2F200024FF000031C
:102478000DF030FA4FF004004FF0350141F66432A8
:10248800C2F200024FF000030DF024FA41F6EF23E8
:10249800C2F200031B780D2B31D140F28C13C2F22B
:1024A80000034FF000041C7041F29813C2F20003BD
:1024B8001C704FF00400214606F000FB0BF052FCA4
:1024C80040F28813C2F200031C70FFF7F1FA4FF0D4
:1024D8001C0006F00FFBC0B241F25413C2F2000315
:1024E800187041F27913C2F2000383F8009041F6A4
:1024F800EF23C2F200034FF0FF021A70C3E441F267
:102508009813C2F200031B78002B7FF4BCACFFF7D2
:10251800CFFA0BF027FC40F28813C2F200034FF009
:10252800000119704FF0040006F0C8FAABE49AF8FD
:1025380000302BB14FF000038AF80030FFF716FB8C
:1025480040F64313C2F2000383F800904FF00400F2
:102558004FF00D0141F64C32C2F200024FF0000379
:102568000DF0B8F94FF004004FF0170141F634327E
:10257800C2F200024FF000030DF0ACF94FF0040076
:102588004FF0210141F69432C2F200024FF00003ED
:102598000DF0A0F94FF004004FF02B0141F67C320A
:1025A800C2F200024FF000030DF094F94FF004005E
:1025B8004FF0350141F66432C2F200024FF00003D9
:1025C8000DF088F941F6EF23C2F200031B780D2BBA
:1025D8001BD140F28813C2F200034FF000011970BA
:1025E80041F29913C2F2000319704FF00C0006F083
:1025F80065FAFFF75DFA0BF0B5FB41F6EF23C2F27F
:1026080000034FF0FF021A703DE441F29913C2F241
:1026180000031B78002B7FF436ACFFF749FA0BF068
:10262800A1FB40F28813C2F200034FF000011970B9
:102638004FF00C0006F042FA25E49AF800302BB16E
:102648004FF000038AF80030FFF7B4FA40F643135E
:10265800C2F2000383F800904FF004004FF00D0120
:1026680041F64C32C2F200024FF000030DF032F98D
:102678004FF004004FF0170141F63432C2F2000265
:102688004FF000030DF026F94FF004004FF0210140
:1026980041F69432C2F200024FF000030DF01AF92D
:1026A8004FF004004FF02B0141F67C32C2F20002D9
:1026B8004FF000030DF00EF94FF004004FF0350114
:1026C80041F66432C2F200024FF000030DF002F945
:1026D80041F6EF23C2F200031B780D2B1CD140F208
:1026E8008813C2F200034FF0000119708AF80090B5
:1026F80041F28013C2F2000319704FF0140006F083
:10270800DDF90BF02FFB41F6EF23C2F200034FF087
:10271800FF021A70FFF7B7BB41F28013C2F2000341
:102728001B78002B7FF4AFAB0BF01CFB40F2881337
:10273800C2F200034FF0000119708AF800904FF0C0
:10274800140006F0BBF9FFF79EBB9AF800301BB1E6
:102758004FF000038AF8003040F64313C2F200033A
:1027680083F800904FF004004FF00D0141F64C3211
:10277800C2F200024FF000030DF0ACF84FF0040075
:102788004FF0170141F63432C2F200024FF0000355
:102798000DF0A0F84FF004004FF0210141F69432FB
:1027A800C2F200024FF000030DF094F84FF004005D
:1027B8004FF02B0141F67C32C2F200024FF00003C9
:1027C8000DF088F84FF004004FF0350141F66432FF
:1027D800C2F200024FF000030DF07CF841F6EF233F
:1027E800C2F200031B780D2B1CD140F28813C2F2F1
:1027F80000034FF0000119708AF8009041F2541359
:10280800C2F2000319704FF01C0006F057F90BF0E4
:10281800A9FA41F6EF23C2F200034FF0FF021A7043
:10282800FFF731BB41F25413C2F200031B78002BAF
:102838007FF429AB0BF096FA40F28813C2F200033A
:102848004FF0000119708AF800904FF01C0006F054
:1028580035F9FFF718BB8AF8009040F28813C2F2E6
:1028680000034FF000021A7002F026FDFFF70BBBC1
:1028780010B54FF47040C0F603004FF00001144A41
:102888004FF00A030CF082FC4FF47840C0F60300C6
:102898004FF000010F4A4FF010030CF077FC40F2A4
:1028A8001C44C2F200044FF43040C0F603004FF05D
:1028B800000104F104024FF004030CF067FC6368A4
:1028C800632B81BF40F21C43234600225A6010BD8F
:1028D800A00200202C1A0020F8B540F29C23C2F276
:1028E80000039B68012B0ED013B1022B20D115E0F9
:1028F8004FF0000043F66821C0F60101024608F0D7
:1029080017FDC0B214E04FF0000043F67C21C0F67A
:102918000101024608F00CFDC0B209E04FF00000CA
:1029280043F69421C0F60101024608F001FDC0B249
:10293800002800F0C2800DF0C1FE40F29C23C2F2D4
:1029480000039B68012B0FD013B1022B24D117E091
:102958004FF01E00014643F6A822C0F601024FF0D0
:1029680000030CF0B7FF22E04FF01E00014643F6CB
:10297800B422C0F601024FF000030CF0ABFF16E0E2
:102988004FF01E00014643F6C022C0F601024FF088
:1029980000030CF09FFF0AE04FF000004FF01E010B
:1029A80043F6CC22C0F6010203460CF093FF40F632
:1029B8004C14C2F200044FF00A03236063604FF026
:1029C800F002A260E3604FF4B47323614FF0050393
:1029D80063614FF00203A3614FF01403E3614FF406
:1029E8007845C0F6030528460CF07AFB28464FF0D8
:1029F800000122464FF012030CF09CFB4FF06400DC
:102A08004FF0010102F032F84FF0000626606660D0
:102A1800A6604FF01E03E3604FF0010727614FF4F3
:102A28007045C0F6030528460CF05AFB2846314687
:102A380022464FF00C030CF07DFB4FF0540031465A
:102A480006F03CF84FF05800314606F037F84FF0E2
:102A58002400314606F032F84FF02800314606F0DF
:102A68002DF806F0DFFE4FF46840C0F603000CF0C6
:102A780037FB4FF06400394601F0F8FF4FF4584037
:102A8800C0F603000CF02CFB4FF06400394601F04F
:102A9800EDFF4FF45040C0F603000CF021FB4FF05F
:102AA8006400394601F0E2FF08F080F8FFF7E0FE25
:102AB8004FF4FA60394601F0D9FFF8BD2DE9F04F1F
:102AC80091B00646012815D010B1022835D123E06F
:102AD8004FF47840C0F603004FF0000140F64C1266
:102AE800C2F200024FF010030CF050FB4FF0080048
:102AF800069022E04FF47040C0F603004FF000014A
:102B080040F64C12C2F200024FF00A030CF03EFBF2
:102B18004FF00501069110E04FF43040C0F6030075
:102B28004FF0000140F64C12C2F200024FF00403CD
:102B38000CF02CFB4FF00202069241F6EF23C2F292
:102B480000034FF0FF021A704FF0000A4FF0010324
:102B58005746994641F6EF24C2F2000440F2347B0E
:102B6800C0F6010B41F62C00C0F6010003900BF5EE
:102B78006E6101F11401059100F19002079222782B
:102B88000A2A02BFFF2222704FF000092278122A77
:102B980002D022780F2A1ED12278122A0CD12FB106
:102BA80007F1FF37FFB24FF0010305E04FF00103D3
:102BB800002E0CBF0727042722780F2A08D107F117
:102BC8000107FFB2069BBB424FF0010398BF0027E5
:102BD8004FF0FF022270002B00F076850DF06EFD9D
:102BE800012E25D016B1022E66D143E04FF01E000B
:102BF8004FF0010143F6E422C0F601024FF0000352
:102C08000CF068FE3D464FF0010100914FF06E0058
:102C18007A184FF002030CF0CFFE4FF0000000903E
:102C28004FF00A014FF07F020B460DF06BFB60E09E
:102C38004FF01E004FF0010143F6F022C0F60102EA
:102C48004FF000030CF046FE3D464FF001010091A5
:102C58004FF06E007A184FF002030CF0ADFE4FF003
:102C6800000000904FF00A014FF07F020B460DF074
:102C780049FB27E14FF01E004FF0010143F6F8220F
:102C8800C0F601024FF000030CF024FE3D464FF061
:102C9800010100914FF06E007A184FF002030CF01A
:102CA8008BFE4FF0000000904FF00A014FF07F02BA
:102CB8000B460DF027FBF9E13D464FF0010100916D
:102CC8004FF06E007A184FF002030CF075FE4FF0CB
:102CD800000000904FF00A014FF07F020B460DF004
:102CE80011FB012E00F0EE801EB1022E40F0298269
:102CF800DCE140F29C23C2F200039B68012B4BD01D
:102D08001BB1022B40F01D8291E04FEA4518A84400
:102D18004FEA88084FF001004FF00C010BEB080256
:102D28004FF000030CF0D6FD08F116024FF0010039
:102D38004FF016015A444FF000030CF0CBFD08F198
:102D48002C024FF001004FF020015A444FF00003CD
:102D58000CF0C0FD08F142024FF06E004FF0380150
:102D68005A444FF000030CF0B5FD05EB45024FEA5D
:102D7800420202F104014FF0160303FB01F11BF8B4
:102D8800018002F1050203FB02F31BF80330A3F1F3
:102D98003003DBB20493D4E14FEA4518A8444FEA64
:102DA80088084FF001004FF00C01BD4B03EB0802FF
:102DB8004FF000030CF08EFD08F116024FF00100F1
:102DC8004FF01601B64B9A184FF000030CF082FD35
:102DD80008F12C024FF001004FF02001B04B9A1877
:102DE8004FF000030CF076FD08F142024FF06E0040
:102DF8004FF03801AA4B9A184FF000030CF06AFD07
:102E080005EB45024FEA420202F104014FF01603B6
:102E180003FB01B191F8208402F1050203FB02B320
:102E280093F82034A3F13003DBB2049389E14FEA2D
:102E38004518A8444FEA88084FF001004FF00C01EC
:102E4800984B03EB08024FF000030CF043FD08F128
:102E580016024FF001004FF01601924B9A184FF0EE
:102E680000030CF037FD08F12C024FF001004FF081
:102E780020018C4B9A184FF000030CF02BFD08F141
:102E880042024FF06E004FF03801864B9A184FF00F
:102E980000030CF01FFD05EB45024FEA420202F168
:102EA80004014FF0160303FB01B191F8408802F1C9
:102EB800050203FB02B393F84038A3F13003DBB2F9
:102EC80004933EE140F29C23C2F200039B68012B6D
:102ED8004FD01BB1022B40F0348195E04FEA4518E2
:102EE800A8444FEA88084FF001004FF00C016E4BE0
:102EF80003EB08024FF000030CF0ECFC08F116029B
:102F08004FF001004FF01601674B9A184FF000037D
:102F18000CF0E0FC08F12C024FF001004FF020010A
:102F2800614B9A184FF000030CF0D4FC08F14202F0
:102F38004FF06E004FF038015B4B9A184FF00003CA
:102F48000CF0C8FC05EB45024FEA420202F104010D
:102F58004FF0160303FB01B191F8608C02F10502F2
:102F680003FB02B393F8603CA3F13003DBB2049394
:102F7800E7E04FEA4518A8444FEA88084FF00100F7
:102F88004FF00C01059B03EB08024FF000030CF017
:102F9800A1FC08F116024FF001004FF01601059B45
:102FA8009A184FF000030CF095FC08F12C024FF032
:102FB80001004FF02001059B9A184FF000030CF018
:102FC80089FC08F142024FF06E004FF03801059B72
:102FD8009A184FF000030CF07DFC05EB45024FEA10
:102FE800420202F104014FF0160303FB01B191F80C
:102FF800F48E02F1050203FB02B393F8F43EA3F149
:103008003003DBB204939CE04FEA4518A8444FEA2A
:1030180088084FF001004FF00C01079B03EB0802F2
:103028004FF000030CF056FC08F116024FF00100B7
:103038004FF01601079B9A184FF000030CF04AFC5A
:1030480008F12C024FF001004FF02001079B9A185D
:103058004FF000030CF03EFC08F142024FF06E0006
:103068004FF03801079B9A184FF000030CF032FC20
:1030780005EB45024FEA420202F104014FF0160344
:10308800039803FB010191F8908002F1050203FB0C
:10309800020393F89030A3F13003DBB2049350E0BD
:1030A800540B0108740F0108941301084FEA4518DE
:1030B800A8444FEA88084FF001004FF00C01CB4BB1
:1030C80003EB08024FF000030CF004FC08F11602B1
:1030D8004FF001004FF01601C44B9A184FF000034F
:1030E8000CF0F8FB08F12C024FF001004FF0200122
:1030F800BE4B9A184FF000030CF0ECFB08F14202AB
:103108004FF06E004FF03801B84B9A184FF000039B
:103118000CF0E0FB05EB45024FEA420202F1040124
:103128004FF01603039803FB010191F8248302F181
:10313800050203FB020393F82433A3F13003DBB247
:103148000493B8F1420F04D0B8F14C0F40F0AE82AE
:1031580041E2012E1BD016B1022E4AD130E005EB18
:1031680045034FEA430303F104034FF0160202FB41
:1031780003B35A78A2F1300202EB820293F802807C
:10318800A8F1300808EB420808F0FF0831E005EB29
:1031980045034FEA430303F104034FF0160202FB11
:1031A80003B393F8612CA2F1300202EB820293F888
:1031B800628CA8F1300808EB420808F0FF0818E014
:1031C80005EB45034FEA430303F104034FF01602EE
:1031D800039902FB031393F82523A2F1300202EBB3
:1031E800820293F82683A8F1300808EB420808F019
:1031F800FF08B8F1010F00F08880B8F1000F06D081
:10320800B8F1030F18BF002340F05E8265E140F675
:103218004C13C2F2000353F82530002B3AD040F289
:103228009C23C2F200039B68012B15D02BB1022B03
:1032380018BF002340F048821DE04FF032004FF0E5
:10324800380143F60432C0F601024FF000030CF0D7
:1032580041FB4FF0000337E24FF032004FF03801E6
:1032680043F60832C0F601024FF000030CF032FBBF
:103278004FF0000328E24FF032004FF0380143F6D8
:103288000C32C0F601024FF000030CF023FB4FF0A4
:10329800000319E240F29C23C2F200039B68012B51
:1032A80015D02BB1022B18BF002340F00D821DE072
:1032B8004FF032004FF0380143F61032C0F60102E9
:1032C8004FF000030CF006FB4FF00003FCE14FF059
:1032D80032004FF0380143F61432C0F601024FF0C5
:1032E80000030CF0F7FA4FF00003EDE14FF0320065
:1032F8004FF0380143F61832C0F601024FF00003D0
:103308000CF0E8FA4FF00003DEE140F29C23C2F231
:1033180000039B68012B4ED02BB1022B18BF002352
:1033280040F0D28191E040F64C13C2F2000353F80A
:103338002530012B12D013B1022B2DD11DE04FF0F7
:103348001E004FF0380143F62032C0F601024FF05C
:1033580000030CF0BFFA4FF00003B5E14FF01E0078
:103368004FF0380143F62C32C0F601024FF000034B
:103378000CF0B0FA4FF00003A6E14FF01E004FF03A
:10338800380143F63832C0F601024FF000030CF062
:10339800A1FA4FF0000397E14FF01E004FF03801FB
:1033A80043F64432C0F601024FF000030CF092FAE3
:1033B8004FF0000388E140F64C13C2F2000353F8C3
:1033C8002530012B14D013B1022B2FD11FE04FF061
:1033D8001E004FF0380143F64832C0F601024FF0A4
:1033E80000030CF077FA4FF000036DE1501B010861
:1033F8004FF01E004FF0380143F65432C0F6010278
:103408004FF000030CF066FA4FF000035CE14FF058
:103418001E004FF0380143F66032C0F601024FF04B
:1034280000030CF057FA4FF000034DE14FF01E0077
:103438004FF0380143F64432C0F601024FF0000362
:103448000CF048FA4FF000033EE140F64C13C2F28C
:10345800000353F82530012B12D013B1022B2DD1C4
:103468001DE04FF01E004FF0380143F66C32C0F6F5
:1034780001024FF000030CF02DFA4FF0000323E196
:103488004FF01E004FF0380143F67432C0F60102C7
:103498004FF000030CF01EFA4FF0000314E14FF058
:1034A8001E004FF0380143F68032C0F601024FF09B
:1034B80000030CF00FFA4FF0000305E14FF01E0077
:1034C8004FF0380143F64432C0F601024FF00003D2
:1034D8000CF000FA4FF00003F6E040F64C13C2F28D
:1034E800000353F82530002B3AD040F29C23C2F257
:1034F80000039B68012B15D02BB1022B18BF0023AA
:1035080040F0E2801DE04FF01E004FF0380143F616
:103518008832C0F601024FF000030CF0DBF94FF0DF
:103528000003D1E04FF01E004FF0380143F6883217
:10353800C0F601024FF000030CF0CCF94FF0000385
:10354800C2E04FF01E004FF0380143F68832C0F653
:1035580001024FF000030CF0BDF94FF00003B3E097
:1035680040F29C23C2F200039B68012B15D02BB1BB
:10357800022B18BF002340F0A7801DE04FF01E006B
:103588004FF0380143F69432C0F601024FF00003C1
:103598000CF0A0F94FF0000396E04FF01E004FF03A
:1035A800380143F69432C0F601024FF000030CF0E4
:1035B80091F94FF0000387E04FF01E004FF03801FB
:1035C80043F69432C0F601024FF000030CF082F982
:1035D8004FF0000378E0012E14D016B1022E33D13B
:1035E80021E005EB45034FEA430303F104034FF0E1
:1035F800160202FB03B393F80180A8F130085FFAC2
:1036080088F821E005EB45034FEA430303F104037F
:103618004FF0160202FB03B393F8618CA8F130084F
:103628005FFA88F810E005EB45034FEA430303F11E
:1036380004034FF01602039802FB030393F8258353
:10364800A8F130085FFA88F840F64C13C2F200037C
:1036580053F82550002D13DA0499A1EB81004FEAA5
:10366800400000F16300C0B24FF0380143F6840215
:10367800C0F601024FF000030CF02CF9C5F100056B
:10368800049AA2EB82004FEA400000F16900CDF8ED
:1036980000804FF000030193C0B24FF038012A4672
:1036A800049B0CF049FA4FF000030DE04FF00200C4
:1036B8004FF0380143F6A032C0F601024FF0000384
:1036C8000CF008F94FF0000322780C2A40F02E8203
:1036D800012E10D016B1022E27D119E007EB4703AF
:1036E8004FEA430303F104034FF0160202FB03F30E
:1036F8001BF8038019E007EB47034FEA430303F184
:1037080004034FF0160202FB03B393F8608C0CE03D
:1037180007EB47034FEA430303F104034FF0160294
:10372800039802FB030393F82483B8F1420F04D0F3
:10373800B8F14C0F40F0D6810BE1012E1AD016B12A
:10374800022E49D12FE007EB47034FEA430303F169
:1037580004034FF0160202FB03B35A78A2F13002B9
:1037680002EB82029B78A3F1300303EB420808F0D6
:10377800FF0831E007EB47034FEA430303F1040373
:103788004FF0160202FB03B393F8612CA2F130024A
:1037980002EB820293F8623CA3F1300303EB420888
:1037A80008F0FF0818E007EB47034FEA430303F16B
:1037B80004034FF01602039902FB031393F8252321
:1037C800A2F1300202EB820293F82633A3F1300310
:1037D80003EB420808F0FF08B8F1150F00F2A081CA
:1037E800DFE818F016002F009E0140009E019E01A0
:1037F8009E019E019E019E0151006200730084009B
:103808009E019E019E019E019E019E019500A600BB
:1038180040F64C13C2F2000353F8273043B140F688
:103828004C13C2F200034FF0000243F8272077E15F
:1038380040F64C13C2F200034FF0010243F8272070
:103848006EE140F64C15C2F2000555F8270043F624
:10385800B831C0F601014FF0010207F069FD45F8E3
:1038680027005DE140F64C15C2F2000555F8270027
:1038780043F6C831C0F601014FF0030207F058FDC6
:1038880045F827004CE140F64C15C2F2000555F802
:10389800270043F6D831C0F601014FF00A0207F0BD
:1038A80047FD45F827003BE140F64C15C2F20005FC
:1038B80055F8270043F6D831C0F601014FF00B0246
:1038C80007F036FD45F827002AE140F64C15C2F20C
:1038D800000555F8270043F6D831C0F601014FF02E
:1038E8000C0207F025FD45F8270019E140F64C15B4
:1038F800C2F2000555F8270043F6D831C0F6010199
:103908004FF00D0207F014FD45F8270008E140F6D6
:103918004C15C2F2000555F8270043F6EC31C0F605
:1039280001014FF0140207F003FD45F82700F7E006
:1039380040F64C15C2F2000555F8270043F6004141
:10394800C0F601014FF0150207F0F2FC45F8270018
:10395800E6E0012E14D016B1022E33D121E007EB98
:1039680047034FEA430303F104034FF0160202FB37
:1039780003B393F80180A8F130085FFA88F821E0D2
:1039880007EB47034FEA430303F104034FF0160222
:1039980002FB03B393F8618CA8F130085FFA88F84A
:1039A80010E007EB47034FEA430303F104034FF02A
:1039B8001602039802FB030393F82583A8F1300845
:1039C8005FFA88F83D4640F64C13C2F2000353F8FC
:1039D80027000499009108A942464FF001030AF014
:1039E8002DF908A807F044FA002800F0998008A8E3
:1039F8004146049A0AF08CF89DF82030032B6AD8C7
:103A0800DFE803F00209294940F64C13C2F200032B
:103A180043F8270084E00CF051FE4FF00A004FF005
:103A28001E0143F61442C0F601024FF000030BF0EA
:103A380051FF4FF03200014643F62842C0F601021A
:103A48004FF000030BF046FF4FF0FF03237023787D
:103A58000A2BFCD164E00CF031FE4FF014004FF05B
:103A68001E0143F62C42C0F601024FF000030BF092
:103A780031FF4FF03200014643F62842C0F60102FA
:103A88004FF000030BF026FF4FF0FF03237023785D
:103A98000A2BFCD144E00CF011FE4FF014004FF05B
:103AA8001E0143F64042C0F601024FF000030BF03E
:103AB80011FF4FF03200014643F62842C0F60102DA
:103AC8004FF000030BF006FF4FF0FF03237023783D
:103AD8000A2BFCD124E040F64C13C2F2000343F851
:103AE80027001DE00CF0EAFD4FF000004FF01E012A
:103AF80043F65042C0F6010203460BF0EBFE4FF0CE
:103B08003200014643F62842C0F601024FF0000396
:103B18000BF0E0FE4FF0FF03237023780A2BFCD153
:103B28004FF0FF0323704FF0010A5346B9F1000F1D
:103B38007FF425A8BAF1000F3DD0012E16D016B19A
:103B4800022E38D125E04FF47844C0F6030420460D
:103B58000BF0C6FA20464FF0000140F64C12C2F2B4
:103B680000024FF012030BF0E5FA24E04FF4704422
:103B7800C0F6030420460BF0B3FA20464FF00001CC
:103B880040F64C12C2F200024FF00C030BF0D2FACE
:103B980011E04FF43044C0F6030420460BF0A0FABD
:103BA80020464FF0000140F64C12C2F200024FF0DE
:103BB80006030BF0BFFA4FF064004FF0010100F06C
:103BC80055FFFEF755FE41F6EF23C2F200034FF012
:103BD800FF021A7011B0BDE8F08F00BF10B582B0B7
:103BE8000CF06CFD4FF000040094204621464FF085
:103BF8007F024FF03F030CF085FB4FF002000146B7
:103C080043F66842C0F6010223460BF063FE0094B7
:103C180020464FF00A014FF07F020B460CF072FB72
:103C280040F29C23C2F200039B68012B10D013B111
:103C3800022B26D119E04FF002004FF00C0143F699
:103C48007C42C0F601024FF000030BF043FE18E07F
:103C58004FF002004FF00C0143F69042C0F601020B
:103C68004FF000030BF036FE0BE04FF002004FF070
:103C78000C0143F6A442C0F601024FF000030BF01A
:103C880029FE43F61454C0F601044FF002004FF029
:103C9800160122464FF000030BF01CFE4FF0020005
:103CA8004FF0200122464FF000030BF013FE4FF0B7
:103CB80002004FF02A0122464FF000030BF00AFEE3
:103CC8004FF0540004F016FF48F68903C8F688033D
:103CD800A3FB0012C2F34F124FF0010400944FF0FF
:103CE80062004FF00C01092A28BF092223460BF075
:103CF80063FE4FF0580004F0FDFE024600944FF0BA
:103D080044004FF00C014FF005030BF055FE41F64F
:103D1800EF23C2F200034FF0FF021A701A4613781D
:103D28000A2BFCD102B010BDF8B506460C4640F28D
:103D3800C003C2F200031B681B7843B143F6B842C4
:103D4800C0F601024FF000030BF0C4FD07E044F693
:103D5800B052C0F601024FF000030BF0BBFD06F1B4
:103D68000807FFB240F2C403C2F200031B681B78C5
:103D780053B13846214643F2E872C0F601024FF0CB
:103D880000030BF0A7FD09E03846214644F6B0527F
:103D9800C0F601024FF000030BF09CFD07F1080587
:103DA800EDB240F2C803C2F200031B681B7853B19E
:103DB8002846214643F65802C0F601024FF0000398
:103DC8000BF088FD09E02846214644F6B052C0F6BB
:103DD80001024FF000030BF07DFD05F10805EDB27F
:103DE80040F2CC03C2F200031B681B7853B128468B
:103DF800214643F66402C0F601024FF000030BF0BF
:103E080069FD09E02846214644F6B052C0F6010291
:103E18004FF000030BF05EFD05F10805EDB240F22E
:103E2800D003C2F200031B681B7853B12846214611
:103E380043F6C802C0F601024FF000030BF04AFD3A
:103E480009E02846214644F6B052C0F601024FF078
:103E580000030BF03FFD05F10805EDB240F2D40375
:103E6800C2F200031B681B7853B12846214643F66B
:103E7800BC42C0F601024FF000030BF02BFD09E035
:103E88002846214644F6B052C0F601024FF000031E
:103E98000BF020FD05F10805EDB240F2D803C2F29F
:103EA80000031B681B7853B12846214643F6C042DD
:103EB800C0F601024FF000030BF00CFD09E02846A4
:103EC800214644F6B052C0F601024FF000030BF051
:103ED80001FD05F10805EDB240F2DC03C2F2000372
:103EE8001B681B7853B12846214643F6C442C0F6E6
:103EF80001024FF000030BF0EDFC09E028462146D3
:103F080044F6B052C0F601024FF000030BF0E2FC99
:103F180005F10805EDB240F2E003C2F200031B68A8
:103F28001B7853B12846214643F6C842C0F6010221
:103F38004FF000030BF0CEFC09E02846214644F67A
:103F4800B052C0F601024FF000030BF0C3FC05F1BC
:103F58000805EDB240F2E403C2F200031B681B78C7
:103F680053B12846214643F6CC42C0F601024FF031
:103F780000030BF0AFFC09E02846214644F6B05296
:103F8800C0F601024FF000030BF0A4FC05F1080590
:103F9800EDB240F2E803C2F200031B681B7853B18C
:103FA8002846214643F6D042C0F601024FF00003EE
:103FB8000BF090FC09E02846214644F6B052C0F6C2
:103FC80001024FF000030BF085FC05F10805EDB286
:103FD80040F2EC03C2F200031B681B7853B1284679
:103FE800214643F6D442C0F601024FF000030BF01D
:103FF80071FC09E02846214644F6B052C0F6010299
:104008004FF000030BF066FC05F10805EDB240F235
:10401800F003C2F200031B681B7853B128462146FF
:1040280043F6D842C0F601024FF000030BF052FCF1
:1040380009E02846214644F6B052C0F601024FF086
:1040480000030BF047FC05F10805E8B240F2F40361
:10405800C2F200031B681B784BB1214643F6DC42D1
:10406800C0F601024FF000030BF034FC08E02146D3
:1040780044F6B052C0F601024FF000030BF02AFCE0
:1040880004F10A04E4B240F2F803C2F200031B6828
:104098001B7853B13046214643F6E042C0F6010290
:1040A8004FF000030BF016FC09E03046214644F6B9
:1040B800B052C0F601024FF000030BF00BFC40F2C7
:1040C800FC03C2F200031B681B7853B13846214633
:1040D80043F6E442C0F601024FF000030BF0FAFB8E
:1040E800F8BD3846214644F6B052C0F601024FF0FA
:1040F80000030BF0EFFBF8BD70B582B004460E4626
:1041080000F10C0044F65055C0F60105C0B22A462D
:104118004FF000030BF0DEFB04F11E00C0B2314685
:104128002A464FF000030BF0D5FB41F61533C2F2D7
:1041380000031A7804F124004FF001050095C0B27D
:1041480031464FF002030BF037FC41F61733C2F249
:1041580000031A7804F112000095C0B231464FF0FE
:1041680002030BF029FC41F60733C2F200031A7868
:104178000095204631464FF002030BF01DFC02B0BB
:1041880070BD00BF30B583B004460D460CF096FAFA
:10419800012C3ED01CB1032C40F06C8106E14FF09D
:1041A8001E004FF00F0143F6E842C0F601024FF03F
:1041B80001030BF08FFB4FF002004FF0280143F68C
:1041C800F042C0F601024FF000030BF083FB4FF002
:1041D80002004FF0320143F60452C0F601024FF0DC
:1041E80000030BF077FB4FF0010200924FF038000C
:1041F8004FF032014FF002030BF0DEFB4FF00001ED
:10420800009108464FF07F024FF03F030CF07AF818
:1042180030E10CF053FA4FF000004FF0020143F682
:104228001852C0F6010203460BF054FB4FF000048D
:10423800009420464FF00B014FF07F020B460CF024
:1042480061F84FF001004FF00D0143F62452C0F61B
:10425800010223460BF03EFB4FF001004FF03701FF
:1042680043F62852C0F6010223460BF033FB4FF009
:1042780016004FF0370143F2E872C0F601022346F8
:104288000BF028FB4FF01F004FF0370143F65802A0
:10429800C0F6010223460BF01DFB4FF028004FF03B
:1042A800370143F66402C0F6010223460BF012FB05
:1042B8004FF031004FF0370143F6C802C0F6010253
:1042C80023460BF007FB4FF03A004FF0370143F657
:1042D800BC42C0F6010223460BF0FCFA4FF0430043
:1042E8004FF0370143F6C042C0F6010223460BF0F7
:1042F800F1FA4FF04C004FF0370143F6C442C0F6D4
:10430800010223460BF0E6FABDBB4FF055004FF013
:10431800020143F62C52C0F6010223460BF0DAFAEA
:104328004FF055004FF0370143F6C842C0F601027E
:1043380023460BF0CFFA4FF05E004FF0370143F6FB
:10434800CC42C0F6010223460BF0C4FA4FF06700D6
:104358004FF0370143F6D042C0F6010223460BF076
:10436800B9FA4FF070004FF0370143F6D442C0F667
:10437800010223460BF0AEFA0AE04FF000004FF0BE
:10438800170143F63452C0F6010203460BF0A2FAB5
:104398004FF0000300934FF00B004FF035014FF042
:1043A80014024FF03F030BF0ADFF63E00CF086F909
:1043B8004FF00F004FF0020143F63852C0F60102E9
:1043C8004FF000030BF086FA4FF0000400942046EB
:1043D8004FF00B014FF07F020B460BF093FF204686
:1043E8004FF00D0143F64852C0F6010223460BF088
:1043F80071FA20464FF0170143F65052C0F60102F9
:1044080023460BF067FA4FF001004FF0370143F6EF
:104418005852C0F6010223460BF05CFA4FF01C001C
:104428004FF0370143F66052C0F6010223460BF005
:1044380051FA4FF02B004FF0370143F66452C0F6A3
:10444800010223460BF046FA4FF03A004FF03701CD
:1044580043F66852C0F6010223460BF03BFA00947B
:104468004FF00B004FF035014FF019024FF03F03AA
:104478000BF048FF03B030BD2DE9F04F85B04FF089
:1044880001004FF00001FFF77DFE4FF00006009697
:104498004FF00B004FF035014FF014024FF03F037F
:1044A8000BF030FF41F6EF23C2F200034FF0FF029A
:1044B8001A704FF0010A1C4641F60C35C2F200058D
:1044C80048F21F5BC5F2EB1B23780C2B22D141F27B
:1044D800D7104FF6FF714FF0010206F0B5FB18B187
:1044E8004FF00200FEF7EAFA4FF001004FF000012A
:1044F800FFF748FE4FF0000300934FF00B004FF01A
:1045080035014FF014024FF03F030BF0FBFE4FF064
:10451800FF03237023780A2B02BFFF2323704FF079
:10452800000A4FF00F004FF00D01FFF7FDFB4FF0B1
:1045380050004FF02301FFF7DFFD2B6813F5004F04
:104548000CD14FF056004FF0170143F64432C0F635
:1045580001024FF000030BF0BDF950E02B6813F493
:10456800004F11D04FF044004FF0170143F66C5242
:10457800C0F601024FF000030BF0ACF92F68C7F149
:1045880000091FFA89F90EE04FF044004FF01701B7
:1045980043F67452C0F601024FF000030BF09AF98B
:1045A8002F681FFA87F9ABFB09274FEA57174FF017
:1045B8000108CDF800804FF05C004FF017013A4633
:1045C8004FF002030BF0F8F94FF068004FF01701B5
:1045D80044F68062C0F601024FF000030BF07AF94E
:1045E8004FF0640303FB1797CDF800804FF06E007F
:1045F8004FF01701BAB24FF002030BF0DDF9237840
:104608000E2B2DD106EBC602D2B202F10B0002F13D
:1046180014024FF001030093C0B24FF03501D2B23B
:104628004FF03F030BF06EFE1EB106F1FF36F6B2F7
:1046380001E04FF00B0606EBC602D2B202F10B0006
:1046480002F114024FF000030093C0B24FF035019D
:10465800D2B24FF03F030BF055FE4FF0FF0323702B
:104668002378132B2CD106EBC602D2B202F10B0031
:1046780002F114024FF001030093C0B24FF035016C
:10468800D2B24FF03F030BF03DFE06F10106F6B241
:104698000B2E88BF002606EBC602D2B202F10B0031
:1046A80002F114024FF000030093C0B24FF035013D
:1046B800D2B24FF03F030BF025FE4FF0FF032370FB
:1046C80023780B2B02D023780D2B64D123780B2B66
:1046D80014BF002301230B2E5AD8DFE806F0060D7D
:1046E800141B222930373E454C5340F20002C2F2D7
:1046F8000002126813704BE040F20402C2F200029A
:104708001268137044E040F20802C2F20002126814
:1047180013703DE040F20C02C2F2000212681370FE
:1047280036E040F21002C2F20002126813702FE065
:1047380040F21402C2F200021268137028E040F23C
:104748001802C2F200021268137021E040F21C0243
:10475800C2F20002126813701AE040F22002C2F29C
:1047680000021268137013E040F22402C2F2000241
:10477800126813700CE040F22802C2F200021268BC
:10478800137005E040F22C02C2F2000212681370A6
:104798004FF0FF0323704FF004038DF80C304FF0F7
:1047A80000038DF80D3040F20003C2F200031B68CD
:1047B8001B784BB14FF00D004FF02C0103AA4FF0BE
:1047C80000030BF087F80BE04FF00D004FF02C01C1
:1047D80044F6B052C0F601024FF000030BF07AF82D
:1047E80040F20403C2F200031B681B784BB14FF080
:1047F80016004FF02C0103AA4FF000030BF06AF8E3
:104808000BE04FF016004FF02C0144F6B052C0F602
:1048180001024FF000030BF05DF840F20803C2F20A
:1048280000031B681B784BB14FF01F004FF02C01A1
:1048380003AA4FF000030BF04DF80BE04FF01F00F8
:104848004FF02C0144F6B052C0F601024FF00003BD
:104858000BF040F840F20C03C2F200031B681B780F
:104868004BB14FF028004FF02C0103AA4FF0000382
:104878000BF030F80BE04FF028004FF02C0144F615
:10488800B052C0F601024FF000030BF023F840F2DB
:104898001003C2F200031B681B784BB14FF03100C4
:1048A8004FF02C0103AA4FF000030BF013F80BE0B4
:1048B8004FF031004FF02C0144F6B052C0F601021F
:1048C8004FF000030BF006F840F21403C2F20003A5
:1048D8001B681B784BB14FF03A004FF02C0103AA2C
:1048E8004FF000030AF0F6FF0BE04FF03A004FF0EC
:1048F8002C0144F6B052C0F601024FF000030AF052
:10490800E9FF40F21803C2F200031B681B784BB1A1
:104918004FF043004FF02C0103AA4FF000030AF0B8
:10492800D9FF0BE04FF043004FF02C0144F6B05292
:10493800C0F601024FF000030AF0CCFF40F21C035E
:10494800C2F200031B681B784BB14FF04C004FF0CC
:104958002C0103AA4FF000030AF0BCFF0BE04FF054
:104968004C004FF02C0144F6B052C0F601024FF053
:1049780000030AF0AFFF40F22003C2F200031B68F5
:104988001B784BB14FF055004FF02C0103AA4FF0A4
:1049980000030AF09FFF0BE04FF055004FF02C0189
:1049A80044F6B052C0F601024FF000030AF092FF3D
:1049B80040F22403C2F200031B681B784BB14FF08E
:1049C8005F004FF02C0103AA4FF000030AF082FFAA
:1049D8000BE04FF05F004FF02C0144F6B052C0F6E8
:1049E80001024FF000030AF075FF40F22803C2F2FB
:1049F80000031B681B784BB14FF068004FF02C0187
:104A080003AA4FF000030AF065FF0BE04FF06800BF
:104A18004FF02C0144F6B052C0F601024FF00003EB
:104A28000AF058FF40F22C03C2F200031B681B78FF
:104A38004BB14FF071004FF02C0103AA4FF0000367
:104A48000AF048FF0BE04FF071004FF02C0144F6DC
:104A5800B052C0F601024FF000030AF03BFFBAF172
:104A6800000F7FF431AD05B0BDE8F08F41F253136C
:104A7800C2F200034FF000021A7041F24E12C2F265
:104A8800000210804FF001021A701A4613780BB119
:104A98000029FBD1704700BF704700BFFEE700BF89
:104AA800FEE700BFFEE700BFFEE700BF704700BF9C
:104AB800704700BF704700BF70B582B00AF084FB32
:104AC8000BF008FB4FF000038DF805304FF4406001
:104AD800C4F201004FF4006102F0AEFF28B19DF866
:104AE800053043F080038DF805304FF4C050C4F210
:104AF80001004FF4004102F0DBFF4FF000038DF896
:104B080007309DF80730132B0AD89DF8073003F1BA
:104B18000103DBB28DF807309DF80730132BF4D969
:104B28004FF4C050C4F201004FF4004102F0B2FF4C
:104B380040F29C13C2F200031B788DF806304FF048
:104B480000038DF804309DF80430072B57D84FF434
:104B58004064C4F201044FF480654FF000069DF8EC
:104B6800063013F0010F04D02046294602F092FFC8
:104B780003E02046294602F09BFF9DF805304FEAE6
:104B880053038DF8053020464FF4006102F054FFBE
:104B980028B19DF8053043F080038DF80530204694
:104BA8004FF4805102F084FF8DF807609DF80730BC
:104BB800092B0AD89DF8073003F10103DBB28DF801
:104BC80007309DF80730092BF4D920464FF480515F
:104BD80002F060FF2046294602F06AFF9DF8063081
:104BE8004FEA53038DF806309DF8043003F10103B2
:104BF800DBB28DF804309DF80430072BAFD99DF84F
:104C0800052040F2A013C2F200031A7009F0D6FD85
:104C180000F076FA41F24D13C2F200031A7802F15D
:104C28000102D2B21A701B78322B0DD940F640130C
:104C3800C2F200034FF001021A7041F24D13C2F2A2
:104C480000034FF000021A7041F25313C2F200033E
:104C58001B78BBB141F24E13C2F200031B889BB212
:104C68004BB141F24E13C2F200031A8802F1FF322F
:104C780092B21A8006E041F25313C2F200034FF0D9
:104C880000021A7002B070BD704700BF704700BFC5
:104C9800704700BF0000000038B54FF0010003F076
:104CA800B3FE002800F02A814FF0010003F0DEFE79
:104CB80003F07CFE40F28A13C2F200031B78002B3B
:104CC8007ED003F01BFE044645F27E13C0F20103BA
:104CD800984228D945F27F13C0F20103984283BF56
:104CE800A0F5A834A4F5BE74033C002440F28A134E
:104CF800C2F200034FF001025A7040F21C43C2F2A4
:104D080000039B68092B9FBFE41840F28A13C2F284
:104D18000003002298BF5A70204603F00DFE03F0EE
:104D280045FE0AF02FF90A2C16D140F28A13C2F276
:104D380000035B7883B140F21C43C2F200039C6815
:104D480004F10A04204603F0F7FD40F28A13C2F288
:104D580000034FF000025A704BF2C532C9F2A2129A
:104D6800A2FB04124FEAD222D1B241F60733C2F2B3
:104D7800000319704FF4616101FB124448F689027F
:104D8800C8F68802A2FB04124FEA5212D1B241F6C9
:104D98001735C2F200052970C2EB0212A4EB820497
:104DA800E4B241F61532C2F20002147019784FF0DD
:104DB800A80003F083FE29784FF0A40003F07EFEDC
:104DC80040F2A413C2F200031B78BBB141F61033C2
:104DD800C2F200031A7841F61733C2F200031B78B7
:104DE8009A420BD041F61733C2F200031A7841F603
:104DF8001033C2F200031A7007F068FE02F01AFBC3
:104E08004FF41055C4F20105284604F07DFC41F624
:104E18000434C2F20004208028464FF010014FF0FD
:104E280001024FF0070304F087FB208880B240F2AC
:104E38001C43C2F200035B68C018FBF771FEFBF766
:104E480033FB2FA3D3E90023FBF782FBFBF792FD8B
:104E580041F60C33C2F2000318601A6842F69763F1
:104E6800C0F202039A421CD841F60C34C2F2000484
:104E78002368C3F50A3303F5D36323602068FBF77F
:104E88004FFEFBF711FB20A3D3E90023FBF78AFCB5
:104E98001FA3D3E90023FBF7A9F9FBF76BFD2060FB
:104EA80038BD41F60C34C2F200042368A3F50A3376
:104EB800A3F5D36323602068FBF732FEFBF7F4FA0F
:104EC80011A3D3E90023FBF76DFCFBF753FD20602A
:104ED800226840F6C4139A4206D92268C2F51C62B9
:104EE80002F10402226038BD41F60C33C2F200031D
:104EF8001A68C2F51C6202F104021A6038BD00BFCC
:104F08003333333333335440333333333333114050
:104F1800000000000088A340704700BF704700BF32
:104F2800704700BF704700BF704700BF704700BFA1
:104F3800704700BF704700BF704700BF704700BF91
:104F4800704700BF704700BF704700BF704700BF81
:104F5800704700BF704700BF08B54FF080404FF062
:104F6800010104F0B0F94FF43053C4F200031B6898
:104F780003F07F034D2B03D84FF07F0005F06CFD45
:104F880000F0BCF809F012F840F29C23C2F20003CA
:104F98001B69002B3BD0282B81BF40F29C23C2F217
:104FA800000328221A6141F60C33C2F200031A6882
:104FB80040F29C23C2F200031B694FF0640101FB1D
:104FC80003F393421AD94FF4C050C4F201004FF0D2
:104FD800100102F031FD40B94FF4C050C4F2010095
:104FE8004FF0100102F056FD19E04FF4C050C4F222
:104FF80001004FF0100102F05BFD10E04FF4C050CB
:10500800C4F201004FF0100102F052FD07E04FF426
:10501800C050C4F201004FF0100102F049FD4FF4F6
:105028000060C4F201004FF0040102F005FD38B938
:1050380041F62533C2F200034FF000021A7008BD92
:1050480041F62533C2F200034FF001021A7008BD81
:1050580008B54FF48060C4F200004FF0010104F07D
:1050680032F900F06BF908BD08B54FF40060C4F2DE
:1050780000004FF0010104F026F908BD704700BF99
:10508800704700BF704700BF704700BF704700BF40
:10509800704700BF704700BF704700BF704700BF30
:1050A80008B54FF49840C4F2000040F2255102F0D0
:1050B8005DFF38B14FF49840C4F2000040F225512A
:1050C80002F0BAFF4FF49840C4F2000040F22661A3
:1050D80002F04CFF38B14FF49840C4F2000040F29F
:1050E800266102F0A9FF08BD08B54FF4805003F00F
:1050F8009BFE08BD704700BF704700BF704700BFE8
:1051080040F2C623C2F200031B78002B39D041F2CB
:105118009013C2F200031B78002B39D041F2901390
:10512800C2F200034FF000021A7041F29B13C2F260
:1051380000031B78C3B141F29B13C2F200031A703B
:1051480041F27A13C2F200031A7841F28413C2F2D0
:1051580000031A6041F28C13C2F200031A6841F28C
:105168007413C2F200031A6041F27A13C2F2000308
:105178004FF000021A7041F28C13C2F200031A6059
:1051880006E041F29013C2F200034FF001021A70D8
:1051980041F28C13C2F200031A6802F101021A608C
:1051A8001B68B3F57A7F81BF41F27413C2F2000322
:1051B80000221A6041F27A13C2F200031A7802F14F
:1051C8000102D2B21A701A7841F28413C2F20003B3
:1051D8001B689A4209D941F27A13C2F200031A787D
:1051E80041F28413C2F200031A6041F62823C2F286
:1051F80000035A69002A5DD040F28C13C2F2000302
:105208001B78002B40D041F28413C2F200031B68C4
:105218000A2B4FD941F28413C2F200031B684EF6E1
:105228006021B1FBF3F39A421AD941F28113C2F219
:1052380000031A7802F10102D2B21A7041F2551233
:10524800C2F200024FF0000111701B78C82B31D94F
:1052580040F28C13C2F200034FF001025A707047FB
:1052680041F25513C2F200031A7802F10102D2B2D8
:105278001A701B78C82B1DD941F28113C2F20003A2
:105288004FF000021A70704741F28412C2F2000215
:105298004FF00003136041F27A12C2F20002137059
:1052A80041F28112C2F20002137040F28C12C2F273
:1052B80000025370704700BF10B541F29813C2F254
:1052C80000034FF000041C704FF00400214603F067
:1052D800F5FB40F2CE23C2F200031C7040F28C139F
:1052E800C2F200031C7041F29913C2F200031C7051
:1052F8004FF00C00214603F0E1FB40F2BB13C2F271
:1053080000031C7041F28013C2F200031C704FF0BE
:105318001400214603F0D2FB40F2B233C2F200037C
:105328001C7041F25413C2F200031C704FF01C00B1
:10533800214603F0C3FB08F015FD10BDF0B583B09E
:1053480041F62533C2F200031B78012B40F0BE80E2
:1053580040F28C13C2F200039B78002B00F0B68059
:105368004FF0240003F0C6FB044610F0010F22D1D1
:1053780040F29D13C2F200031B78E3B140F29D1680
:10538800C2F20006317801F1FF314FF000050095B7
:1053980001954FF00100C9B22A462B4604F00CFAD9
:1053A800357044F00104A4B24FF02400214603F004
:1053B80085FBFFF781FF14F0080F2DD140F2C723BA
:1053C800C2F200031B7803BB40F28C13C2F2000345
:1053D800DA7802F10102D2B2DA70DB78322B1BD90B
:1053E800FFF76AFF4FF00003009301934FF00800A6
:1053F80019461A4604F0E0F944F00804A4B24FF044
:105408002400214603F05AFB06E040F28C13C2F256
:1054180000034FF00002DA7014F0200F34D140F28C
:105428001643C2F200031B783BBB40F2C723C2F20B
:1054380000031B78012B20D140F28C13C2F2000329
:105448001A7902F10102D2B21A711B79322B1BD9D7
:10545800FFF732FF4FF00003009301934FF00C0069
:1054680019461A4604F0A8F944F02004A4B24FF0F3
:105478002400214603F022FB06E040F28C13C2F21E
:1054880000034FF000021A7140F28C13C2F20003BD
:105498001B78DBB114F0100F18D140F28C13C2F254
:1054A80000035B7893B1FFF707FF4FF00003009309
:1054B80001934FF01A0019461A4604F07DF944F09A
:1054C80010014FF0240089B203F0F8FA40F2881373
:1054D800C2F200031B78012B40F0498441F62533C2
:1054E800C2F200031B78012B40F0418441F298136B
:1054F800C2F200031B78032B00F03F8104D8012B74
:105508000CD03DD800F033BCC82B00F02D83C92B3C
:1055180000F03983042B40F01F8465E241F25413F4
:10552800C2F200031B7833B141F25413C2F20003F4
:105538004FF000021A7041F28813C2F200034FF0D4
:1055480001021A7041F27C13C2F200034FF000010D
:10555800196041F25813C2F2000319604FF0440079
:1055680003F0ACFA4FF004004FF0020103F0A6FA82
:1055780041F29813C2F200034FF002021A70F6E3E8
:1055880041F28813C2F200031B78002B00F09780C9
:1055980041F28813C2F200034FF000021A7040F281
:1055A8009C23C2F200039B68012B1CD013B1022B71
:1055B8004AD131E043F67C50C0F6010041F64C3147
:1055C800C2F200014FF0130208F08AFA43F6945031
:1055D800C0F6010041F63431C2F200014FF0130267
:1055E80008F07EFA30E043F6AC50C0F6010041F610
:1055F8004C31C2F200014FF0130208F071FA43F681
:10560800C450C0F6010041F63431C2F200014FF037
:10561800130208F065FA17E043F6DC50C0F6010003
:1056280041F64C31C2F200014FF0130208F058FA6B
:1056380043F69450C0F6010041F63431C2F200013D
:105648004FF0130208F04CFA43F6F450C0F601008C
:1056580041F69431C2F200014FF0130208F040FA0B
:1056680043F60C60C0F6010041F67C31C2F200013D
:105678004FF0130208F034FA43F62460C0F6010034
:1056880041F66431C2F200014FF0130208F028FA23
:1056980040F2CE23C2F200034FF001021A7041F229
:1056A8007C13C2F200034FF000021A604FF044006E
:1056B80003F020FA41F25813C2F20003186041F2D5
:1056C8007C13C2F200031A6802F101021A601B6817
:1056D8000A2B81BF40F28C13C2F2000301221A7018
:1056E80041F25814C2F20004236803F10103236055
:1056F80021684FF0440089B203F0E0F922684CF6C3
:10570800CD43CCF6CC43A3FB02134FF00402009226
:105718004FEAD300CE494FF00002134608F08EFA44
:10572800226841F62823C2F200031B6903EB8303B6
:10573800B2EB430FC0F01B8341F27C13C2F20003AB
:105748004FF00001196021604FF0440003F0B6F9F2
:1057580041F28813C2F200034FF001021A704FF0B1
:1057680004004FF0030103F0A9F941F29813C2F2C3
:1057780000034FF003021A70F9E241F28813C2F2F3
:1057880000031B78002B00F0978041F28813C2F2C7
:1057980000034FF000021A7040F29C23C2F200038B
:1057A8009B68012B1CD013B1022B4AD131E043F680
:1057B8003C60C0F6010041F64C31C2F200014FF0E6
:1057C800130208F08DF943F60C60C0F6010041F6AB
:1057D8003431C2F200014FF0130208F081F930E0D1
:1057E80043F65460C0F6010041F64C31C2F20001A4
:1057F8004FF0130208F074F943F60C60C0F601008C
:1058080041F63431C2F200014FF0130208F068F992
:1058180017E043F66C60C0F6010041F64C31C2F265
:1058280000014FF0130208F05BF943F60C60C0F674
:10583800010041F63431C2F200014FF0130208F0C2
:105848004FF943F68460C0F6010041F69431C2F284
:1058580000014FF0130208F043F943F60C60C0F65C
:10586800010041F67C31C2F200014FF0130208F04A
:1058780037F943F69C60C0F6010041F66431C2F284
:1058880000014FF0130208F02BF940F2CE23C2F2C8
:1058980000034FF001021A7041F27C13C2F20003B8
:1058A8004FF000021A604FF0440003F023F941F270
:1058B8005813C2F20003186041F27C13C2F20003CD
:1058C8001A6802F101021A601B680A2B81BF40F2B4
:1058D8008C13C2F2000301221A7041F25814C2F26A
:1058E8000004236803F10103236021684FF044009A
:1058F80089B203F0E3F822684CF6CD43CCF6CC43EA
:10590800A3FB02134FF0040200924FEAD300504960
:105918004FF00002134608F091F9226841F6282357
:10592800C2F20003DB6803EB8303B2EB430F2ED311
:1059380041F27C13C2F200034FF000041C6041F2F4
:105948005813C2F200031C604FF04400214603F0D4
:10595800B5F841F28813C2F200034FF001021A7041
:105968004FF00400014603F0A9F841F29813C2F27F
:1059780000034FF004021A70009401944FF01500D0
:1059880021462246234603F017FFFFF795FC40F215
:10599800C523C2F200031B78002B00F0E88140F217
:1059A8008C13C2F200034FF000021A7040F2CE23AB
:1059B800C2F200031A7041F27C13C2F200031A60AB
:1059C80041F28813C2F200034FF001021A704FF03F
:1059D8000400014603F072F841F29813C2F2000382
:1059E8004FF004021A70C2E141F28813C2F20003B8
:1059F8001B78002B00F08D8041F28813C2F200035F
:105A08004FF000021A7040F29C23C2F200039B6818
:105A1800012B1FD013B1022B4DD134E043F6B460F3
:105A2800C0F6010041F64C31C2F200014FF01302FA
:105A380008F056F843F6CC60C0F6010041F6343160
:105A4800C2F200014FF0130208F04AF833E000BF39
:105A5800A11B002043F6B460C0F6010041F64C31AA
:105A6800C2F200014FF0130208F03AF843F6E4607E
:105A7800C0F6010041F63431C2F200014FF01302C2
:105A880008F02EF817E043F6FC60C0F6010041F676
:105A98004C31C2F200014FF0130208F021F843F62E
:105AA8001470C0F6010041F63431C2F200014FF023
:105AB800130208F015F843F60C64C0F601042046FA
:105AC80041F69431C2F200014FF0130208F008F8D1
:105AD800204641F67C31C2F200014FF0130207F074
:105AE800FFFF43F62C70C0F6010041F66431C2F2A4
:105AF80000014FF0130207F0F3FF40F2CE23C2F289
:105B080000034FF000021A7041F27C13C2F2000346
:105B18001A6041F27C13C2F200031A6802F1010212
:105B28001A601B681E2B40F222814FF01C0002F005
:105B3800E1FFC0B241F25413C2F20003187041F2FF
:105B48007913C2F200034FF001021A704FF00400FB
:105B58004FF0000102F0B2FF41F29813C2F20003C5
:105B68004FF000021A7002E141F28813C2F20003FA
:105B78004FF001021A7041F29813C2F200034FF07D
:105B8800C9021A70F3E041F28813C2F200031B78CD
:105B9800002B00F0968041F28813C2F200034FF008
:105BA80000021A7040F29C23C2F200039B68012B8A
:105BB8001CD013B1022B4AD131E043F64470C0F631
:105BC800010041F64C31C2F200014FF0130207F018
:105BD80087FF43F67C50C0F6010041F63431C2F22B
:105BE80000014FF0130207F07BFF30E043F65C70D2
:105BF800C0F6010041F64C31C2F200014FF0130229
:105C080007F06EFF43F67470C0F6010041F63431B8
:105C1800C2F200014FF0130207F062FF17E043F6EB
:105C28008C70C0F6010041F64C31C2F200014FF011
:105C3800130207F055FF43F67C50C0F6010041F609
:105C48003431C2F200014FF0130207F049FF43F666
:105C58000C64C0F60104204641F69431C2F20001FA
:105C68004FF0130207F03CFF204641F67C31C2F2A8
:105C780000014FF0130207F033FF43F62460C0F62B
:105C8800010041F66431C2F200014FF0130207F03F
:105C980027FF40F2CE23C2F200034FF000021A7031
:105CA80040F69903C2F200034FF00101197041F266
:105CB8007C13C2F200031A6041F25813C2F20003C7
:105CC8001A6041F27C13C2F200031A6802F1010261
:105CD8001A601B680A2B21D941F27C13C2F2000317
:105CE8004FF000021A6040F69903C2F200031B78D5
:105CF8006BB140F69903C2F200031A7041F25813CF
:105D0800C2F200031A6802F101021A6006E040F6C6
:105D18009903C2F200034FF001021A7041F25813BE
:105D2800C2F200031B68032B21D941F28813C2F287
:105D380000034FF001021A704FF0080002F0DAFE7B
:105D4800C0B241F29813C2F20003187019784FF0EC
:105D5800040002F0B3FE0AE041F29813C2F2000315
:105D68004FF0000119704FF0040002F0A7FE40F256
:105D78008813C2F200031B78022B40F0CD8341F652
:105D88002533C2F200031B78012B40F0C58341F292
:105D98009913C2F200031B78032B00F0048103D887
:105DA800012B0BD02FD8B7E3C82B00F0B082C92B3A
:105DB80000F0BC82042B40F0A483FCE141F289137B
:105DC800C2F200034FF001021A7041F27C13C2F2D2
:105DD80000034FF00001196041F25813C2F20003AA
:105DE80019604FF0440002F069FE4FF00C004FF0CC
:105DF800020102F063FE41F29913C2F200034FF070
:105E080002021A7088E341F28913C2F200031B7878
:105E1800002B00F08C8041F28913C2F200034FF08E
:105E280000021A7040F29C23C2F200039B68012B07
:105E38001CD013B1022B4AD131E043F67C50C0F696
:105E4800010041F64C31C2F200014FF0130207F095
:105E580047FE43F6A470C0F6010041F63431C2F2A1
:105E680000014FF0130207F03BFE30E043F6AC5060
:105E7800C0F6010041F64C31C2F200014FF01302A6
:105E880007F02EFE43F6A470C0F6010041F6343147
:105E9800C2F200014FF0130207F022FE17E043F6AA
:105EA8007C50C0F6010041F64C31C2F200014FF0BF
:105EB800130207F015FE43F6BC70C0F6010041F668
:105EC8003431C2F200014FF0130207F009FE43F625
:105ED8000C64C0F60104204641F69431C2F2000178
:105EE8004FF0130207F0FCFD204641F67C31C2F268
:105EF80000014FF0130207F0F3FD43F62460C0F6EB
:105F0800010041F66431C2F200014FF0130207F0BC
:105F1800E7FD40F2BB13C2F200034FF001021A7012
:105F280041F27C13C2F200034FF000021A6041F202
:105F38007C13C2F200031A6802F101021A601B689E
:105F48001E2B40F2E98241F27C13C2F200034FF0AB
:105F580000021A6041F62823C2F200039B684FF43E
:105F6800167202FB03F241F25813C2F200031A60E0
:105F780019684FF0440089B202F0A0FD41F289137C
:105F8800C2F200034FF001021A704FF00C004FF0FC
:105F9800030102F093FD41F29913C2F200034FF09E
:105FA80003021A70B8E241F28913C2F200031B78A7
:105FB800002B00F0978041F28913C2F200034FF0E2
:105FC80000021A7040F29C23C2F200039B68012B66
:105FD8001CD013B1022B4AD131E043F6D470C0F67D
:105FE800010041F64C31C2F200014FF0130207F0F4
:105FF80077FD43F6EC70C0F6010041F63431C2F289
:1060080000014FF0130207F06BFD30E044F204008A
:10601800C0F6010041F64C31C2F200014FF0130204
:1060280007F05EFD43F6EC70C0F6010041F634312E
:10603800C2F200014FF0130207F052FD17E044F2DC
:106048001C00C0F6010041F64C31C2F200014FF0CD
:10605800130207F045FD44F23400C0F6010041F692
:106068003431C2F200014FF0130207F039FD44F257
:106078004C00C0F6010041F69431C2F200014FF025
:10608800130207F02DFD43F60C60C0F6010041F63F
:106098007C31C2F200014FF0130207F021FD43F6F4
:1060A8009C60C0F6010041F66431C2F200014FF075
:1060B800130207F015FD40F2BB13C2F200034FF0C4
:1060C80001021A7041F27C13C2F200034FF0000281
:1060D8001A604FF0440002F00DFD41F25813C2F26D
:1060E8000003186041F25813C2F200031B68002B2A
:1060F80040D041F25814C2F20004236803F1FF3380
:10610800236021684FF0440089B202F0D7FC206870
:1061180048F2B515C1F64E35A5FB0020A94F4FF042
:10612800020600964FEA901039464FF000021346D7
:1061380007F084FD2368A5FB03124FEA92124FF47F
:10614800167101FB123241F29413C2F200031A6075
:106158001A684CF6CD43CCF6CC43A3FB0213009649
:106168004FEAD30007F103014FF00002134607F08E
:1061780065FDD1E140F2BB13C2F200034FF000020B
:106188001A7041F27C13C2F200031A6041F28913BB
:10619800C2F200034FF001021A704FF00C004FF0EA
:1061A800040102F08BFC41F29913C2F200034FF094
:1061B80004021A70B0E141F28913C2F200031B789D
:1061C800002B00F08A8041F28913C2F200034FF0DD
:1061D80000021A7040F29C23C2F200039B68012B54
:1061E8001CD013B1022B4AD131E043F6B460C0F69B
:1061F800010041F64C31C2F200014FF0130207F0E2
:106208006FFC44F26400C0F6010041F63431C2F27A
:1062180000014FF0130207F063FC30E043F6B4606E
:10622800C0F6010041F64C31C2F200014FF01302F2
:1062380007F056FC44F26400C0F6010041F6343120
:10624800C2F200014FF0130207F04AFC17E044F2D3
:106258007C00C0F6010041F64C31C2F200014FF05B
:10626800130207F03DFC44F29400C0F6010041F629
:106278003431C2F200014FF0130207F031FC43F64B
:106288000C64C0F60104204641F69431C2F20001C4
:106298004FF0130207F024FC204641F67C31C2F28D
:1062A80000014FF0130207F01BFC43F62C70C0F6F8
:1062B800010041F66431C2F200014FF0130207F009
:1062C8000FFC40F2BB13C2F200034FF000021A7039
:1062D80041F27C13C2F200031A6041F27C13C2F24D
:1062E80000031A6802F101021A601B681E2B40F2B3
:1062F80013814FF00C004FF0000102F0DFFB41F278
:106308009913C2F200034FF000021A7004E141F23F
:106318008913C2F200034FF001021A7041F2991377
:10632800C2F200034FF0C9021A70F5E041F2891376
:10633800C2F200031B78002B00F0988041F2891309
:10634800C2F200034FF000021A7040F29C23C2F21E
:1063580000039B68012B1CD013B1022B4CD133E0F6
:1063680043F64470C0F6010041F64C31C2F2000118
:106378004FF0130207F0B4FB43F67C50C0F601005F
:1063880041F63431C2F200014FF0130207F0A8FBC6
:1063980032E044F2AC00C0F6010041F64C31C2F2E2
:1063A80000014FF0130207F09BFB43F6AC50C0F618
:1063B800010041F63431C2F200014FF0130207F038
:1063C8008FFB19E0A01B002044F2C400C0F60100B6
:1063D80041F64C31C2F200014FF0130207F080FB86
:1063E80043F67C50C0F6010041F63431C2F2000198
:1063F8004FF0130207F074FB43F60C64C0F6010477
:10640800204641F69431C2F200014FF0130207F022
:1064180067FB204641F67C31C2F200014FF01302BF
:1064280007F05EFB44F2DC00C0F6010041F664317F
:10643800C2F200014FF0130207F052FB40F2BB1307
:10644800C2F200034FF000021A7040F69903C2F23C
:1064580000034FF00101197041F27C13C2F20003EE
:106468001A6041F25813C2F200031A6041F27C1319
:10647800C2F200031A6802F101021A601B680A2BB3
:1064880021D941F27C13C2F200034FF000021A60D6
:1064980040F69903C2F200031B786BB140F69903EA
:1064A800C2F200031A7041F25813C2F200031A68CC
:1064B80002F101021A6006E040F69903C2F20003F5
:1064C8004FF001021A7041F25813C2F200031B6820
:1064D800032B21D941F28913C2F200034FF00102C4
:1064E8001A704FF0100002F005FBC0B241F2991388
:1064F800C2F20003187019784FF00C0002F0DEFAAF
:106508000AE041F29913C2F200034FF0000119703A
:106518004FF00C0002F0D2FA40F28813C2F20003E6
:106528001B78032B40F0C28441F62533C2F20003E6
:106538001B78012B40F0BA8441F28013C2F20003A9
:106548001B78032B00F0348104D8012B0ED03ED8E1
:1065580000F0ACBC052B00F0F282C0F0FC81C82B27
:1065680000F09E83C92B40F09684A8E341F278138B
:10657800C2F200034FF001021A7041F27C13C2F21A
:1065880000034FF000021A6041F62823C2F200030C
:106598005B6803EB83034FEA430241F25813C2F2EC
:1065A80000031A6019684FF0440089B202F086FAB5
:1065B8004FF014004FF0020102F080FA41F280130C
:1065C800C2F200034FF002021A7000F06FBC41F2F1
:1065D8007813C2F200031B78002B00F09C8041F274
:1065E8007813C2F200034FF000021A7040F29C23A5
:1065F800C2F200039B68012B1CD013B1022B4AD1B5
:1066080031E043F67C50C0F6010041F64C31C2F24D
:1066180000014FF0130207F063FA44F2F400C0F6E9
:10662800010041F63431C2F200014FF0130207F0C5
:1066380057FA30E044F20C10C0F6010041F64C3134
:10664800C2F200014FF0130207F04AFA44F2241094
:10665800C0F6010041F63431C2F200014FF01302D6
:1066680007F03EFA17E044F23C10C0F6010041F68C
:106678004C31C2F200014FF0130207F031FA44F234
:106688005410C0F6010041F63431C2F200014FF057
:10669800130207F025FA44F26C10C0F6010041F627
:1066A8009431C2F200014FF0130207F019FA43F6D1
:1066B8000C60C0F6010041F67C31C2F200014FF0D7
:1066C800130207F00DFA43F62460C0F6010041F604
:1066D8006431C2F200014FF0130207F001FA40F2F0
:1066E800B233C2F200034FF001021A7040F2B52330
:1066F800C2F200034FF000021A7041F27C13C2F29A
:1067080000031A604FF0440002F0F4F941F2581304
:10671800C2F20003186041F25813C2F200031B686A
:1067280003B341F25814C2F20004236803F1FF33A3
:10673800236021684FF0440089B202F0BFF9226853
:106748004CF6CD43CCF6CC43A3FB02134FF0020228
:1067580000924FEAD300A6494FF00002134607F013
:106768006DFAA3E340F2B233C2F200034FF0000225
:106778001A7040F2B523C2F200031A7041F27C137A
:10678800C2F200031A6041F27813C2F200034FF01C
:1067980001021A704FF014004FF0030102F08EF955
:1067A80041F28013C2F200034FF003021A707DE336
:1067B80041F27813C2F200031B78002B00F091809D
:1067C80041F27813C2F200034FF000021A7040F24F
:1067D8009C23C2F200039B68012B1CD013B1022B2F
:1067E8004AD131E044F28410C0F6010041F64C3140
:1067F800C2F200014FF0130207F072F943F60C6081
:10680800C0F6010041F63431C2F200014FF0130224
:1068180007F066F930E044F20C10C0F6010041F6CA
:106828004C31C2F200014FF0130207F059F944F25B
:106838009C10C0F6010041F63431C2F200014FF05D
:10684800130207F04DF917E043F6DC50C0F60100DB
:1068580041F64C31C2F200014FF0130207F040F943
:1068680044F2B410C0F6010041F63431C2F200011E
:106878004FF0130207F034F943F60C64C0F6010434
:10688800204641F69431C2F200014FF0130207F09E
:1068980027F9204641F67C31C2F200014FF013027D
:1068A80007F01EF943F62460C0F6010041F6643192
:1068B800C2F200014FF0130207F012F940F2B233AE
:1068C800C2F200034FF000021A7040F2B523C2F280
:1068D80000034FF00101197041F27C13C2F200036A
:1068E8001A6041F27C13C2F200031A6802F1010235
:1068F8001A601B681E2B40F2D98241F27C13C2F247
:1069080000034FF000021A6040F2B523C2F2000300
:106918004FF001041C7041F25813C2F200034FF00B
:1069280096021A6019684FF0440089B202F0C6F85E
:1069380041F27813C2F200031C704FF014004FF0BC
:10694800040102F0BBF841F28013C2F200034FF0D9
:1069580004021A70AAE241F27813C2F200031B780B
:10696800002B00F09F8041F27813C2F200034FF031
:1069780000021A7040F29C23C2F200039B68012BAC
:106988001CD013B1022B4DD134E043F6D470C0F6BD
:10699800010041F64C31C2F200014FF0130207F03A
:1069A8009FF844F2CC10C0F6010041F63431C2F22F
:1069B80000014FF0130207F093F833E044F20400AB
:1069C800C0F6010041F64C31C2F200014FF013024B
:1069D80007F086F844F2E410C0F6010041F63431BD
:1069E800C2F200014FF0130207F07AF81AE000BF74
:1069F800A31B002044F2FC10C0F6010041F64C3104
:106A0800C2F200014FF0130207F06AF844F21420B2
:106A1800C0F6010041F63431C2F200014FF0130212
:106A280007F05EF844F26C10C0F6010041F69431AC
:106A3800C2F200014FF0130207F052F843F60C605F
:106A4800C0F6010041F67C31C2F200014FF013029A
:106A580007F046F843F69C60C0F6010041F6643141
:106A6800C2F200014FF0130207F03AF840F2B233D5
:106A7800C2F200034FF001021A7040F2B523C2F2CD
:106A880000031A7041F27C13C2F200034FF00002B7
:106A98001A604FF0440002F02DF841F25813C2F288
:106AA8000003186041F25813C2F200031B6803B3D5
:106AB80041F25814C2F20004236803F1FF33236043
:106AC80021684FF0440089B201F0F8FF22684CF6C3
:106AD800CD43CCF6CC43A3FB02134FF00202009245
:106AE8004FEAD3009C494FF00002134607F0A6F87E
:106AF800DCE140F2B233C2F200034FF000021A7038
:106B080040F2B523C2F200031A7041F27C13C2F2BC
:106B180000031A6041F27813C2F200034FF0010239
:106B28001A704FF014004FF0050101F0C7FF41F251
:106B38008013C2F200034FF005021A70B6E141F269
:106B48007813C2F200031B78002B00F08F8041F20B
:106B58007813C2F200034FF000021A7040F29C232F
:106B6800C2F200039B68012B1CD013B1022B4AD13F
:106B780031E043F6B460C0F6010041F64C31C2F290
:106B880000014FF0130206F0ABFF44F22C20C0F6D0
:106B9800010041F63431C2F200014FF0130206F051
:106BA8009FFF30E043F6B460C0F6010041F64C3177
:106BB800C2F200014FF0130206F092FF44F24420A3
:106BC800C0F6010041F63431C2F200014FF0130261
:106BD80006F086FF17E044F25C20C0F6010041F69B
:106BE8004C31C2F200014FF0130206F079FF44F273
:106BF8007020C0F6010041F63431C2F200014FF0B6
:106C0800130206F06DFF43F60C64C0F6010420463B
:106C180041F69431C2F200014FF0130206F060FF12
:106C2800204641F67C31C2F200014FF0130206F013
:106C380057FF43F62C70C0F6010041F66431C2F2EA
:106C480000014FF0130206F04BFF40F2B233C2F2DC
:106C580000034FF000021A7040F2B523C2F200039D
:106C68001A7041F27C13C2F200031A6041F27C13DD
:106C7800C2F200031A6802F101021A601B681E2B97
:106C880040F214814FF014004FF0000101F016FF9C
:106C980041F28013C2F200034FF000021A7005E1BE
:106CA80041F27813C2F200034FF001021A7041F268
:106CB8008013C2F200034FF0C9021A70F6E041F2E5
:106CC8007813C2F200031B78002B00F0998041F280
:106CD8007813C2F200034FF000021A7040F29C23AE
:106CE800C2F200039B68012B1CD013B1022B4DD1BB
:106CF80034E043F64470C0F6010041F64C31C2F26C
:106D080000014FF0130206F0EBFE43F67C50C0F68C
:106D1800010041F63431C2F200014FF0130206F0CF
:106D2800DFFE33E043F65C70C0F6010041F64C31FB
:106D3800C2F200014FF0130206F0D2FE44F28420A2
:106D4800C0F6010041F63431C2F200014FF01302DF
:106D580006F0C6FE1AE000BFA31B002044F29C20E8
:106D6800C0F6010041F64C31C2F200014FF01302A7
:106D780006F0B6FE43F67C50C0F6010041F6343109
:106D8800C2F200014FF0130206F0AAFE43F60C64AB
:106D9800C0F60104204641F69431C2F200014FF0DA
:106DA800130206F09DFE204641F67C31C2F2000136
:106DB8004FF0130206F094FE44F2DC00C0F6010026
:106DC80041F66431C2F200014FF0130206F088FE6A
:106DD80040F2B233C2F200034FF000021A7040F6DC
:106DE8009903C2F200034FF00101197041F27C13BC
:106DF800C2F200031A6041F25813C2F200031A608B
:106E080041F27C13C2F200031A6802F101021A600F
:106E18001B680A2B21D941F27C13C2F200034FF000
:106E280000021A6040F69903C2F200031B786BB1A6
:106E380040F69903C2F200031A7041F25813C2F2E5
:106E480000031A6802F101021A6006E040F699038D
:106E5800C2F200034FF001021A7041F25813C2F255
:106E680000031B68032B21D941F27813C2F20003F7
:106E78004FF001021A704FF0180001F03BFEC0B24B
:106E880041F28013C2F20003187019784FF0140011
:106E980001F014FE0AE041F28013C2F200034FF041
:106EA800000119704FF0140001F008FE41F6253377
:106EB800C2F200031B78012B40F0B78241F2541351
:106EC800C2F200031B78052B00F29F82DFE813F063
:106ED800AD0206003600100179019D0141F27913D7
:106EE800C2F200034FF001021A7041F27C13C2F2A1
:106EF80000034FF000021A6041F62823C2F2000393
:106F0800DB694FF4167202FB03F241F25813C2F226
:106F180000031A6019684FF0200089B201F0CEFD15
:106F28004FF01C004FF0020101F0C8FD41F254136C
:106F3800C2F200034FF002021A7076E241F27913AE
:106F4800C2F200031B78002B40D041F27913C2F241
:106F580000034FF000021A7040F29C23C2F20003B3
:106F68009B68012B10D013B1022B26D119E044F2F3
:106F7800B420C0F6010041F25C11C2F200014FF0EA
:106F8800130206F0ADFD18E044F2CC20C0F6010073
:106F980041F25C11C2F200014FF0130206F0A0FDAD
:106FA8000BE044F2E420C0F6010041F25C11C2F2A9
:106FB80000014FF0130206F093FD4FF0200001F09E
:106FC80099FD41F25813C2F20003186040F263437E
:106FD800C2F20003197840F2B413C2F20003187821
:106FE80040F26043C2F200031A7800EA01031A4231
:106FF80020D041F62823C2F20003DB694FF4167251
:1070080002FB03F241F25813C2F200031A60196836
:107018004FF0200089B201F051FD40F28C13C2F20A
:1070280000034FF000021A7040F2CE23C2F20003B0
:107038001A70FAE141F25813C2F200031B68002BE0
:1070480040D041F25814C2F20004236803F1FF3320
:10705800236021684FF0200089B201F02FFD2068DD
:1070680048F2B515C1F64E35A5FB0030B04F4FF0CC
:10707800020600964FEA901039464FF00002134678
:1070880006F0DCFD2368A5FB03124FEA92124FF4C9
:10709800167101FB123241F29413C2F200031A6016
:1070A8001A684CF6CD43CCF6CC43A3FB02130096EA
:1070B8004FEAD30007F103014FF00002134606F030
:1070C800BDFDB2E141F27C13C2F200034FF00002B1
:1070D8001A6041F27913C2F200034FF001021A70EC
:1070E80041F25413C2F200034FF003021A709CE1FC
:1070F80041F27913C2F200031B78BBB141F2791354
:10710800C2F200034FF000021A7040F69903C2F26F
:1071180000034FF00101197041F27C13C2F2000321
:107128001A6041F25813C2F200031A6041F27C134C
:10713800C2F200031A6802F101021A601B680A2BE6
:1071480021D941F27C13C2F200034FF000021A6009
:1071580040F69903C2F200031B786BB140F699031D
:10716800C2F200031A7041F25813C2F200031A68FF
:1071780002F101021A6006E040F69903C2F2000328
:107188004FF001021A7041F25813C2F200031B6853
:10719800032B40F24A8140F2CE23C2F200034FF0A3
:1071A80001021A7041F27C13C2F200034FF0000290
:1071B8001A6041F25413C2F200034FF004021A702D
:1071C80033E141F27C13C2F200031A6802F10102B2
:1071D8001A601B680A2B40F2288141F27913C2F227
:1071E80000034FF001021A7040F28C13C2F2000340
:1071F8001A7041F25413C2F200034FF005011970DE
:107208004FF01C0001F05AFC0FE141F27913C2F271
:1072180000031B78002B4ED041F27913C2F2000311
:107228004FF000021A7040F29C23C2F200039B68E0
:10723800012B10D013B1022B26D119E044F2FC2007
:10724800C0F6010041F25C11C2F200014FF01302D6
:1072580006F046FC18E044F21430C0F6010041F292
:107268005C11C2F200014FF0130206F039FC0BE08A
:1072780044F22C30C0F6010041F25C11C2F2000168
:107288004FF0130206F02CFC40F2CE23C2F20003AA
:107298004FF001021A7041F27C13C2F200034FF062
:1072A80000021A604FF0200001F024FC41F258134C
:1072B800C2F20003186041F27C13C2F200031A689C
:1072C80002F101021A601B680A2B81BF40F28C137D
:1072D800C2F2000301221A7040F26343C2F20003B3
:1072E800197840F2B413C2F20003187840F26043F0
:1072F800C2F200031A7800EA01031A421AD040F2D7
:107308008C13C2F200034FF000021A7040F2CE2331
:10731800C2F200031A7041F25413C2F200034FF094
:10732800010119704FF01C0001F0C8FB7DE000BF9F
:107338006B11002041F25814C2F20004236803F1D3
:107348000103236021684FF0200089B201F0B6FBE9
:10735800226841F62823C2F200031B6A4FF4167113
:1073680001FB03F3934219D240F2CE23C2F2000389
:107378004FF000041C7041F25413C2F200031C7059
:107388004FF01C00214601F099FB009401944FF046
:107398001B0021462246234602F00EFA41F25814F9
:1073A800C2F20004206848F2B515C1F64E35A5FBB7
:1073B80000201F4F4FF0020600964FEA9010394602
:1073C8004FF00002134606F039FC2368A5FB0315AD
:1073D8004FEA95154FF4167202FB153541F29413D6
:1073E800C2F200031D601A684CF6CD43CCF6CC43BC
:1073F800A3FB021300964FEAD30007F103014FF0F5
:107408000002134606F01AFC0FE040F28C13C2F299
:1074180000034FF00001197041F25413C2F2000347
:1074280019704FF01C0001F049FB03B0F0BD00BF1C
:107438006B11002010B540F2CE23C2F200031B7876
:10744800002B42D040F29213C2F200031A8802F1D4
:10745800010292B21A801B889BB23B2B35D94FF0A0
:10746800540001F047FB40F29214C2F2000420805D
:10747800238803F101039BB2238021884FF0540035
:1074880089B201F01BFB23889BB2B3F5167F15D395
:107498004FF054004FF0000101F010FB4FF058007E
:1074A80001F028FB2080228802F1010292B222809A
:1074B80021884FF0580089B201F000FB40F2921386
:1074C800C2F200034FF000021A8041F29B13C2F28D
:1074D80000031A7802F10102D2B21A7040F6C4030E
:1074E800C2F200031B7863B341F29D13C2F200039A
:1074F8001A7802F10102D2B21A701A7841F62823DA
:10750800C2F200039B699A4240D3DBB241F29D125A
:10751800C2F20002137040F29C23C2F200035B69BE
:107528003BB140F2C523C2F200034FF001021A70CA
:107538002CE040F2C523C2F200034FF000021A709B
:1075480024E041F29D13C2F200031B784BB141F2D3
:107558009D13C2F200031A7802F1FF32D2B21A70F8
:1075680014E040F29C23C2F200035B693BB140F295
:10757800C523C2F200034FF000021A7006E040F281
:10758800C523C2F200034FF001021A7040F2E13342
:10759800C2F200031B7863B341F29C13C2F20003EA
:1075A8001A7802F10102D2B21A701A7841F6282329
:1075B800C2F200039B699A4240D3DBB241F29C12AB
:1075C800C2F20002137040F29C23C2F200035B690E
:1075D8003BB140F26343C2F200034FF001021A705C
:1075E8002CE040F26343C2F200034FF000021A702D
:1075F80024E041F29C13C2F200031B784BB141F224
:107608009C13C2F200031A7802F1FF32D2B21A7048
:1076180014E040F29C23C2F200035B693BB140F2E4
:107628006343C2F200034FF000021A7006E040F212
:107638006343C2F200034FF001021A7040F2BD2307
:10764800C2F200031B7863B341F29E13C2F2000337
:107658001A7802F10102D2B21A701A7841F6282378
:10766800C2F200039B699A4240D3DBB241F29E12F8
:10767800C2F20002137040F29C23C2F200035B695D
:107688003BB140F2B413C2F200034FF001021A708A
:107698002CE040F2B413C2F200034FF000021A705B
:1076A80024E041F29E13C2F200031B784BB141F271
:1076B8009E13C2F200031A7802F1FF32D2B21A7096
:1076C80014E040F29C23C2F200035B693BB140F234
:1076D800B413C2F200034FF000021A7006E040F241
:1076E800B413C2F200034FF001021A7040F66A03A5
:1076F800C2F200031B7863B341F29F13C2F2000386
:107708001A7802F10102D2B21A701A7841F62823C7
:10771800C2F200039B699A4240D3DBB241F29F1246
:10772800C2F20002137040F29C23C2F200035B69AC
:107738003BB140F26043C2F200034FF001021A70FD
:107748002CE040F26043C2F200034FF000021A70CE
:1077580024E041F29F13C2F200031B784BB141F2BF
:107768009F13C2F200031A7802F1FF32D2B21A70E4
:1077780014E040F29C23C2F200035B693BB140F283
:107788006043C2F200034FF000021A7006E040F2B4
:107798006043C2F200034FF001021A7041F2A013D5
:1077A800C2F200031B78B3B940F29613C2F2000389
:1077B8001B7883B140F29613C2F200034FF0000227
:1077C8001A7002F013FE30B140F29713C2F20003B0
:1077D8004FF001021A7040F29713C2F200031B78AF
:1077E800012B06D013B1022B27D10CE002F0CEF802
:1077F80010BD02F007FE40F29713C2F200034FF0EB
:1078080002021A7010BD4FF46840C0F6030007F07A
:1078180067FC4FF024004FF0000101F04FF94FF0E2
:1078280028004FF0000101F049F940F29713C2F225
:1078380000034FF000021A7010BD40F29713C2F215
:1078480000034FF000021A7010BD00BF80B489B069
:1078580000AF786039604FF00003FB614FF0000320
:107868003B614FF00003BB614FF00003FB604FF03A
:1078780000037B614FF00003BB603B68DB7803F0DB
:107888000F03FB613B68DB7803F01003002B05D086
:107898003B689B78FA6942EA0303FB613B681B88F3
:1078A80003F0FF03002B51D07B681B687B614FF00E
:1078B8000003BB6144E0BB694FF0010202FA03F325
:1078C800FB603B681B881A46FB6802EA03033B61BE
:1078D8003A69FB689A422FD1BB694FEA8303FB6080
:1078E800FB684FF00F0202FA03F3BB60BB686FEA54
:1078F80003037A6902EA03037B61FB68FA6902FA07
:1079080003F37A6942EA03037B613B68DB78282B3F
:1079180007D1BB694FF0010202FA03F27B685A6192
:107928000AE03B68DB78482B06D1BB694FF00102BF
:1079380002FA03F27B681A61BB6903F10103BB61B8
:10794800BB69072BB7D97B687A691A603B681B88C3
:10795800FF2B56D97B685B687B614FF00003BB61E6
:1079680049E0BB6903F108034FF0010202FA03F38F
:10797800FB603B681B881A46FB6802EA03033B610D
:107988003A69FB689A4232D1BB694FEA8303FB60CC
:10799800FB684FF00F0202FA03F3BB60BB686FEAA3
:1079A80003037A6902EA03037B61FB68FA6902FA56
:1079B80003F37A6942EA03037B613B68DB78282B8F
:1079C80008D1BB6903F108034FF0010202FA03F280
:1079D8007B685A613B68DB78482B08D1BB6903F1A7
:1079E80008034FF0010202FA03F27B681A61BB69CF
:1079F80003F10103BB61BB69072BB2D97B687A69C4
:107A08005A6007F12407BD4680BC704780B483B034
:107A180000AF78607B684FF6FF721A807B684FF082
:107A280002029A707B684FF00402DA7007F10C07C3
:107A3800BD4680BC704700BF80B485B000AF786099
:107A48000B467B804FF00003FB737B689B681A46EC
:107A58007B8802EA0303002B03D04FF00103FB737A
:107A680002E04FF00003FB73FB7B184607F1140795
:107A7800BD4680BC704700BF80B483B000AF78605B
:107A88007B689B689BB2184607F10C07BD4680BC13
:107A9800704700BF80B483B000AF78600B467B802E
:107AA8007A887B681A6107F10C07BD4680BC70476D
:107AB80080B483B000AF78600B467B807A887B689F
:107AC8005A6107F10C07BD4680BC704780B487B087
:107AD80000AF78600B46FB704FF000033B614FF03E
:107AE8000003FB604FF000037B614FF00003BB60B5
:107AF8007B68002B06DA4FF00003C4F20103DB6950
:107B08007B6105E04FF00003C4F201035B687B6111
:107B18007B6803F470234FEA1343BB607B684FEA2A
:107B280003434FEA13433B617B6803F44013B3F507
:107B3800401F10D17B6923F070637B614FF0000315
:107B4800C4F201034FF00002C4F20102526822F0AD
:107B580070625A6028E07B6803F48013002B11D010
:107B6800BB684FF0030202FA03F3FB60FB686FEA9D
:107B780003037A6902EA03037B617B6943F070635C
:107B88007B6111E07B684FEA53534FEA03133A696C
:107B980002FA03F36FEA03037A6902EA03037B61DB
:107BA8007B6943F070637B61FB78002B0BD07B68AB
:107BB8004FEA53534FEA03133A6902FA03F37A6917
:107BC80042EA03037B617B68002B06DA4FF000036F
:107BD800C4F201037A69DA6105E04FF00003C4F2E8
:107BE80001037A695A6007F11C07BD4680BC7047DB
:107BF80080B483B000AF78607B68042B0CD14EF260
:107C08001003CEF200034EF21002CEF20002126808
:107C180042F004021A600BE04EF21003CEF20003A9
:107C28004EF21002CEF20002126822F004021A602C
:107C380007F10C07BD4680BC704700BF80B483B015
:107C480000AF78604EF21003CEF200037A685A60F3
:107C580007F10C07BD4680BC704700BF80B483B0F5
:107C680000AF78607B68012B0CD14EF21003CEF286
:107C780000034EF21002CEF20002126842F0010236
:107C88001A6017E07B6813F1020F0CD14EF2100353
:107C9800CEF200034EF21002CEF20002126822F079
:107CA80001021A6006E04EF21003CEF200034FF014
:107CB80000029A6007F10C07BD4680BC704700BF00
:107CC80080B483B000AF0346FB71FB79002B0CD066
:107CD8004EF21003CEF200034EF21002CEF2000272
:107CE800126842F002021A600BE04EF21003CEF264
:107CF80000034EF21002CEF20002126822F00202D5
:107D08001A6007F10C07BD4680BC704780B58CB07F
:107D180000AF786039604FF00003FB624FF000035A
:107D2800BB624FF000037B624FF000033B624FF0F1
:107D38000003FB617B68FB617B681B8A9BB2FB626B
:107D4800FA6A4CF6FF7302EA0303FB623B68DB88BE
:107D5800FA6A42EA0303FB62FB6A9AB27B681A82F8
:107D68007B689B899BB2FB62FA6A4EF6F31302EAC0
:107D78000303FB623B689A883B681B8942EA03035A
:107D88009AB23B685B8942EA03039BB2FA6A42EA09
:107D98000303FB62FB6A9AB27B689A817B689B8AC1
:107DA8009BB2FB62FA6A4FF6FF4302EA0303FB62E7
:107DB8003B689B89FA6A42EA0303FB62FB6A9AB250
:107DC8007B689A8207F10803184600F043FBFA69BA
:107DD8004FF46053C4F201039A4202D17B69BB623B
:107DE80001E03B69BB627B689B899BB29BB21BB27B
:107DF800002B0FDABA6A13464FEA83039B184FEA3F
:107E080083029A183B681B684FEA4303B2FBF3F3FB
:107E18007B620EE0BA6A13464FEA83039B184FEA67
:107E280083029A183B681B684FEA8303B2FBF3F39B
:107E38007B627A6A48F21F53C5F2EB13A3FB021365
:107E48004FEA53134FEA0313FB62FB6A4FEA13131B
:107E58004FF0640202FB03F37A6AD31A3B627B6831
:107E68009B899BB29BB21BB2002B13DA3B6A4FEA89
:107E7800C30303F1320248F21F53C5F2EB13A3FB0D
:107E880002134FEA531303F00703FA6A42EA0303A3
:107E9800FB6212E03B6A4FEA031303F1320248F235
:107EA8001F53C5F2EB13A3FB02134FEA531303F05E
:107EB8000F03FA6A42EA0303FB62FB6A9AB27B6821
:107EC8001A8107F13007BD4680BD00BF80B485B078
:107ED80000AF786039604FF00003FB607B681B8A55
:107EE8009BB2FB60FA684FF2FF0302EA0303FB60F0
:107EF8003B681A883B685B8842EA03039AB23B688E
:107F08009B8842EA03039AB23B68DB8842EA030390
:107F18009BB2FA6842EA0303FB60FB689AB27B688B
:107F28001A8207F11407BD4680BC704780B483B03D
:107F380000AF78600B46FB70FB78002B08D07B689D
:107F48009B899BB243F400539AB27B689A8107E0FD
:107F58007B689B899BB223F400539AB27B689A8111
:107F680007F10C07BD4680BC704700BF80B487B0DE
:107F780000AF78600B467B804FF00003FB604FF04A
:107F880000037B614FF00003BB604FF00003FB74FC
:107F98007B88DBB24FEA5313DBB2BB607B8803F00C
:107FA8001F037B617B694FF0010202FA03F37B61D7
:107FB800BB68012B07D17B689B899BB27A6902EA6F
:107FC80003037B6111E0BB68022B07D17B681B8A26
:107FD8009BB27A6902EA03037B6106E07B689B8AAD
:107FE8009BB27A6902EA03037B617B884FEA132319
:107FF8009BB2FB60FB684FF0010202FA03F3FB60DF
:108008007B681B889BB2FA6802EA0303FB607B6902
:10801800002B06D0FB68002B03D04FF00103FB7444
:1080280002E04FF00003FB74FB7C184607F11C07C5
:10803800BD4680BC704700BF80B485B000AF786093
:108048000B467B804FF00003FB814FF00003BB81A0
:108058007B884FEA1323FB81FB894FF0010202FA68
:1080680003F3BB81BB896FEA03039AB27B681A806A
:1080780007F11407BD4680BC704700BF80B400AF4D
:108088004FF48053C4F202034FF48052C4F2020248
:10809800126842F001021A604FF48052C4F20202E0
:1080A8004FF48053C4F202035B6819464FF0000393
:1080B800CFF6FF0301EA030353604FF48053C4F281
:1080C80002034FF48052C4F20202126822F0847252
:1080D80022F480321A604FF48053C4F202034FF442
:1080E8008052C4F20202126822F480221A604FF40D
:1080F8008053C4F202034FF48052C4F20202526861
:1081080022F4FE025A604FF48053C4F202034FF483
:108118001F029A60BD4680BC704700BF80B483B020
:1081280000AF78604FF48053C4F202034FF48052DA
:10813800C4F20202126822F480321A604FF48053AB
:10814800C4F202034FF48052C4F20202126822F40D
:1081580080221A607B68B3F5803F03D0B3F5802F87
:108168000DD019E04FF48053C4F202034FF480524B
:10817800C4F20202126842F480321A600CE04FF432
:108188008053C4F202034FF48052C4F20202126810
:1081980042F4A0221A6000BF07F10C07BD4680BC5C
:1081A800704700BF80B582B000AF4FF000033B605E
:1081B8004FF00003FB714FF00003BB714FF031002B
:1081C80000F0FAFA0346BB713B6803F101033B6018
:1081D8003B68B3F5A06F02D0BB79002BEED04FF00F
:1081E800310000F0E9FA0346002B03D04FF00103F9
:1081F800FB7102E04FF00003FB71FB79184607F1B1
:108208000807BD4680BD00BF80B485B000AF786068
:1082180039604FF00003FB604FF48053C4F202034F
:108228005B68FB60FB6823F47C13FB607A683B683F
:1082380042EA0303FA6842EA0303FB604FF48053FF
:10824800C4F20203FA685A6007F11407BD4680BCFD
:10825800704700BF80B483B000AF0346FB714FF096
:108268006003C4F24223FA791A6007F10C07BD468D
:1082780080BC704780B485B000AF78604FF00003D1
:10828800FB604FF48053C4F202035B68FB60FB6839
:1082980023F00303FB60FA687B6842EA0303FB6090
:1082A8004FF48053C4F20203FA685A6007F11407C6
:1082B800BD4680BC704700BF80B400AF4FF4805308
:1082C800C4F202035B68DBB203F00C03DBB21846AE
:1082D800BD4680BC704700BF80B485B000AF7860F1
:1082E8004FF00003FB604FF48053C4F202035B6855
:1082F800FB60FB6823F0F003FB60FA687B6842EAE6
:108308000303FB604FF48053C4F20203FA685A6017
:1083180007F11407BD4680BC704700BF80B485B024
:1083280000AF78604FF00003FB604FF48053C4F255
:1083380002035B68FB60FB6823F4E063FB60FA6898
:108348007B6842EA0303FB604FF48053C4F20203E4
:10835800FA685A6007F11407BD4680BC704700BF31
:1083680080B485B000AF78604FF00003FB604FF435
:108378008053C4F202035B68FB60FB6823F460531C
:10838800FB607B684FEAC303FA6842EA0303FB60B9
:108398004FF48053C4F20203FA685A6007F11407D5
:1083A800BD4680BC704700BF80B483B000AF0346B1
:1083B800FB714FF48153C4F202034FF000021A70AC
:1083C8004FF48153C4F202034FF000021A70FB7994
:1083D800012B02D0042B08D00FE04FF48153C4F2D4
:1083E80002034FF001021A7007E04FF48153C4F200
:1083F80002034FF005021A7000BF07F10C07BD46D3
:1084080080BC704780B483B000AF78604FF480536D
:10841800C4F202034FF48052C4F20202126A1146F7
:108428007A6841EA02021A6207F10C07BD4680BC6D
:10843800704700BF80B483B000AF0346FB7140F2C1
:108448003C43C4F24223FA791A6007F10C07BD468F
:1084580080BC704780B487B000AF78604FF00003ED
:108468007B614FF000033B614FF00003FB604FF06E
:108478000003BB604FF48053C4F202035B6803F04F
:108488000C037B617B69042B0AD0082B0FD0002BCF
:108498004DD17A684FF49053C0F27A0313604DE0DF
:1084A8007A684FF49053C0F27A03136046E04FF4B1
:1084B8008053C4F202035B6803F470133B614FF40A
:1084C8008053C4F202035B6803F48033FB603B69AA
:1084D8004FEA934303F102033B61FB68002B09D188
:1084E8003A694FF41063C0F23D0303FB02F27B6864
:1084F8001A6023E04FF48053C4F202035B6803F46C
:108508000033002B09D03A694FF41063C0F23D03E1
:1085180003FB02F27B681A6010E03A694FF490534B
:10852800C0F27A0303FB02F27B681A6006E07A68FD
:108538004FF49053C0F27A03136000BF4FF4805396
:10854800C4F202035B6803F0F0037B617B694FEAC6
:1085580013137B6140F27413C2F200037A699B180B
:108568001B78DBB2BB607B681A68BB6822FA03F22F
:108578007B685A604FF48053C4F202035B6803F4CB
:10858800E0637B617B694FEA13237B6140F27413DC
:10859800C2F200037A699B181B78DBB2BB607B6868
:1085A8005A68BB6822FA03F27B689A604FF48053DA
:1085B800C4F202035B6803F460537B617B694FEA92
:1085C800D3237B6140F27413C2F200037A699B18CB
:1085D8001B78DBB2BB607B685A68BB6822FA03F27F
:1085E8007B68DA604FF48053C4F202035B6803F4DB
:1085F80040437B617B694FEA93337B6140F284138C
:10860800C2F200037A699B181B78DBB2BB607B68F7
:10861800DA68BB68B2FBF3F27B681A6107F11C07E2
:10862800BD4680BC704700BF80B483B000AF78609F
:108638000B46FB70FB78002B0ED04FF48053C4F22E
:1086480002034FF48052C4F20202526911467A685A
:1086580041EA02025A610FE04FF48053C4F2020368
:108668004FF48052C4F20202526911467A686FEAE6
:10867800020201EA02025A6107F10C07BD4680BCFA
:10868800704700BF80B483B000AF78600B46FB70C2
:10869800FB78002B0ED04FF48053C4F202034FF442
:1086A8008052C4F20202926911467A6841EA0202D3
:1086B8009A610FE04FF48053C4F202034FF48052E2
:1086C800C4F20202926911467A686FEA020201EA6C
:1086D80002029A6107F10C07BD4680BC704700BFD3
:1086E80080B483B000AF78600B46FB70FB78002B3A
:1086F8000ED04FF48053C4F202034FF48052C4F2F8
:108708000202D26911467A6841EA0202DA610FE090
:108718004FF48053C4F202034FF48052C4F20202B1
:10872800D26911467A686FEA020201EA0202DA6146
:1087380007F10C07BD4680BC704700BF80B483B00A
:1087480000AF78600B46FB70FB78002B0ED04FF41F
:108758008053C4F202034FF48052C4F20202D2687A
:1087680011467A6841EA0202DA600FE04FF480535A
:10877800C4F202034FF48052C4F20202D2681146D6
:108788007A686FEA020201EA0202DA6007F10C076E
:10879800BD4680BC704700BF80B483B000AF0346BD
:1087A800FB714FF48863C4F24223FA791A6007F127
:1087B8000C07BD4680BC704780B487B000AF034645
:1087C800FB714FF00003FB604FF000037B614FF03B
:1087D8000003FB74FB794FEA5313DBB2FB60FB68C1
:1087E800012B06D14FF48053C4F202031B687B614E
:1087F8000FE0FB68022B06D14FF48053C4F202034A
:108808001B6A7B6105E04FF48053C4F202035B6A84
:108818007B61FB7903F01F03FB60FB687A6922FA2E
:1088280003F303F00103DBB2002B03D04FF0010385
:10883800FB7402E04FF00003FB74FB7C184607F161
:108848001C07BD4680BC704780B483B000AF0246A9
:108858000B46FA807B717B79002B0FD04FF42053A5
:10886800C4F200034FF42052C4F20002128891B2FD
:10887800FA8841EA020292B21A8011E04FF42053BA
:10888800C4F200034FF42052C4F20002128891B2DD
:10889800FA886FEA020292B201EA020292B21A80E0
:1088A80007F10C07BD4680BC704700BF80B400AF1D
:1088B8004FF42053C4F200034FF42052C4F20002D4
:1088C800928892B242F0100292B29A80BD4680BC61
:1088D800704700BF80B400AF4FF42053C4F20003C8
:1088E8004FF42052C4F20002928892B222F0100291
:1088F80092B29A80BD4680BC704700BF80B483B0F6
:1089080000AF4FF00003FB804FF42053C4F2000384
:108918009B8BFB804FF42053C4F200031B8B9BB24C
:108928004FEA0342FB8842EA0303184607F10C07A3
:10893800BD4680BC704700BF80B582B000AF78608C
:10894800FFF7B4FF4FF42053C4F200037A684FEAEC
:10895800124292B21A834FF42053C4F200037A6889
:1089680092B29A83FFF7B6FF07F10807BD4680BDAC
:1089780080B582B000AF7860FFF798FF4FF42053BE
:10898800C4F200037A6802F470224FEA124292B2EB
:108998001A814FF42053C4F200037A6892B29A8184
:1089A800FFF798FF07F10807BD4680BD80B400AF08
:1089B80000BF4FF42053C4F200039B889BB203F01E
:1089C8002003002BF5D0BD4680BC704780B400AFB3
:1089D8004FF42053C4F200034FF42052C4F20002B3
:1089E800928892B222F0080292B29A8000BF4FF4A5
:1089F8002053C4F200039B889BB203F00803002BAA
:108A0800F5D0BD4680BC704780B485B000AF034642
:108A1800FB804FF00003FB734FF42053C4F20003B4
:108A28009B889BB2DAB2FB88DBB202EA0303FB73D2
:108A38004FF42053C4F200031B889AB2FB8802EA61
:108A480003039BB2002B06D0FB7B002B03D04FF017
:108A58000103FB7302E04FF00003FB73FB7B184636
:108A680007F11407BD4680BC704700BF80B483B0CF
:108A780000AF0346FB804FF42053C4F200034FF4C9
:108A88002052C4F20002928891B2FA886FEA020278
:108A980092B201EA020292B29A8007F10C07BD462F
:108AA80080BC704780B500AF4FF00100FFF774FE3F
:108AB8004FF00000FFF770FE80BD00BF80B485B0A6
:108AC80000AF02460B46FA80BB804FF00003FB6004
:108AD8004FF4D843C4F20003FB60FA88FB68D3184C
:108AE800FB60FB68BA881A6007F11407BD4680BCB2
:108AF800704700BF80B485B000AF0346FB804FF0DD
:108B08000003FB604FF4D843C4F20003FB60FA880B
:108B1800FB68D318FB60FB681B889BB2184607F1FB
:108B28001407BD4680BC704780B483B000AF78603E
:108B38004FF46D43CEF200037A6842F0BE6242F40D
:108B48002022DA6007F10C07BD4680BC704700BFE1
:108B580080B487B000AF78604FF000037B614FF0BE
:108B680000033B614FF00F03FB607B68DB78002B51
:108B780049D04FF46D43CEF20003DB686FEA03037C
:108B880003F4E0634FEA13237B617B69C3F10403B9
:108B98003B617B69FA6822FA03F3FB607B685B78C8
:108BA8001A463B6902FA03F37B617B689B781A4695
:108BB800FB6802EA03037A6942EA03037B617B6983
:108BC8004FEA03137B614FF46143CEF200037A68E6
:108BD800127811467A69D2B25B1883F800234FF4F1
:108BE8006143CEF200037A6812784FEA5212D2B289
:108BF8007968097801F01F014FF0010000FA01F1CE
:108C080043F8221014E04FF46143CEF200037A686F
:108C180012784FEA5212D2B27968097801F01F012E
:108C28004FF0010000FA01F102F1200243F822108E
:108C380007F11C07BD4680BC704700BF80B483B0F5
:108C480000AF786039604FF46D43CEF200033A68A4
:108C580022F0604222F07F0279680A439A6007F1A5
:108C68000C07BD4680BC704780B483B000AF034694
:108C7800FB714FF02003C4F20E23FA791A6007F152
:108C88000C07BD4680BC704780B483B000AF034674
:108C9800FB714FF01003C4F20E23FA791A6007F142
:108CA8000C07BD4680BC704780B485B000AF7860C3
:108CB80039604FF00003FB817B681B88FB81FB89CF
:108CC80003F44153FB813B681A883B685B8842EA9E
:108CD80003039AB23B689B8842EA03039AB23B6853
:108CE800DB8842EA03039AB23B681B8942EA030322
:108CF8009AB23B685B8942EA03039AB23B689B8954
:108D080042EA03039AB23B68DB8942EA03039AB258
:108D1800FB8942EA0303FB817B68FA891A807B6836
:108D28009B8B9BB223F400639AB27B689A833B685F
:108D38001A8A7B681A8207F11407BD4680BC7047FF
:108D480080B483B000AF78600B46FB70FB78002BD3
:108D580008D07B681B889BB243F040039AB27B68BB
:108D68001A8007E07B681B889BB223F040039AB205
:108D78007B681A8007F10C07BD4680BC704700BFAE
:108D880080B483B000AF786013460A467A807B705F
:108D98007B78002B09D07B689B889AB27B8842EA53
:108DA80003039AB27B689A800BE07B689B889AB22F
:108DB8007B886FEA03039BB202EA03039AB27B68DB
:108DC8009A8007F10C07BD4680BC704780B483B019
:108DD80000AF78600B467B807B687A889A8107F1C0
:108DE8000C07BD4680BC704780B483B000AF786084
:108DF8000B46FB70FB78002B08D07B689B889BB2E6
:108E080043F004039AB27B689A8007E07B689B88EA
:108E18009BB223F004039AB27B689A8007F10C078F
:108E2800BD4680BC704700BF80B483B000AF786097
:108E38004FF48063C4F201037A685A6107F10C07A2
:108E4800BD4680BC704700BF80B483B000AF786077
:108E58007B681B681A464FF6FE7302EA03037A68BA
:108E680013607B684FF000021A607B684FF00002C5
:108E78005A607B684FF000029A607B684FF00002EE
:108E8800DA607A684FF00803C4F202039A420CD100
:108E98004FF00003C4F202034FF00002C4F20202D2
:108EA800526842F00F025A60DAE07A684FF01C0309
:108EB800C4F202039A420CD14FF00003C4F2020339
:108EC8004FF00002C4F20202526842F0F0025A6007
:108ED800C6E07A684FF03003C4F202039A420CD11C
:108EE8004FF00003C4F202034FF00002C4F2020282
:108EF800526842F470625A60B2E07A684FF04403F4
:108F0800C4F202039A420CD14FF00003C4F20203E8
:108F18004FF00002C4F20202526842F470425A60F2
:108F28009EE07A684FF05803C4F202039A420CD1CB
:108F38004FF00003C4F202034FF00002C4F2020231
:108F4800526842F470225A608AE07A684FF06C03E3
:108F5800C4F202039A420CD14FF00003C4F2020398
:108F68004FF00002C4F20202526842F470025A60E2
:108F780076E07A684FF08003C4F202039A420CD17B
:108F88004FF00003C4F202034FF00002C4F20202E1
:108F9800526842F070625A6062E07A684FF4816306
:108FA800C4F202039A420CD14FF48063C4F2020364
:108FB8004FF48062C4F20202526842F00F025A6013
:108FC8004EE07A6840F21C43C4F202039A420CD184
:108FD8004FF48063C4F202034FF48062C4F20202C9
:108FE800526842F0F0025A603AE07A684FF48663B9
:108FF800C4F202039A420CD14FF48063C4F2020314
:109008004FF48062C4F20202526842F470625A60FD
:1090180026E07A6840F24443C4F202039A420CD133
:109028004FF48063C4F202034FF48062C4F2020278
:10903800526842F470425A6012E07A684FF48B63C7
:10904800C4F202039A420BD14FF48063C4F20203C4
:109058004FF48062C4F20202526842F470225A60ED
:1090680007F10C07BD4680BC704700BF80B485B0CF
:1090780000AF786039604FF00003FB607B681B68C5
:10908800FB60FB6823F4FE4323F0F003FB603B68BE
:109098009A683B681B6A1A433B681B691A433B681A
:1090A8005B691A433B689B691A433B68DB691A434F
:1090B8003B685B6A1A433B689B6A42EA0303FA68A7
:1090C80042EA0303FB607B68FA681A603B68DA6867
:1090D8007B685A603B681A687B689A603B685A6884
:1090E8007B68DA6007F11407BD4680BC704700BF93
:1090F80080B483B000AF78600B46FB70FB78002B20
:1091080006D07B681B6843F001027B681A6008E0A0
:109118007B681B681A464FF6FE7302EA03037A68F7
:10912800136007F10C07BD4680BC704780B485B05A
:1091380000AF78604FF00003FB734FF00003BB6093
:109148007B6803F08053002B06D04FF48063C4F291
:1091580002031B68BB6005E04FF00003C4F2020382
:109168001B68BB60BA687B6802EA0303002B03D064
:109178004FF00103FB7302E04FF00003FB73FB7B2E
:10918800184607F11407BD4680BC704780B483B009
:1091980000AF78607B6803F08053002B06D04FF453
:1091A8008063C4F202037A685A6005E04FF0000356
:1091B800C4F202037A685A6007F10C07BD4680BC06
:1091C800704700BF204A038890429BB20ED01F4AC6
:1091D80090420BD0B0F1804F08D01D4A904205D084
:1091E8001C4A904202D01C4A904206D14FF68F7218
:1091F80003EA02024B8842EA0303184A904209D064
:10920800174A904206D04FF6FF4203EA0202CB8883
:1092180042EA030303808B8883850B8803850A4B06
:1092280098420BD0094B984208D00E4B984205D073
:109238000D4B984202D00D4B984201D10B7A038610
:1092480001238382704700BF002C01400034014095
:109258000004004000080040000C004000100040DE
:109268000014004000400140004401400048014013
:109278004FF0FF33838000230380C3804380037251
:1092880070470023038043808380C3800381438128
:109298008381C381704721B103889BB243F00103E6
:1092A80004E0038823F001031B041B0C03807047B0
:1092B8001AB183899BB2194303E083899BB223EADD
:1092C800010181817047C94389B20182704700005A
:1092D80080B582B000AF78607A684FF41053C4F25A
:1092E80001039A420CD14FF400704FF00101FFF7CF
:1092F80025FA4FF400704FF00001FFF71FFA26E03F
:109308007A684FF42053C4F201039A420CD14FF407
:1093180080604FF00101FFF711FA4FF480604FF0C1
:109328000001FFF70BFA12E07A684FF47053C4F2A9
:1093380001039A420BD14FF400404FF00101FFF7AF
:10934800FDF94FF400404FF00001FFF7F7F907F17E
:109358000807BD4680BD00BF80B485B000AF786007
:1093680039604FF00003FB604FF00003FB727B682D
:109378005B68FB60FB6823F4702323F48073FB6055
:109388003B681A683B681B794FEA032342EA0303E8
:10939800FA6842EA0303FB607B68FA685A607B68F4
:1093A8009B68FB60FA684FF2FD73CFF6F17302EA2F
:1093B8000303FB603B68DA683B689B681A433B68B9
:1093C8005B794FEA430342EA0303FA6842EA03037C
:1093D800FB607B68FA689A607B68DB6AFB60FB6805
:1093E80023F47003FB603B681B7C03F1FF33DAB2A4
:1093F800FB7A42EA0303FB72FB7A4FEA0353FA68EB
:1094080042EA0303FB607B68FA68DA6207F1140733
:10941800BD4680BC704700BF80B483B000AF7860A1
:109428000B46FB70FB78002B06D07B689B6843F0EB
:1094380001027B689A6005E07B689B6823F0010263
:109448007B689A6007F10C07BD4680BC704700BF77
:1094580080B483B000AF78607B689B6843F00802F3
:109468007B689A6007F10C07BD4680BC704700BF57
:1094780080B485B000AF78604FF00003FB737B6861
:109488009B6803F00803002B03D04FF00103FB7324
:1094980002E04FF00003FB73FB7B184607F114074B
:1094A800BD4680BC704700BF80B483B000AF786011
:1094B8007B689B6843F004027B689A6007F10C079D
:1094C800BD4680BC704700BF80B485B000AF7860EF
:1094D8004FF00003FB737B689B6803F00403002BC9
:1094E80003D04FF00103FB7302E04FF00003FB735E
:1094F800FB7B184607F11407BD4680BC704700BFC8
:1095080080B483B000AF78600B46FB70FB78002B0B
:1095180006D07B689B6843F4A0027B689A6005E0EC
:109528007B689B6823F4A0027B689A6007F10C07AC
:10953800BD4680BC704700BF80B485B000AF78607E
:10954800F970BA707B704FF00003FB604FF00003B6
:10955800BB60FB78092B29D97B68DB68FB60FA784C
:1095680013464FEA43039B18A3F11E034FF007026B
:1095780002FA03F3BB60BB686FEA0303FA6802EA06
:109588000303FB607978FA7813464FEA43039B1884
:10959800A3F11E0301FA03F3BB60FA68BB6842EA51
:1095A8000303FB607B68FA68DA6024E07B681B6968
:1095B800FB60FA7813464FEA43039B184FF0070203
:1095C80002FA03F3BB60BB686FEA0303FA6802EAB6
:1095D8000303FB607978FA7813464FEA43039B1834
:1095E80001FA03F3BB60FA68BB6842EA0303FB6055
:1095F8007B68FA681A61BB78062B29D87B685B6B95
:10960800FB60BB7803F1FF3213464FEA83039B18D4
:109618004FF01F0202FA03F3BB60BB686FEA030353
:10962800FA6802EA0303FB60F978BB7803F1FF32BA
:1096380013464FEA83039B1801FA03F3BB60FA68E9
:10964800BB6842EA0303FB607B68FA685A6355E02B
:10965800BB780C2B29D87B681B6BFB60BA78134648
:109668004FEA83039B18A3F123034FF01F0202FA6A
:1096780003F3BB60BB686FEA0303FA6802EA0303FB
:10968800FB60F978BA7813464FEA83039B18A3F175
:10969800230301FA03F3BB60FA68BB6842EA0303D9
:1096A800FB607B68FA681A6328E07B68DB6AFB600A
:1096B800BA7813464FEA83039B18A3F141034FF08E
:1096C8001F0202FA03F3BB60BB686FEA0303FA6880
:1096D80002EA0303FB60F978BA7813464FEA83037A
:1096E8009B18A3F1410301FA03F3BB60FA68BB6856
:1096F80042EA0303FB607B68FA68DA6207F1140741
:10970800BD4680BC704700BF80B483B000AF7860AE
:109718007B68DB6C9BB2184607F10C07BD4680BC22
:10972800704700BF80B483B000AF0346FB71FB797C
:10973800002B0CD04FF41053C4F201034FF4105215
:10974800C4F20102926842F400029A600BE04FF4FE
:109758001053C4F201034FF41052C4F2010292688C
:1097680022F400029A6007F10C07BD4680BC7047DE
:1097780010B40B46E1B1016889B24FF6FF7291420D
:109788001CBF00224FF6FF740AD105E050F80C1FE9
:1097980089B2A14204D101E04FF00002104609E06D
:1097A80002F10102D2B29342F0D84FF6FF7001E005
:1097B8004FF6FF7010BC70472DE9F0019DF814803A
:1097C8009DF818C04FF00004254641F2A017C2F2D8
:1097D80000073E5DDEB905EB45054FEA4505EDB2EC
:1097E80005F1010641F2A014C2F20004A15505F1E9
:1097F8000201625405F10302A35405F1040304F8BD
:10980800038005F1050304F803C0605506E005F17F
:109818000105EDB204F10604142DDAD1BDE8F0011A
:10982800704700BF4FF0000341F2A012C2F20002DD
:109838001946D15403F10103782BFAD1704700BFC0
:1098480010B584B004464FF46840C0F603004FF0EA
:109858003201FFF78DFFC1B2FF2900F0838046F681
:10986800B043C4F200031B888DF8003046F6B443B9
:10987800C4F200031B888DF8013046F6B843C4F2E1
:1098880000031B888DF8023041F60733C2F200034B
:109898001B788DF8033041F61733C2F200031B78AA
:1098A8008DF8043041F61533C2F200031B788DF8A9
:1098B800053041F2A013C2F200031B5DDAB28DF845
:1098C8000630192A23D140F21043C2F200031B7854
:1098D8008DF8073040F2CB23C2F200031B788DF8D5
:1098E800083040F2F823C2F200031B788DF80930E3
:1098F80040F2E813C2F200031B788DF80A3040F2F8
:109908001443C2F200031B788DF80B301CE004F1FD
:10991800010241F2A013C2F200039A5C8DF80720FD
:1099280004F102029A5C8DF8082004F103029A5CA3
:109938008DF8092004F104029A5C8DF80A2004F1DC
:1099480005041B5D8DF80B3001EB41014FF46840B5
:10995800C0F603004FEA81016A464FF0060305F09E
:10996800E9FB10E04FF000004FF0010144F24432EF
:10997800C0F60102034605F0ADFF4FF4FA604FF060
:109988000101FBF773F804B010BD00BF10B54FF02C
:1099980000031C4641F2A011C2F20001CA5C7AB170
:1099A80004EB44044FEA4404E4B22046FFF748FFBE
:1099B80041F2A013C2F200034FF000021A5510BD85
:1099C80004F10104E4B203F10603142CE6D110BD3E
:1099D800F0B583B005460668374640F29C23C2F2CC
:1099E80000039B68012B0FD013B1022B23D117E082
:1099F8004FF000004FF00C0144F25C32C0F6010257
:109A0800034605F067FF16E04FF000004FF00C0129
:109A180044F27432C0F60102034605F05BFF0AE027
:109A28004FF000004FF00C0144F28C32C0F60102F6
:109A3800034605F04FFF4FF000004FF0160144F2C7
:109A4800A032C0F60102034605F044FF4FF00104BE
:109A580000944FF000004FF01601FAB24FF00203E5
:109A680005F0AAFF00944FF012004FF01601C6F35C
:109A780007224FF0020305F09FFF05F10207D5F812
:109A8800025000944FF024004FF01601EAB24FF054
:109A9800020305F091FF00944FF04E004FF01601BD
:109AA800C5F307224FF0020305F086FF07F102060F
:109AB800D7F8025000944FF060004FF01601EAB258
:109AC8004FF0020305F078FF00944FF072004FF05A
:109AD8001601C5F307224FF0020305F06DFF06F1EA
:109AE8000204D6F80250EBB203F1FF331A2B00F24E
:109AF8007883DFE813F01B0076037603760376039A
:109B0800760376036200250176037603D400760394
:109B180076037603760376037603760376034701A6
:109B28009D027603B902D2022B02B90140F29C23AE
:109B3800C2F200039B68012B0FD013B1022B23D173
:109B480017E04FF000004FF0280144F2B832C0F699
:109B58000102034605F0BEFE16E04FF000004FF08C
:109B6800280144F2CC32C0F60102034605F0B2FEE9
:109B78000AE04FF000004FF0280144F2E032C0F64E
:109B88000102034605F0A6FE4FF000004FF0320137
:109B980044F2F432C0F60102034605F09BFE4FF092
:109BA800010300934FF006004FF03201C5F307227E
:109BB8004FF0020305F000FF34E340F29C23C2F2A9
:109BC80000039B68012B26D01BB1022B40F02A838F
:109BD80043E04FF000004FF0230144F2F832C0F6A2
:109BE8000102034605F076FE4FF000004FF02D010C
:109BF80044F21042C0F60102034605F06BFE4FF036
:109C080000004FF0370144F22842C0F60102034633
:109C180005F060FE06E34FF000004FF0230144F228
:109C28004042C0F60102034605F054FE4FF0000022
:109C38004FF02D0143F60C62C0F60102034605F011
:109C480049FE4FF000004FF0370144F25842C0F689
:109C58000102034605F03EFEE4E24FF000004FF03B
:109C6800230144F27042C0F60102034605F032FEB9
:109C78004FF000004FF02D0143F60C62C0F60102D0
:109C8800034605F027FE4FF000004FF0370144F27D
:109C98008842C0F60102034605F01CFEC2E240F20B
:109CA8009C23C2F200039B68012B1BD01BB1022B23
:109CB80040F0B8822DE04FF000004FF0280144F248
:109CC800A042C0F60102034605F004FE4FF0000072
:109CD8004FF0320144F2B842C0F60102034605F0E3
:109CE800F9FD9FE24FF000004FF0280144F2A04236
:109CF800C0F60102034605F0EDFD4FF000004FF0FD
:109D0800320144F2B842C0F60102034605F0E2FD12
:109D180088E24FF000004FF0280144F2A042C0F65C
:109D28000102034605F0D6FD4FF000004FF0320166
:109D380044F2B842C0F60102034605F0CBFD71E2D9
:109D48004FF000004FF0230144F2F832C0F6010250
:109D5800034605F0BFFD4FF000004FF02D0144F21F
:109D6800D042C0F60102034605F0B4FD4FF00000F2
:109D78004FF0370144F2E842C0F60102034605F00D
:109D8800A9FD4FE240F29C23C2F200039B68012B1D
:109D980026D01BB1022B40F0458243E04FF0000073
:109DA8004FF0230144F20052C0F60102034605F0C9
:109DB80091FD4FF000004FF02D0144F21852C0F60B
:109DC8000102034605F086FD4FF000004FF0370111
:109DD80044F23052C0F60102034605F07BFD21E251
:109DE8004FF000004FF0230144F24852C0F6010240
:109DF800034605F06FFD4FF000004FF02D0144F2CF
:109E08006052C0F60102034605F064FD4FF0000001
:109E18004FF0370144F27852C0F60102034605F0CC
:109E280059FDFFE14FF000004FF0230144F290523A
:109E3800C0F60102034605F04DFD4FF000004FF05B
:109E48002D0144F2A852C0F60102034605F042FD76
:109E58004FF000004FF0370144F2C052C0F6010243
:109E6800034605F037FDDDE140F29C23C2F2000312
:109E78009B68012B26D01BB1022B40F0D38143E015
:109E88004FF000004FF0230144F20052C0F60102E7
:109E9800034605F01FFD4FF000004FF02D0144F27E
:109EA800D852C0F60102034605F014FD4FF0000039
:109EB8004FF0370144F2F052C0F60102034605F0B4
:109EC80009FDAFE14FF000004FF0230144F2485282
:109ED800C0F60102034605F0FDFC4FF000004FF00C
:109EE8002D0144F20862C0F60102034605F0F2FCB7
:109EF8004FF000004FF0370144F27852C0F60102EB
:109F0800034605F0E7FC8DE14FF000004FF0230118
:109F180044F29052C0F60102034605F0DBFC4FF014
:109F280000004FF02D0144F22062C0F60102034602
:109F380005F0D0FC4FF000004FF0370144F2C0525A
:109F4800C0F60102034605F0C5FC6BE140F29C2314
:109F5800C2F200039B68012B26D01BB1022B40F0F4
:109F6800618143E04FF000004FF0230144F2386272
:109F7800C0F60102034605F0ADFC4FF000004FF0BB
:109F88002D0144F25062C0F60102034605F0A2FC1E
:109F98004FF000004FF0370144F26862C0F601024A
:109FA800034605F097FC3DE14FF000004FF0230118
:109FB80044F28062C0F60102034605F08BFC4FF0C4
:109FC80000004FF02D0143F60C62C0F60102034673
:109FD80005F080FC4FF000004FF0370144F2986222
:109FE800C0F60102034605F075FC1BE14FF00000C6
:109FF8004FF0230144F28842C0F60102034605F0FF
:10A0080069FC4FF000004FF02D0144F2B062C0F639
:10A018000102034605F05EFC4FF000004FF03701E7
:10A0280044F29862C0F60102034605F053FCF9E0D9
:10A038004FF000004FF0280144F2C862C0F6010258
:10A04800034605F047FCC5F30725002D40F0EA80DC
:10A058004FF000004FF0320144F2E062C0F6010216
:10A06800034605F037FCDDE04FF000004FF0280113
:10A0780044F2F062C0F60102034605F02BFC4FF0F3
:10A08800010300934FF01E004FF02801C5F307228B
:10A098004FF0020305F090FCC4E04FF030004FF0A1
:10A0A8000C0144F20872C0F601024FF0000305F0FB
:10A0B80011FC40F29C23C2F200039B68012B1AD0CA
:10A0C80013B1022B44D12DE04FF000004FF02401D2
:10A0D80044F21072C0F60102034605F0FBFB4FF094
:10A0E80000004FF02E0144F25C32C0F60102034634
:10A0F80005F0F0FB2CE04FF000004FF0240144F293
:10A108002872C0F60102034605F0E4FB4FF0000098
:10A118004FF02E0144F24072C0F60102034605F0EA
:10A12800D9FB15E04FF000004FF0240144F25872BB
:10A13800C0F60102034605F0CDFB4FF000004FF0DA
:10A148002E0144F27072C0F60102034605F0C2FB0C
:10A158004FF000004FF0380144F28872C0F6010257
:10A16800034605F0B7FB4FF0010600964FF00000DC
:10A178004FF03801C5F307224FF0020305F01CFC2D
:10A1880004F10205D4F8024000964FF012004FF097
:10A198003801E2B24FF0020305F00EFC00964FF0D2
:10A1A80024004FF03801C4F307224FF0020305F0F2
:10A1B80003FCD5F8024000964FF04E004FF03801EE
:10A1C800E2B24FF0020305F0F7FB00964FF0600093
:10A1D8004FF03801C4F307224FF0020305F0ECFBFF
:10A1E80020E04FF000004FF0230144F2A072C0F6C7
:10A1F8000102034605F06EFB4FF000004FF02D0101
:10A2080044F2B872C0F60102034605F063FB4FF052
:10A2180000004FF0370143F60C62C0F60102034616
:10A2280005F058FB03B0F0BD2DE9F04782B04FF0C0
:10A2380001073E464FF0000441F6EF25C2F2000543
:10A2480040F29C29C2F2000944F60C0AC0F6010A41
:10A258002B780A2B02BFFF232B700027FF2C25D059
:10A268002B78122B18D12CB104F1FF34E4B24FF043
:10A2780001060EE04FF46840C0F603004FF03201CB
:10A28800FFF776FAC0B220B100F1FF30C4B24FF048
:10A2980001064FF0FF032B702B780F2B06D104F12A
:10A2A8000104E4B24FF0FF032B7002E0002E00F02F
:10A2B800978004EB44064FEA860606F1006606F529
:10A2C8007A36326892B24FF6FF739A4248D006F057
:10A2D800F5F9D9F80830012B0FD013B1022B23D18F
:10A2E80017E04FF000004FF0010144F2D072C0F6C1
:10A2F8000102034605F0EEFA16E04FF000004FF0B9
:10A30800010144F2E072C0F60102034605F0E2FAE8
:10A318000AE04FF000004FF0010144F2F072C0F67D
:10A328000102034605F0D6FA4FF0010100914FF003
:10A33800420022464FF0020305F03EFB4FF00008B2
:10A34800CDF8008040464FF00A014FF07F024FF0F1
:10A358000B0305F0D7FF3046FFF73AFB46463FE0D0
:10A36800002C39D106F0AAF9D9F80830012B16D0FB
:10A378002BB1022B1CBF0026FF2431D11CE04FF06B
:10A388001E00014644F60002C0F601024FF0000329
:10A3980005F0A0FA4FF000064FF0FF0420E04FF060
:10A3A8001E00014652464FF0000305F093FA4FF0A5
:10A3B80000064FF0FF0413E04FF01E00014644F67C
:10A3C8001C02C0F601024FF0000305F083FA4FF0BB
:10A3D80000064FF0FF0403E04FF001064FF00004C1
:10A3E800002F7FF435AF02B0BDE8F0874FF4684323
:10A3F800C0F60303186880B24FF6FF73C01A18BF7F
:10A4080001207047F0B583B04FF46840C0F60300F0
:10A418004FF05001FFF7ACF9C4B2002C00F01D81D9
:10A428004DF6FE73C0F603031E68B6B24DF2FE7316
:10A43800C0F603031D68ADB24FF6FF739D4214BF0B
:10A44800002201229E4214BF134642F00103002B52
:10A4580044D04FF45845C0F60305284604F040FEA2
:10A468004FF064004FF00101FAF700FB4FF450463B
:10A47800C0F60306304604F033FE04EB44044FEA0A
:10A48800440741F21824C2F200044FF46840C0F6B1
:10A4980003004FF0000122463B4604F077FE2846B1
:10A4A8004FF0000122463B4604F044FE4FF00107FE
:10A4B80002AC24F8047D284640F2FE7122463B4651
:10A4C80004F038FE4FF00003ADF80430304640F297
:10A4D800FE7122463B4604F02DFEBEE0AE425ED938
:10A4E8004FF45840C0F603004FF08201FFF740F9DF
:10A4F80005464F2826D84FF6FF73984222D004EB22
:10A5080044044FEA440641F21824C2F200044FF40E
:10A518006840C0F603004FF000012246334604F0BD
:10A5280035FE05EB45054FEA85054FF45840C0F662
:10A5380003004FF6FC7105EA01012246334604F098
:10A54800F9FD8AE04FF45045C0F60305284604F0AB
:10A55800C7FD04EB44044FEA440741F21824C2F251
:10A5680000044FF46840C0F603004FF00001224693
:10A578003B4604F00BFE28464FF0000122463B46BE
:10A5880004F0D8FD06F1010602AA22F8046D284657
:10A5980040F2FE714FF0010304F0CCFD5DE04FF492
:10A5A8005040C0F603004FF08201FFF7E1F806467D
:10A5B8004F2826D84FF6FF73984222D004EB440464
:10A5C8004FEA440541F21824C2F200044FF46840EF
:10A5D800C0F603004FF0000122462B4604F0D6FDDA
:10A5E80006EB46064FEA86064FF45040C0F60300D5
:10A5F8004FF6FC7106EA010122462B4604F09AFD4B
:10A608002BE04FF45846C0F60306304604F068FDC8
:10A6180004EB44044FEA440741F21824C2F2000450
:10A628004FF46840C0F603004FF0000122463B4655
:10A6380004F0ACFD30464FF0000122463B4604F0E2
:10A6480079FD05F1010502AA22F8045D304640F2C1
:10A65800FE714FF0010304F06DFD03B0F0BD00BFC3
:10A668002DE9F04F87B04DF6FE73C0F603031B6863
:10A678001FFA83F94DF2FE73C0F603031C68A4B2F7
:10A688004FF6FF739C4214BF00220122994514BF64
:10A69800134642F00103002B36D006F00FF840F2C3
:10A6A8009C23C2F200039B68012B0FD013B1022B2D
:10A6B80023D117E04FF01E00014644F60002C0F611
:10A6C80001024FF0000305F005F916E04FF01E00F7
:10A6D800014644F60C02C0F601024FF0000305F0F3
:10A6E800F9F80AE04FF01E00014644F61C02C0F6D5
:10A6F80001024FF0000305F0EDF84FF4FA604FF057
:10A708000101FAF7B3F982E14FF45840C0F60300AB
:10A718004FF08201FFF72CF883464FF6FF739842FB
:10A7280008BF4FF0500B4FF45040C0F603004FF0F5
:10A738008201FFF71DF882464FF6FF73984208BF63
:10A748004FF0500AA1458CBF4FF000094FF00109A6
:10A75800B9F1000F15D04DF2FE78C0F60308BAF132
:10A76800000F00F032810AF1FF3303EB43034FEA95
:10A77800830808F1006808F574380AF1FF35EDB26E
:10A7880023E14DF2FE78C0F60308BBF1000F00F09C
:10A798001C810BF1FF3303EB43034FEA830808F1F5
:10A7A800006808F576380BF1FF35EDB20DE1237836
:10A7B800092B33D841F2D7104FF6FF714FF0010241
:10A7C80000F042FA38B305F079FF4FF01E00014659
:10A7D80044F62802C0F601024FF0000305F07AF8AB
:10A7E8004FF45840C0F6030004F07AFC4FF06400C0
:10A7F8004FF00101FAF73AF94FF45040C0F6030060
:10A8080004F06EFC4FF4FA604FF00101FAF72EF9EC
:10A818004FF0000637464FF0FF03237023780A2BCA
:10A8280002BFFF23237000262378122B46D1B9F1EB
:10A83800000F1ED005F10105EDB2AA4510D84FF062
:10A8480000054FF45048C0F60308BBF1000F30D0A4
:10A858004FF000094D464FF45848C0F6030828E069
:10A8680005EB45084FEA880808F1006808F57438D0
:10A878001FE005F10105EDB2AB4512D8BAF1000FA2
:10A8880018BF4FF001094FF000054FF45848C0F6C3
:10A8980003084FF45043C0F60303AA4518BF98466F
:10A8A80007E005EB45084FEA880808F1006808F555
:10A8B80076384FF0FF0323704FF0010723780F2BF2
:10A8C8003FD1B9F1000F1DD05DB105F1FF35EDB2F3
:10A8D80005EB45084FEA880808F1006808F5743860
:10A8E8002BE0BBF1000F05D0059DDDF80C804FF083
:10A8F800000922E00AF1FF35EDB2DDF810804FF0D3
:10A9080001091AE05DB105F1FF35EDB205EB450827
:10A918004FEA880808F1006808F576380DE0BAF1C2
:10A92800000F07D00AF1FF35EDB2DDF810804FF0C7
:10A93800010902E0059DDDF80C804FF0FF0323704C
:10A9480001E0002F3DD005F0B9FE40F29C23C2F291
:10A9580000039B68012B0FD013B1022B23D117E002
:10A968004FF000004FF0010144F63802C0F6010232
:10A97800034604F0AFFF16E04FF000004FF001016E
:10A9880044F64402C0F60102034604F0A3FF0AE0BD
:10A998004FF000004FF0010144F65002C0F60102EA
:10A9A800034604F097FF4FF00007009738464FF032
:10A9B8000B014FF07F020B4605F0A4FC4046FFF761
:10A9C80007F8002E7FF4F3AE21E00BF1FF3303EB21
:10A9D80043034FEA830303F1006303F576330393DC
:10A9E8000AF1FF3303EB43034FEA830303F10063E8
:10A9F80003F5743304934FF00106374641F6EF240C
:10AA0800C2F200040BF1FF33DBB20593CFE607B0C7
:10AA1800BDE8F08F4FF43053C4F200035A6822F4B3
:10AA2800C07240EA02025A60704700BF82B04FF01D
:10AA3800000301934FF43053C4F200035A6822F024
:10AA48007F020192019A00F07F0040EA020201921F
:10AA5800019A5A6002B0704700F07F004FF43053FB
:10AA6800C4F200031860704740F080004FF4305380
:10AA7800C4F20003186070474FF43053C4F2000367
:10AA88004FF000029A60704710B44FF44843C0F684
:10AA980003031B68DCB24CF60202C0F6030213681B
:10AAA800D9B24CF60402C0F603021368DBB24FF0C9
:10AAB8000000002B2FD046F6B842C4F200021288DC
:10AAC80092B29A421DD146F6B443C4F200031B88E1
:10AAD8009BB28B420AD146F6B043C4F200031888F1
:10AAE80080B2A04234BF0020012014E046F6B443EF
:10AAF800C4F20003188880B281422CBF00200120D4
:10AB080009E046F6B842C4F20002108880B28342D7
:10AB18002CBF0020012010BC704700BF30B5A1B089
:10AB28004FF46040C0F603004FF000016A464FF052
:10AB3800400304F02BFB41F60733C2F200031A78F6
:10AB480041F61733C2F200031B78C2EB021203EB83
:10AB58008205ADB24FF000031C464FF0010200A879
:10AB6800C118887868B1487800F10F001DF8031003
:10AB7800C1EB011100EB81018D42CCBF144394431A
:10AB880000E0144303F10403802B02D04FEA420291
:10AB9800E5E74FF09800A1B2FDF790FF4FF09C0059
:10ABA8004FEA1441FDF78AFF21B030BD10B5A0B0BF
:10ABB8004FF00003194620A8C21802F8801C03F1C0
:10ABC8000103DBB2802BF6D14FF098004FF6FF71EE
:10ABD800FDF774FF4FF09C004FF6FF71FDF76EFF15
:10ABE8004FF46044C0F60304204604F079FA204686
:10ABF8004FF000016A464FF0400304F09BFA20B082
:10AC080010BD00BF00B583B04FF000038DF80430CD
:10AC18008DF805304FF44840C0F603004FF00601A8
:10AC280001AA4FF0010304F085FA03B000BD00BF8C
:10AC38004CF60603C0F603031868C0B2D0F1010051
:10AC480038BF0020704700BF2DE9F04F85B0039052
:10AC58008B464FF00107002A00F0058105F02EFD14
:10AC680040F29C23C2F200039B68012B1BD013B156
:10AC7800022B47D12FE04FF00100014644F65C0259
:10AC8800C0F601024FF0000304F024FE4FF032003A
:10AC98004FF01E0144F67002C0F601024FF00003A7
:10ACA80004F018FE2EE04FF00100014644F6780249
:10ACB800C0F601024FF0000304F00CFE4FF0320022
:10ACC8004FF01E0144F68C02C0F601024FF000035B
:10ACD80004F000FE16E04FF00100014644F694022D
:10ACE800C0F601024FF0000304F0F4FD4FF032000B
:10ACF8004FF01E0144F68C02C0F601024FF000032B
:10AD080004F0E8FD4FF00007009738464FF00B01BC
:10AD18004FF07F020B4605F0F5FA41F6EF23C2F239
:10AD280000034FF0FF021A70B9463D464FF0010686
:10AD38001C46B846BA4623780A2B08BF464608BFC1
:10AD4800574623780C2B4BD1D94514BF0023012338
:10AD5800039A914508BF43F00103002B3DD14FF002
:10AD680032004FF01E0144F6A802C0F60102434625
:10AD780004F0B0FD40F29C23C2F200039B68012B53
:10AD88000FD013B1022B23D117E04FF014004FF06E
:10AD9800320144F6B002C0F60102434604F09AFDBF
:10ADA80016E04FF002004FF0320144F6C402C0F63C
:10ADB8000102434604F08EFD0AE04FF00A004FF00E
:10ADC800320144F6DC02C0F60102434604F082FD7B
:10ADD8004FF0FF032370454602E046464FF0010757
:10ADE8002378092B3CD8D5B94FF032004FF01E011B
:10ADF80044F6A802C0F60102434604F06BFD94F83D
:10AE080000904FF032004FF01E0144F64012C0F699
:10AE18000102434604F05EFD4FF001051DE009EB19
:10AE28008909237803EB49091FFA89F905EB4500DD
:10AE38004FEA400000F1320000F0FE004FF01E0122
:10AE480044F64012C0F60102434604F043FD05F102
:10AE58000105EDB2032D88BF00254FF0FF032370D5
:10AE6800002E7FF468AF384605B0BDE8F08F00BF0C
:10AE78002DE9F04F89B0824605F020FC4FF0000420
:10AE88000094204621464FF07F024FF03F0305F023
:10AE980039FA009420464FF00B014FF07F020B4621
:10AEA80005F030FA40F29C23C2F200039B68012BA4
:10AEB80010D013B1022B26D119E04FF01E004FF02D
:10AEC800020144F6F402C0F601024FF0000304F058
:10AED80001FD18E04FF01E004FF0020144F6041285
:10AEE800C0F601024FF0000304F0F4FC0BE04FF051
:10AEF80014004FF0020144F61412C0F601024FF09C
:10AF0800000304F0E7FC4FF002004FF0370144F66D
:10AF18002412C0F601024FF0000304F0DBFC524695
:10AF28004FF0000312F8011B29B103F10103DBB252
:10AF3800202BF7D100E09B46BBF1010F91BF3D20CC
:10AF48004FEA5B03A3EB8303580084BF403000F053
:10AF5800FE004FF01E0152464FF0000304F0BAFC09
:10AF680041F6EF23C2F200034FF0FF021A70D046F9
:10AF78004FF00003039304930793069399461D46E5
:10AF88004FF0010741F6EF24C2F200041E46059374
:10AF980023780A2B01BFFF2323703546059F2378AA
:10AFA8000C2B07D1B9F1000F08BF00254FF0FF03A4
:10AFB800237037462378092B46D8092D44D8B9F190
:10AFC800000F16D14FF002004FF01E0143F60C623D
:10AFD800C0F60102334604F07DFC237803F1300308
:10AFE800D04608F8013B8AF801604FF00109059D39
:10AFF80008E0237803F1300388F8003008F8016F7F
:10B00800012D08D84FF03D004FF01E01524633463F
:10B0180004F060FC0FE04FEA5503A3EB83034FEA0B
:10B02800430000F1400000F0FE004FF01E015246C0
:10B03800334604F04FFC05F10105EDB24FF0FF0374
:10B0480023704FF0010304932378102B64D1049BE1
:10B05800002B3CD14FF002004FF01E0143F60C626A
:10B06800C0F60102334604F035FC069B2BB1D046EE
:10B078004FF00109002B4CD014E0D0464FF02D03BF
:10B0880008F8013B8AF801604FF03D004FF01E01BF
:10B098005246059B04F01EFC4FF0010306939946A7
:10B0A8001D4636E0D0464FF02B0308F8013B8AF8DE
:10B0B80001604FF03D004FF01E015246059B04F021
:10B0C80009FC059B06934FF001094D4621E0B9F1B3
:10B0D800000F1ED0079BE3B94FF02E0388F800300D
:10B0E80008F8016F012D91BF3D206B08A3EB830386
:10B0F800580084BF403000F0FE004FF01E01524659
:10B10800334604F0E7FB05F10105EDB24FF001030A
:10B1180007934FF0FF03237023780E2B45D1B9F125
:10B12800000F12D1BBF1000F16D0039B1BB9D844F6
:10B138004FF00103039308F8016D0BF1FF3B5FFA31
:10B148008BFB5D464FF0010906E0002D39D005F173
:10B15800FF35EDB208F8016D4FF002004FF01E0107
:10B1680043F60C62C0F60102334604F0B3FB012D2E
:10B1780008D84FF03D004FF01E015246334604F008
:10B18800A9FB0FE04FEA5503A3EB83034FEA430003
:10B1980000F1400000F0FE004FF01E015246334619
:10B1A80004F098FB4FF0FF0323702378132B04BFA0
:10B1B800FF232370002F7FF4EBAE284609B0BDE8CB
:10B1C800F08F4FF002004FF01E0143F60C62C0F6FC
:10B1D8000102334604F07EFBCBE700BF2DE9F04FB8
:10B1E80085B083460391174641F6EF23C2F2000368
:10B1F8004FF0FF021A704FF000094FF001054E465C
:10B208001C46C84644F63C1AC0F6010A23780A2BA5
:10B2180004BF3E46454606D023780C2B08BF3E4661
:10B228000C2B08BF00252378122B04BF3E46454649
:10B2380006D023780F2B08BF3E460F2B08BF0025EA
:10B248002378092B6CD8B9F1000F06D15846039919
:10B258005246434604F03EFB09E0B9F1030F58D8C3
:10B26800B9F1030F3BD8DFE809F002102336237841
:10B27800022B237883BF64275F434FF001094FF403
:10B288007A779CBF5F43C14629E0B7F5FA6F09D3C7
:10B298002378032B8FBF84F800802378642202FB75
:10B2A80003771CE023784FF0640202FB037716E073
:10B2B8002378052B09D941F6EF23C2F200031E7843
:10B2C8004FF0FF021A70F6192DE0237803EB830381
:10B2D80007EB430703E02378FF183E464546B9F1DC
:10B2E800010F227899BF09EB49000BEB40000BF1E5
:10B2F800060309EB490088BF03EB40004FF0010348
:10B308000093C0B2039904F057FB09F101095FFAF1
:10B3180089F94FF0FF032370002D7FF477AF02E027
:10B32800002D7FF473AF304605B0BDE8F08F00BF45
:10B338002DE9F04F87B0814603911746062888BF4C
:10B348004FF00009022A14BF4FF00A0A4FF0090A09
:10B3580041F6EF23C2F200034FF0FF021A704FF0DC
:10B36800010846461C46A7F10A0B5FFA8BFB44F618
:10B378005C32C0F60102059223780A2B02BFFF2334
:10B38800237000262378122B02D023780F2B58D154
:10B398000AFB05F1C9B2022F0DD101F10A0E4FF0D7
:10B3A800010300934FF000004FF07F025FFA8EF325
:10B3B80004F0A8FF0EE001F10B0201F115034FF0B4
:10B3C800010100914FF00000D1B24FF07F02DBB2D3
:10B3D80004F098FF2378122B08D11DB105F1FF3531
:10B3E800EDB203E0049B03F1FF35EDB223780F2B98
:10B3F80006D105F10105EDB2049A954228BF002552
:10B408000AFB05F1C9B2022F0BD101F10A0E4FF068
:10B41800000000904FF07F025FFA8EF304F072FF95
:10B428000CE001F10B0201F115034FF00000009050
:10B43800D1B24FF07F02DBB204F064FF4FF0FF039C
:10B448002370BBF1090F06D823780B2B01BFA9463F
:10B45800FF232370002623780C2B01BFA946FF2366
:10B4680023700026B8F1000F00F0218405F026F9BA
:10B478004FF001000146039A4FF0000304F02AFA46
:10B48800039A92F900304BB14FF0000000904FF052
:10B4980009014FF07F020B4604F034FF0A2F00F237
:10B4A800CD83DFE817F00B006E00F5001202CB0326
:10B4B800CB037502CB03CB03CB03FC0240F29C23E6
:10B4C800C2F200039B68012B23D033B1022B1CBFAF
:10B4D8000223049340F0CA8337E04FF032004FF064
:10B4E8000D0143F61032C0F601024FF0000304F0DC
:10B4F800F1F94FF032004FF0170143F60432C0F66D
:10B5080001024FF0000304F0E5F94FF00202049243
:10B51800D4E34FF032004FF00D0143F61432C0F679
:10B5280001024FF0000304F0D5F94FF032004FF05C
:10B53800170143F60832C0F601024FF0000304F089
:10B54800C9F94FF002030493BCE34FF032004FF007
:10B558000D0143F61832C0F601024FF0000304F063
:10B56800B9F94FF032004FF0170143F60C32C0F62C
:10B5780001024FF0000304F0ADF94FF0020204920B
:10B5880074E340F29C23C2F200039B68012B2FD086
:10B5980033B1022B1CBF0322049240F067834FE0B3
:10B5A8004FF01E004FF00D0143F62032C0F60102A5
:10B5B8004FF0000304F08EF94FF01E004FF0170112
:10B5C80043F62C32C0F601024FF0000304F082F972
:10B5D8004FF01E004FF0210143F63832C0F6010249
:10B5E8004FF0000304F076F94FF00303049365E38A
:10B5F8004FF01E004FF00D0143F64832C0F601022D
:10B608004FF0000304F066F94FF01E004FF01701E9
:10B6180044F64412C0F601024FF0000304F05AF950
:10B628004FF01E004FF0210143F66032C0F60102D0
:10B638004FF0000304F04EF94FF00302049241E387
:10B648004FF01E004FF00D0143F66C32C0F60102B8
:10B658004FF0000304F03EF94FF01E004FF01701C1
:10B6680043F67432C0F601024FF0000304F032F9D9
:10B678004FF01E004FF0210143F68032C0F6010260
:10B688004FF0000304F026F94FF003030493EDE2B2
:10B6980040F29C23C2F200039B68012B62D033B1B5
:10B6A800022B1CBF0723049340F0E082B5E04FF063
:10B6B8001E004FF0020144F64C12C0F601024FF092
:10B6C800000304F007F94FF01E004FF00B0144F699
:10B6D8005412C0F601024FF0000304F0FBF84FF0DB
:10B6E8001E004FF0140144F65C12C0F601024FF040
:10B6F800000304F0EFF84FF01E004FF01D0144F670
:10B708006412C0F601024FF0000304F0E3F84FF0B2
:10B718001E004FF0260144F66C12C0F601024FF0ED
:10B72800000304F0D7F84FF01E004FF02F0144F645
:10B738007412C0F601024FF0000304F0CBF84FF08A
:10B748001E004FF0380144F67C12C0F601024FF09B
:10B75800000304F0BFF809FB0AF1C9B24FF0070271
:10B76800049288E24FF01E004FF0020144F6841262
:10B77800C0F601024FF0000304F0ACF84FF01E00D1
:10B788004FF00B0144F69012C0F601024FF000038F
:10B7980004F0A0F84FF01E004FF0140144F69C127C
:10B7A800C0F601024FF0000304F094F84FF01E00B9
:10B7B8004FF01D0144F6A812C0F601024FF0000335
:10B7C80004F088F84FF01E004FF0260144F6B4123A
:10B7D800C0F601024FF0000304F07CF84FF01E00A1
:10B7E8004FF02F0144F6C012C0F601024FF00003DB
:10B7F80004F070F84FF01E004FF0380144F6CC12F8
:10B80800C0F601024FF0000304F064F809FB0AF1E6
:10B81800C9B24FF0070304932DE24FF01E004FF01A
:10B82800020144F6D812C0F601024FF0000304F0FA
:10B8380051F84FF01E004FF00B0144F6E412C0F629
:10B8480001024FF0000304F045F84FF01E004FF0DE
:10B85800140144F6F412C0F601024FF0000304F09C
:10B8680039F84FF01E004FF01D0144F60022C0F6D3
:10B8780001024FF0000304F02DF84FF01E004FF0C6
:10B88800260144F60822C0F601024FF0000304F036
:10B8980021F84FF01E004FF02F0144F61422C0F695
:10B8A80001024FF0000304F015F84FF01E004FF0AE
:10B8B800380144F62022C0F601024FF0000304F0DC
:10B8C80009F84FF007020492D0E140F29C23C2F23B
:10B8D80000039B68012B23D033B1022B1CBF02222B
:10B8E800049240F0C38137E04FF01E004FF00D0185
:10B8F80043F69432C0F601024FF0000303F0EAFF6A
:10B908004FF01E004FF0170143F68832C0F60102CF
:10B918004FF0000303F0DEFF4FF002030493CDE184
:10B928004FF01E004FF00D0143F69432C0F60102AD
:10B938004FF0000303F0CEFF4FF01E004FF0170149
:10B9480043F68832C0F601024FF0000303F0C2FF4D
:10B958004FF002020492B5E14FF01E004FF00D01C6
:10B9680043F69432C0F601024FF0000303F0B2FF31
:10B978004FF01E004FF0170143F68832C0F601025F
:10B988004FF0000303F0A6FF4FF0020304936DE1AC
:10B9980040F29C23C2F200039B68012B2FD033B1E5
:10B9A800022B1CBF0323049340F060814FE04FF04B
:10B9B8001E004FF00D0144F62C22C0F601024FF094
:10B9C800000303F087FF4FF01E004FF0170144F605
:10B9D8003022C0F601024FF0000303F07BFF4FF066
:10B9E8001E004FF0210144F63C22C0F601024FF040
:10B9F800000303F06FFF4FF0030204925EE14FF083
:10BA08001E004FF00D0144F64822C0F601024FF027
:10BA1800000303F05FFF4FF01E004FF0170144F6DC
:10BA28005022C0F601024FF0000303F053FF4FF01D
:10BA38001E004FF0210144F65C22C0F601024FF0CF
:10BA4800000303F047FF4FF0030304933AE14FF07C
:10BA58001E004FF00D0144F66822C0F601024FF0B7
:10BA6800000303F037FF4FF01E004FF0170144F6B4
:10BA78007422C0F601024FF0000303F02BFF4FF0D1
:10BA88001E004FF0210144F68022C0F601024FF05B
:10BA9800000303F01FFF4FF003020492E6E040F2B8
:10BAA8009C23C2F200039B68012B47D033B1022BC1
:10BAB8001CBF0522049240F0D9807FE04FF01400AB
:10BAC8004FF00D0144F68C22C0F601024FF000033E
:10BAD80003F000FF4FF014004FF0170144F69C22CA
:10BAE800C0F601024FF0000303F0F4FE4FF014001B
:10BAF8004FF0210144F6AC22C0F601024FF00003DA
:10BB080003F0E8FE4FF014004FF02B0144F6BC227E
:10BB1800C0F601024FF0000303F0DCFE4FF0140002
:10BB28004FF0350144F6CC22C0F601024FF0000375
:10BB380003F0D0FE4FF005030493BFE04FF014006C
:10BB48004FF00D0144F6DC22C0F601024FF000036D
:10BB580003F0C0FE4FF014004FF0170144F6EC223A
:10BB6800C0F601024FF0000303F0B4FE4FF01400DA
:10BB78004FF0210144F6FC22C0F601024FF0000309
:10BB880003F0A8FE4FF014004FF02B0144F60C32DE
:10BB9800C0F601024FF0000303F09CFE4FF01400C2
:10BBA8004FF0350144F61C32C0F601024FF0000395
:10BBB80003F090FE4FF00502049283E04FF014006A
:10BBC8004FF00D0144F62C32C0F601024FF000038D
:10BBD80003F080FE4FF014004FF0170144F6EC22FA
:10BBE800C0F601024FF0000303F074FE4FF014009A
:10BBF8004FF0210144F6FC22C0F601024FF0000389
:10BC080003F068FE4FF014004FF02B0144F63C326D
:10BC1800C0F601024FF0000303F05CFE4FF0140081
:10BC28004FF0350144F64C32C0F601024FF00003E4
:10BC380003F050FE4FF00503049317E04FF0140093
:10BC48004FF00D01059A4FF0000303F043FE4FF04B
:10BC580014004FF0170144F67432C0F601024FF099
:10BC6800000303F037FE4FF00002049209FB0AF1CB
:10BC7800C9B2022F0AD101F10A054FF00000009065
:10BC88004FF07F02EBB204F03DFB0CE001F10B0238
:10BC980001F115034FF000000090D1B24FF07F0280
:10BCA800DBB204F02FFB5FFA89F54FF00008002E95
:10BCB8007FF462AB484607B0BDE8F08F09FB0AF194
:10BCC800C9B2E3E709FB0AF1C9B2DFE72DE9F04F92
:10BCD80093B04FF44843C0F603031B684CF60203C5
:10BCE800C0F603031B684CF60403C0F603031B6885
:10BCF8004CF60803C0F60303196840F29C23C2F20D
:10BD0800000341F6EE0089B21A79FEF79DFF00287C
:10BD180000F0D88646F6B843C4F20003B3F800A092
:10BD28005FFA8AFA46F6B443C4F20003B3F800B0E7
:10BD38005FFA8BFB46F6B043C4F200031B88DBB204
:10BD4800049346F6AC43C4F200031B88DBB20393AA
:10BD580041F60733C2F200031B78069341F6173306
:10BD6800C2F200031B78059341F61533C2F20003B3
:10BD78001B7807934FF44840C0F603004FF00001CA
:10BD88000BAA4FF0060303F001FA9DF835204FEA9D
:10BD980002229DF83430D3189BB2089341F6EF2362
:10BDA800C2F200034FF0FF021A704FF00009CDF8FD
:10BDB80024904F464D461C4640F29C28C2F200088B
:10BDC8002378122B02D023780F2B6DD105EBC501F8
:10BDD800C9B277B1042D01F109034FF001020092B5
:10BDE8004FF0610094BF73227F22DBB204F08AFA1D
:10BDF8000BE001F109034FF0010200924FF04D00F2
:10BE08004FF05E02DBB204F07DFA2378122B18D1D2
:10BE180037B1022D84BF05F1FF35EDB20ED804E02D
:10BE280045B105F1FF35EDB208E04FF000074FF0DE
:10BE3800060503E04FF001074FF005054FF0FF033B
:10BE4800237023780F2B0FD105F10105EDB227B12F
:10BE5800052D84BF00273D4603E0062D84BF01273A
:10BE680002254FF0FF03237005EBC501C9B277B176
:10BE7800042D01F109034FF0000200924FF0610018
:10BE880094BF73227F22DBB204F03CFA0FE001F189
:10BE980009034FF0000200924FF04D004FF05E0290
:10BEA800DBB204F02FFA1AE1002F00F0188104F039
:10BEB80005FC4FF0000000904FF00B014FF07F029F
:10BEC8000B4604F01FFAD8F80830012B40D01BB1FC
:10BED800022B40F0B48077E04FF00100014644F6B1
:10BEE8008832C0F601024FF0000303F0F3FC4FF074
:10BEF80001004FF0130144F69832C0F601024FF0EA
:10BF0800000303F0E7FC4FF001004FF01C0144F67A
:10BF1800A832C0F601024FF0000303F0DBFC4FF03B
:10BF280001004FF0250144F6B832C0F601024FF087
:10BF3800000303F0CFFC4FF001004FF02E0144F650
:10BF4800C832C0F601024FF0000303F0C3FC76E0EC
:10BF58004FF00100014644F6D832C0F601024FF016
:10BF6800000303F0B7FC4FF001004FF0130144F653
:10BF7800E832C0F601024FF0000303F0ABFC4FF0CB
:10BF880001004FF01C0144F6FC32C0F601024FF0EC
:10BF9800000303F09FFC4FF001004FF0250144F629
:10BFA8001042C0F601024FF0000303F093FC4FF07B
:10BFB80001004FF02E0144F62442C0F601024FF072
:10BFC800000303F087FC3AE04FF00100014644F615
:10BFD8003842C0F601024FF0000303F07BFC4FF03B
:10BFE80001004FF0130144F64C42C0F601024FF035
:10BFF800000303F06FFC4FF001004FF01C0144F602
:10C008006042C0F601024FF0000303F063FC4FF0FA
:10C0180001004FF0250144F67442C0F601024FF0CA
:10C02800000303F057FC4FF001004FF02E0144F6D7
:10C038008842C0F601024FF0000303F04BFC9DF864
:10C04800323063B14FF06E004FF0010144F69C426C
:10C05800C0F601024FF0000303F03CFC0BE04FF088
:10C068006E004FF0010143F6D442C0F601024FF0D2
:10C07800000303F02FFC9DF82C204FF001060096DA
:10C088004FF065004FF013014FF0020303F094FCEA
:10C098009DF82E2000964FF065004FF01C014FF0E0
:10C0A800020303F089FC9DF8302000964FF06500EC
:10C0B8004FF025014FF0020303F07EFC00964FF08D
:10C0C80065004FF02E01089A4FF0040303F074FC4A
:10C0D80005EBC501C9B2042D40F2BA82C5E204F0ED
:10C0E800EDFAD8F80830012B58D01BB1022B40F0DC
:10C0F800FC80A7E04FF00100014644F6A042C0F6DC
:10C1080001024FF0000303F0E5FB4FF001004FF090
:10C118000A0144F6B042C0F601024FF0000303F0F2
:10C12800D9FB4FF001004FF0130144F6C042C0F6AE
:10C1380001024FF0000303F0CDFB4FF001004FF078
:10C148001C0144F6D042C0F601024FF0000303F090
:10C15800C1FB4FF001004FF0250144F6E042C0F664
:10C1680001024FF0000303F0B5FB4FF001004FF060
:10C178002E0144F6F042C0F601024FF0000303F02E
:10C18800A9FB4FF001004FF0370144F60052C0F60A
:10C1980001024FF0000303F09DFBA6E04FF0010001
:10C1A800014644F61052C0F601024FF0000303F0B6
:10C1B80091FB4FF001004FF00A0144F61852C0F607
:10C1C80001024FF0000303F085FB4FF001004FF030
:10C1D800130144F62052C0F601024FF0000303F0A9
:10C1E80079FB4FF001004FF01C0144F62852C0F6CD
:10C1F80001024FF0000303F06DFB4FF001004FF018
:10C20800250144F63852C0F601024FF0000303F04E
:10C2180061FB4FF001004FF02E0144F64052C0F68A
:10C2280001024FF0000303F055FB4FF001004FF0FF
:10C23800370144F64852C0F601024FF0000303F0FC
:10C2480049FB52E04FF00100014644F6A042C0F617
:10C2580001024FF0000303F03DFB4FF001004FF0E7
:10C268000A0144F65452C0F601024FF0000303F0ED
:10C2780031FB4FF001004FF0130144F66452C0F651
:10C2880001024FF0000303F025FB4FF001004FF0CF
:10C298001C0144F67452C0F601024FF0000303F08B
:10C2A80019FB4FF001004FF0250144F68452C0F607
:10C2B80001024FF0000303F00DFB4FF001004FF0B7
:10C2C8002E0144F69452C0F601024FF0000303F029
:10C2D80001FB4FF001004FF0370144F6A452C0F6BD
:10C2E80001024FF0000303F0F5FA4FF00106009643
:10C2F8004FF05100314652464FF0020303F05CFB09
:10C3080000964FF051004FF00A015A464FF00203D1
:10C3180003F052FB00964FF051004FF01301049ABE
:10C328004FF0020303F048FBD8F80830B34278D046
:10C338001BB1022B40F05C81E7E00399062960D825
:10C34800DFE801F004111E2B384552004FF0510070
:10C358004FF01C0144F6B452C0F601024FF000033E
:10C3680003F0B8FA44E14FF051004FF01C0144F6D5
:10C37800B852C0F601024FF0000303F0ABFA37E100
:10C388004FF051004FF01C0144F6BC52C0F60102B8
:10C398004FF0000303F09EFA2AE14FF051004FF0EE
:10C3A8001C0144F6C052C0F601024FF0000303F02E
:10C3B80091FA1DE14FF051004FF01C0144F6C452B0
:10C3C800C0F601024FF0000303F084FA10E14FF0C9
:10C3D80051004FF01C0144F6C852C0F601024FF05C
:10C3E800000303F077FA03E14FF051004FF01C010E
:10C3F80044F6CC52C0F601024FF0000303F06AFA8B
:10C40800F6E04FF051004FF01C0144F6B452C0F66C
:10C4180001024FF0000303F05DFA4FF000030393AD
:10C42800E6E00399062960D8DFE801F004111E2B25
:10C43800384552004FF051004FF01C0144F6D052DD
:10C44800C0F601024FF0000303F044FAD0E04FF0C9
:10C4580051004FF01C0144F6B852C0F601024FF0EB
:10C46800000303F037FAC3E04FF051004FF01C010E
:10C4780044F6D452C0F601024FF0000303F02AFA42
:10C48800B6E04FF051004FF01C0144F6D852C0F608
:10C4980001024FF0000303F01DFAA9E04FF051002C
:10C4A8004FF01C0144F6DC52C0F601024FF00003C5
:10C4B80003F010FA9CE04FF051004FF01C0144F6D5
:10C4C800E052C0F601024FF0000303F003FA8FE0D8
:10C4D8004FF051004FF01C0144F6E452C0F601023F
:10C4E8004FF0000303F0F6F982E04FF051004FF0EF
:10C4F8001C0144F6D052C0F601024FF0000303F0CD
:10C50800E9F94FF00003039372E00399062960D814
:10C51800DFE801F004111E2B384552004FF051009E
:10C528004FF01C0144F6E852C0F601024FF0000338
:10C5380003F0D0F95CE04FF051004FF01C0144F6D5
:10C54800B852C0F601024FF0000303F0C3F94FE000
:10C558004FF051004FF01C0144F6EC52C0F60102B6
:10C568004FF0000303F0B6F942E04FF051004FF0EE
:10C578001C0144F6D852C0F601024FF0000303F044
:10C58800A9F935E04FF051004FF01C0144F6F05284
:10C59800C0F601024FF0000303F09CF928E04FF0C9
:10C5A80051004FF01C0144F6F452C0F601024FF05E
:10C5B800000303F08FF91BE04FF051004FF01C010E
:10C5C80044F6CC52C0F601024FF0000303F082F9A2
:10C5D8000EE04FF051004FF01C0144F6E852C0F64F
:10C5E80001024FF0000303F075F94FF000030393C5
:10C5F8004FF0010600964FF051004FF02501069AC2
:10C608004FF0020303F0D8F900964FF051004FF0B5
:10C618002E01059A4FF0020303F0CEF900964FF071
:10C6280051004FF03701079A4FF0020303F0C4F9A5
:10C6380005EBC501C9B201F109034FF000020092F0
:10C648004FF04D004FF05E02DBB203F05BFE18E0E6
:10C6580001F109034FF0000200924FF061004FF022
:10C668007302DBB203F04EFE0BE001F109034FF059
:10C67800000200924FF061004FF07F02DBB203F03E
:10C6880041FE4FF0FF0323702378122B08D0237844
:10C698000F2B05D023780A2B02D023780C2BF3D14B
:10C6A80023780C2B40F0EF814FF0FF032370002F0D
:10C6B80000F0D680A5F10203032B00F28280DFE8A8
:10C6C80003F002203E5B9DF82C004FF0020300931C
:10C6D8000EA94FF000024FF0010301F0AFFA0EA8C7
:10C6E800FEF7C6FB00286CD00EA84FF000014FF0F3
:10C6F800020201F00DFA1F2888BF01208DF82C00D6
:10C708005FE09DF82E004FF0020300930EA94FF052
:10C7180000024FF0010301F091FA0EA8FEF7A8FB02
:10C7280000284ED00EA84FF000014FF0020201F091
:10C73800EFF90C2888BF00208DF82E0041E09DF805
:10C7480030004FF0020300930EA94FF000024FF0A3
:10C75800010301F073FA0EA8FEF78AFB88B30EA84E
:10C768004FF000014FF0020201F0D2F9632888BFB0
:10C7780000208DF8300024E04FF00403009308985F
:10C788000EA94FF000024FF0010301F057FA0EA86E
:10C79800FEF76EFBA8B10EA84FF000014FF004029F
:10C7A80001F0B6F940F2574342F20F72904288BF47
:10C7B800184682B208928DF834004FEA10208DF89E
:10C7C80035004FF0FF038DF832309DF830304FF0D0
:10C7D8000109002B00F0578146F6B842C4F2000266
:10C7E800128892B29A422BD146F6B443C4F200039F
:10C7F8001A8892B29DF82E309A4211D146F6B0436B
:10C80800C4F200031B889BB29DF82C209A429EBF5D
:10C8180000238DF832304FF0010940F234812AE1CB
:10C8280046F6B442C4F20002128892B293423EBF66
:10C8380000238DF832304FF00109C0F024811DE14A
:10C8480046F6B842C4F20002128892B293423EBF42
:10C8580000238DF832304FF00109C0F0148110E147
:10C86800062D00F2DA80DFE805F0042242627194B6
:10C87800B7004FF00203009350460EA94FF0000294
:10C888004FF0010301F0DAF90EA8FEF7F1FA0028DB
:10C8980000F0C3800EA84FF000014FF0020201F033
:10C8A80037F9632888BF00205FFA80FAB5E04FF0B7
:10C8B8000203009358460EA94FF000024FF00103FF
:10C8C80001F0BCF90EA8FEF7D3FA002800F0A58005
:10C8D8000EA84FF000014FF0020201F019F900F123
:10C8E800FF330B2B88BF01205FFA80FB95E04FF0E8
:10C8F8000203009304980EA94FF000024FF00103C1
:10C9080001F09CF90EA8FEF7B3FA002800F0858024
:10C918000EA84FF000014FF0020201F0F9F800F103
:10C92800FF331E2B88BF0120C0B2049075E0039826
:10C9380043F62061C0F601014FF00202FEF7F8FC51
:10C94800062888BF0020C0B2039066E04FF00203BB
:10C95800009306980EA94FF000024FF0010301F072
:10C968006DF90EA8FEF784FA002856D00EA84FF0ED
:10C9780000014FF0020201F0CBF80999069A8242B1
:10C9880018BF01210991172888BF0020C0B206905E
:10C9980043E04FF00203009305980EA94FF0000200
:10C9A8004FF0010301F04AF90EA8FEF761FA0028DA
:10C9B80033D00EA84FF000014FF0020201F0A8F8A2
:10C9C800099B0599814218BF012309933B2888BF19
:10C9D8000020C0B2059020E04FF0020300930798B2
:10C9E8000EA94FF000024FF0010301F027F90EA83D
:10C9F800FEF73EFA88B10EA84FF000014FF0020290
:10CA080001F086F8099A079B834218BF0122099210
:10CA18003B2888BF0020C0B2079046F6B843C4F24E
:10CA28000003A3F800A046F6B043C4F2000304993B
:10CA3800198046F6B443C4F20003A3F800B046F6E2
:10CA4800AC43C4F20003039A1A80099BDBB1059931
:10CA5800C1EB01124FEA82024FF46163069903FBAE
:10CA68000123079A9818FBF767FFFBF79FFF4FF022
:10CA78000003099307E04FF0010904E04FF00109B2
:10CA880001E04FF0010923780A2B7FF499A941F6B8
:10CA9800EF23C2F200034FF0FF021A70FEF73EF8D0
:10CAA800B9F1000F0ED04FF44844C0F603042046F5
:10CAB80002F016FB20464FF000010BAA4FF00603C8
:10CAC80002F038FB13B0BDE8F08F00BF2DE9F04F3E
:10CAD80087B0FEF7ADF8054641F60733C2F200030A
:10CAE8001A7841F61733C2F200031B78C2EB021220
:10CAF80003EB82091FFA89F94FF0AC00FBF7FAFF44
:10CB0800C4B24FF0A000FBF7F5FF844219D04FF0F4
:10CB1800A0002146FBF7D2FF4FF098004FF000012C
:10CB2800FBF7CCFF4FF09C004FF00001FBF7C6FF6E
:10CB3800002D40F01281FDF7A7FF28B1FEF762F83B
:10CB48000BE1002D40F009814FF09C00FBF7D2FF6C
:10CB580080464FF09800FBF7CDFF4FEA0848804425
:10CB68004FF0000A4FF001054FF46044C0F603048B
:10CB7800564641F2981BC2F2000B40F26C12C2F208
:10CB88000002039241F25413C2F20003059340F2EB
:10CB98009612C2F200020492DCE02168CAB2C1F324
:10CBA8000721D4F80230DBB204F10404002B00F0B2
:10CBB800C18015EA080F40F0BD80C2EB021201EBFC
:10CBC800820292B29145C0F0B58002F10F02914500
:10CBD8000CDD06F101014FF00003009301934FF0C3
:10CBE8001800C9B21A46FCF7E7FD91E003F1FF33DC
:10CBF800032B00F28B80DFE803F002264F7340F22C
:10CC08008813C2F200031B784FF0C806002B7FD1AF
:10CC18004FF0C8068BF800604FF004003146FBF770
:10CC28004DFF4FF008004FF00101FBF747FF40F2BE
:10CC38008812C2F200024FF001031370039A1370B6
:10CC4800049A137064E040F28813C2F200031B7860
:10CC58004FF0C806002B5BD141F29913C2F20003D2
:10CC68004FF0C8061E704FF00C003146FBF726FF48
:10CC78004FF010004FF00101FBF720FF40F288133E
:10CC8800C2F200034FF002021A704FF00103039A38
:10CC98001370049A13703BE040F28813C2F2000349
:10CCA8001B784FF0C806002B32D140F28813C2F22D
:10CCB80000034FF003021A704FF014004FF0010107
:10CCC800FBF7FCFE4FF00103039A137041F2801248
:10CCD800C2F200021370049A13704FF0C80617E0EE
:10CCE8009BF800304FF0C80693B94FF01C004FF086
:10CCF8000101FBF7E3FE4FF00103039A1370059A55
:10CD08001370049A13704FF0C80601E04FF0C8067C
:10CD180048EA0508BAF1000F06D04FF09C004FEA28
:10CD28001841FBF7CBFE05E04FF098001FFA88F199
:10CD3800FBF7C4FE4FEA450506F10106F6B2BC4210
:10CD48007FF42BAF0AF1010A4EF28003C0F6030309
:10CD58009F4202D004F140071FE707B0BDE8F08FFB
:10CD68002DE9F04FA5B04FF46040C0F603004FF036
:10CD7800000104AA4FF0400302F008FA4FF09C00AB
:10CD8800FBF7B8FE80464FF09800FBF7B3FE4FEA7A
:10CD98000848804441F6EF23C2F200034FF0FF0237
:10CDA8001A704FF0010A4FF0000B5E461D4640F224
:10CDB8009C20C2F20000029048F21F51C5F2EB110C
:10CDC800039171E22B780F2B0CD11E2E9DBF0136DB
:10CDD800F6B24FEA4A0A4FF0010A88BF00264FF020
:10CDE800FF032B702B78122B0DD12EB106F1FF36D5
:10CDF800F6B24FEA5A0A03E04FF0004A4FF01F0616
:10CE08004FF0FF032B7003F059FC4FF00000009027
:10CE18004FF00B014FF07F020B4603F073FA029AB2
:10CE28009368012B10D013B1022B26D119E04FF0D3
:10CE380006004FF0010144F6F852C0F601024FF027
:10CE4800000302F047FD18E04FF006004FF0010123
:10CE580044F60C62C0F601024FF0000302F03AFDFE
:10CE68000BE04FF006004FF0010144F62062C0F6D7
:10CE780001024FF0000302F02DFD4FF000004FF0CB
:10CE8800140144F63062C0F60102034602F022FDA6
:10CE98004FF000004FF01E0144F64462C0F6010254
:10CEA800034602F017FD34464FF0010100914FF0A0
:10CEB800600072184FF0020302F07EFD24A800EB18
:10CEC800860313F8802CC2EB021213F87F3C03EBA5
:10CED8008202B2F5B46FA1BF00EB8603002203F80B
:10CEE800802C03F87F2C24A901EB860717F8802CE7
:10CEF8004FF00109CDF800904FF036004FF01401C3
:10CF08004FF0020302F058FD4FF042004FF01401B9
:10CF180043F68402C0F601024FF0000302F0DAFC87
:10CF280017F87F2CCDF800904FF048004FF014010F
:10CF38004FF0020302F040FD17F87E3C042B81BF3E
:10CF480024AA02EB8603002203F87E2C1AEA080FB3
:10CF58004FF074004FF0010119BF43F6D442C0F6F8
:10CF6800010244F69C42C0F601024FF0000302F0B1
:10CF7800B1FC02988368012B50D01BB1022B40F002
:10CF8800E48097E024A901EB860313F87E3C032B89
:10CF980037D8DFE803F0020F1C294FF036004FF0B6
:10CFA8001E0144F65862C0F601024FF0000302F079
:10CFB80091FCCAE04FF036004FF01E0144F6A02263
:10CFC800C0F601024FF0000302F084FCBDE04FF010
:10CFD80036004FF01E0144F66062C0F601024FF0C1
:10CFE800000302F077FCB0E04FF036004FF01E016E
:10CFF80043F66802C0F601024FF0000302F06AFC33
:10D00800A3E04FF036004FF01E0144F66C62C0F604
:10D0180001024FF0000302F05DFC96E024A800EB4B
:10D02800860313F87E3C032B37D8DFE803F0020FA2
:10D038001C294FF036004FF01E0144F67462C0F60A
:10D0480001024FF0000302F045FC7EE04FF036008D
:10D058004FF01E0144F6F022C0F601024FF0000323
:10D0680002F038FC71E04FF036004FF01E0144F634
:10D078006062C0F601024FF0000302F02BFC64E08E
:10D088004FF036004FF01E0144F67C62C0F60102F4
:10D098004FF0000302F01EFC57E04FF036004FF04F
:10D0A8001E0144F68462C0F601024FF0000302F04C
:10D0B80011FC4AE024AA02EB860313F87E3C032BFA
:10D0C80037D8DFE803F0020F1C294FF036004FF085
:10D0D8001E0144F65862C0F601024FF0000302F048
:10D0E800F9FB32E04FF036004FF01E0144F6F02213
:10D0F800C0F601024FF0000302F0ECFB25E04FF010
:10D1080036004FF01E0144F66062C0F601024FF08F
:10D11800000302F0DFFB18E04FF036004FF01E016D
:10D1280043F6A802C0F601024FF0000302F0D2FB5A
:10D138000BE04FF036004FF01E0144F68462C0F653
:10D1480001024FF0000302F0C5FB24A901EB8403A0
:10D1580013F8807C07EB870707EB870713F87F3CFA
:10D1680003EB8707BFB24FF036004FF014013A4681
:10D17800FEF734F880B2B84218BF4FF0010B24AA6A
:10D1880002EB84030399A1FB00124FEA521203F841
:10D19800802C4FF0640101FB120003F87F0C2B7800
:10D1A8000C2B58D14FF0000044F68C61C0F60101F9
:10D1B8004FF00A02FEF7BCF824AA02EB84034FF0F2
:10D1C800000203F87D2CC0B205283FD8DFE800F044
:10D1D800030B131B273324A800EB84034FF0000232
:10D1E80003F87E2C32E024A901EB84034FF00102FE
:10D1F80003F87E2C2AE024AA02EB84034FF00202F3
:10D2080003F87E2C22E024A800EB84034FF00302ED
:10D2180003F87E2C4FF0010203F87D2C16E024A9B8
:10D2280001EB84034FF0040203F87E2C4FF0020256
:10D2380003F87D2C0AE024AA02EB84034FF00502D0
:10D2480003F87E2C4FF0000203F87D2C4FF0FF030B
:10D258002B704FF0010B41F60733C2F200031A7826
:10D2680041F61733C2F200031B78194624A800EBD5
:10D27800840313F87E3CABB1C2EB021201EB8203CC
:10D288009BB200EB840414F8801CC1EB011114F864
:10D298007F2C02EB81018B42CCBF48EA0A0828EABE
:10D2A8000A0801E048EA0A082B780A2B7FF48AADBD
:10D2B8004FF098001FFA88F1FBF700FC4FF09C0034
:10D2C8004FEA1841FBF7FAFBBBF1000F0ED04FF401
:10D2D8006044C0F60304204601F002FF20464FF0E8
:10D2E800000104AA4FF0400301F024FF41F6EF23A8
:10D2F800C2F200034FF0FF021A7025B0BDE8F08FAC
:10D308002DE9F04782B041F6EF23C2F200034FF057
:10D31800FF021A704FF001064FF000073D46B04675
:10D328001C4640F29C29C2F2000945F20C0AC0F6DC
:10D33800010A23780A2B02BFFF2323704FF000084D
:10D348002378122B02D023780F2B47D105EB8501C8
:10D358004FEA4101C9B201F10A034FF001020092FC
:10D368004FF000004FF07F0203F0FE0302F0CAFF07
:10D378002378122B0DD11DB105F1FF35EDB208E070
:10D3880027B14FF001064FF0000702E04FF0010609
:10D39800374623780F2B0ED105F10105EDB22FB1D9
:10D3A800042D82BF012600273D4604E0052D82BFDB
:10D3B80001263746002505EB85014FEA4101C9B230
:10D3C80001F10A034FF0000000904FF0800203F0D3
:10D3D800FE0302F097FF4FF0FF03237023780C2B16
:10D3E80040F00881002F3ED04FEA4703DB1905EBD8
:10D3F8004303A3F10603042B00F2F880DFE803F0EF
:10D40800030614223000FDF72BF9EFE04FF6FF700A
:10D4180040F6560199F80420FDF716FC002800F0A4
:10D42800E580F3F7B3FFE1E04FF6FF7040F65601F1
:10D4380099F80420FDF708FC002800F0D780F7F7DA
:10D448001BF8D3E04FF6FF7041F6EE0199F804207F
:10D45800FDF7FAFB002800F0C980F5F73DFAC5E0B2
:10D46800F6F7BCFBC2E0052D00F2C080DFE805F04E
:10D478000313212427B14FF6FF7040F6560199F89F
:10D488000420FDF7E1FB002800F0B0804FF0000019
:10D49800F5F714FBAAE040F656004FF6FF7199F82D
:10D4A8000420FDF7D1FB002800F0A080FFF758FC0E
:10D4B8009CE0FEF70BFC99E0FCF7B6FE96E040F224
:10D4C8008E13C2F200034FF000021A70FCF78EFFB1
:10D4D800002851D04FF0000044F69C61C0F60101CD
:10D4E8000246FDF725FF002866D003F0E7F84FF065
:10D4F8000A004FF01E0144F6B062C0F601024FF078
:10D50800000302F0E7F940F29613C2F200034FF06D
:10D5180001061E7040F6B8303146F7F7A7FA03F057
:10D52800CDF84FF032004FF01E0144F6C862C0F645
:10D5380001024FF0000302F0CDF94FF46840C0F645
:10D54800030001F0CDFD4FF4FA603146F7F78EFA8B
:10D5580003F0B4F84FF028004FF01E0144F6D062F3
:10D56800C0F601024FF0000302F0B4F94FF4FA607C
:10D578003146F7F77BFA1FE003F0A0F84FF00A00F6
:10D588004FF01E0144F6DC62C0F601024FF00003C2
:10D5980002F0A0F94FF00A004FF0280144F6F062BB
:10D5A800C0F601024FF0000302F094F94FF4FA605C
:10D5B8004FF00101F7F75AFA4FF024004FF000013D
:10D5C800FBF77CFA4FF028004FF00001FBF776FAE2
:10D5D8000CE041F6EE004FF6FF7199F80420FDF7D4
:10D5E80033FB18B14FF00100F5F768FA4FF0FF036D
:10D5F800237002E0002E00F0AF81002F00F0BF8002
:10D6080003F05CF8D9F80830012B40D01BB1022B8D
:10D6180040F08E8177E04FF00200014644F6047234
:10D62800C0F601024FF0000302F054F94FF0020077
:10D638004FF00C0144F61C72C0F601024FF00003D3
:10D6480002F048F94FF002004FF0160144F6347228
:10D65800C0F601024FF0000302F03CF94FF002005F
:10D668004FF0200144F64C72C0F601024FF000035F
:10D6780002F030F94FF002004FF02A0144F66472CC
:10D68800C0F601024FF0000302F024F950E14FF018
:10D698000200014644F67C72C0F601024FF0000316
:10D6A80002F018F94FF002004FF00C0144F61C721A
:10D6B800C0F601024FF0000302F00CF94FF002002F
:10D6C8004FF0160144F63472C0F601024FF0000321
:10D6D80002F000F94FF002004FF0200144F6947276
:10D6E800C0F601024FF0000302F0F4F84FF0020018
:10D6F8004FF02A0144F6AC72C0F601024FF0000365
:10D7080002F0E8F814E14FF00200014644F6C47252
:10D71800C0F601024FF0000302F0DCF84FF00200FF
:10D728004FF00C0144F61C72C0F601024FF00003E2
:10D7380002F0D0F84FF002004FF0160144F6DC7208
:10D74800C0F601024FF0000302F0C4F84FF00200E7
:10D758004FF0200144F6F472C0F601024FF00003C6
:10D7680002F0B8F84FF002004FF02A0144F6647254
:10D77800C0F601024FF0000302F0ACF8D8E002F066
:10D788009DFFD9F80830012B49D01BB1022B40F07E
:10D79800CF8089E04FF00200014652464FF0000367
:10D7A80002F098F84FF002004FF00C0145F2240205
:10D7B800C0F601024FF0000302F08CF84FF00200AF
:10D7C8004FF0160145F23C02C0F601024FF000038B
:10D7D80002F080F84FF002004FF0200145F25402A9
:10D7E800C0F601024FF0000302F074F84FF0020097
:10D7F8004FF02A0145F26C02C0F601024FF0000317
:10D8080002F068F84FF002004FF0340145F284024C
:10D81800C0F601024FF0000302F05CF888E04FF018
:10D828000200014652464FF0000302F053F84FF051
:10D8380002004FF00C0145F29C02C0F601024FF0C5
:10D84800000302F047F84FF002004FF0160145F2CE
:10D85800B402C0F601024FF0000302F03BF84FF0AB
:10D8680002004FF0200145F2CC02C0F601024FF051
:10D87800000302F02FF84FF002004FF02A0145F2A2
:10D88800E402C0F601024FF0000302F023F84FF063
:10D8980002004FF0340145F2FC02C0F601024FF0DD
:10D8A800000302F017F843E04FF002000146524629
:10D8B8004FF0000302F00EF84FF002004FF00C0199
:10D8C80045F21412C0F601024FF0000302F002F80C
:10D8D8004FF002004FF0160145F22C12C0F601027B
:10D8E8004FF0000301F0F6FF4FF002004FF0200167
:10D8F80045F24412C0F601024FF0000301F0EAFFBE
:10D908004FF002004FF02A0145F25C12C0F6010206
:10D918004FF0000301F0DEFF4FF002004FF034013A
:10D9280045F27412C0F601024FF0000301F0D2FF75
:10D9380005EB85014FEA4101C9B201F10A034FF035
:10D948000006009630464FF0800203F0FE0302F016
:10D95800D9FC4FF0FF032370B8F1000F7FF4E9AC56
:10D96800F4F786FF40F28E13C2F200034FF0010273
:10D978001A7002B0BDE8F0874FF40053C4F20203F6
:10D988001A6802F0380240EA02021A60704700BFC3
:10D998004FF40053C4F202031A6822F010021A600E
:10D9A8001A6840EA02021A60704700BF4FF4005339
:10D9B800C4F2020340F22312C4F267525A6048F6D6
:10D9C800AB12CCF6EF525A60704700BF4FF40053C9
:10D9D800C4F202031A6942F080021A61704700BF5C
:10D9E8004FF40053C4F20203D86070474FF4005359
:10D9F800C4F20203DB6813F0010F13D14FF4005394
:10DA0800C4F20203DB6813F0040F0ED14FF4005385
:10DA1800C4F20203D86800F0100000280CBF0420EC
:10DA2800032070474FF0010070474FF00200704725
:10DA380010B50446FFF7DAFF012814BF00220122BF
:10DA4800002C0CBF002302F0010333B1013C0CBFD2
:10DA5800002302F00103002BF8D1002C08BF052099
:10DA680010BD00BF70B506460C464FF40050FFF7D6
:10DA7800DFFF042812D14FF40055C4F202052B69C8
:10DA880043F001032B6134804FF40050FFF7D0FFBF
:10DA98002A6941F6FE7302EA03032B6170BD00BFD9
:10DAA80038B505464FF43020FFF7C2FF042816D1D9
:10DAB8004FF40054C4F20204236943F002032361C3
:10DAC8006561236943F0400323614FF43020FFF779
:10DAD800AFFF226941F6FD7302EA0303236138BDF3
:10DAE80070B44FF000044FF00103264610F8015BB4
:10DAF800002D08BF002301F8015B04F10104A4B262
:10DB0800944228BF0E70002BF0D170BC704700BF44
:10DB18002DE9F00F82B00346007844B22D2C04BFE3
:10DB28005D1C4FF0010A06D040B22B280CBF5D1CCB
:10DB38001D464FF0000A95F90000002834D04FF038
:10DB480000008146844606464FF00107834601934C
:10DB580090462A782E2A04D1002E69D14FF001066A
:10DB68001EE02AB3A2F13004E4B2092C84BF4FF0BE
:10DB7800020C5F4610D800EB80004FEA4000A0F18D
:10DB88003000801809F101095FFA89F9C14581BFA0
:10DB980003221A70019D5F4616B106F10106F6B21E
:10DBA80037B105F10105D4E74FF000008446064679
:10DBB800002930D0A6B106F1FF36F6B2B14204D939
:10DBC800891BC9B24FF000050CE0B14224BF83F8AD
:10DBD80000C001231CD2711AC9B24FF0010501E03F
:10DBE8004FF0000583F800C00C464FF0010359B10F
:10DBF8004FF000024FF0010303EB83034FEA4303A6
:10DC080002F10102A242F7D315B1B0FBF3F006E02E
:10DC180003FB00F003E016B14FF001021A70BAF1ED
:10DC2800000F01D0C0F1000002B0BDE8F00F70474E
:10DC38004FF000004FF0010C6646B9E72DE9F00FF0
:10DC480004469DF820004FF0010B18B94FF0000B67
:10DC58004FF00A00904287BFC2EB00025FFA82F8D9
:10DC680010464FF000080546012898BF01220AD93E
:10DC78004FF00100024602EB82024FEA420200F135
:10DC88000100A842F7D3002CBFBF2D2001F8010BDB
:10DC980064420120A8BF0020B4FBF2F6092E82BF1F
:10DCA800452201F8012B012054D8D8F1010638BFCC
:10DCB8000026002C14BF002606F001060EB93DB957
:10DCC80048E04FF0300201F8012B4FF0010041E02D
:10DCD8004FF000064FF001094CF6CD4ACCF6CC4A7D
:10DCE80037469C4646450FD137B94FF0300301F807
:10DCF800013B00F10100C0B24FF02E0301F8013BD7
:10DD080000F10100C0B24F46B4FBF2F3DBB25BB9DD
:10DD180057EA0B0310D04FF0300301F8013B00F134
:10DD28000100C0B24F4607E003F1300301F8013BA0
:10DD380000F10100C0B24F4606F10106AE4208D21A
:10DD4800B4FBF2F302FB1344AAFB02324FEAD202FD
:10DD5800C8E7634613B14FF000030B70BDE8F00F3E
:10DD6800704700BF40F20003C2F200031A684FF088
:10DD78000003137040F20402C2F20002126813702A
:10DD880040F20802C2F200021268137040F20C025C
:10DD9800C2F200021268137040F21002C2F20002CE
:10DDA8001268137040F21402C2F200021268137073
:10DDB80040F21802C2F200021268137040F21C020C
:10DDC800C2F200021268137040F22002C2F200028E
:10DDD8001268137040F22402C2F200021268137033
:10DDE80040F22802C2F200021268137040F22C02BC
:10DDF800C2F200021268137040F23002C2F200024E
:10DE08001268137040F23402C2F2000212681370F2
:10DE180040F23802C2F200021268137040F23C026B
:10DE2800C2F200021268137040F24002C2F200020D
:10DE38001268137040F24402C2F2000212681370B2
:10DE480040F24802C2F200021268137040F24C021B
:10DE5800C2F200021268137040F25002C2F20002CD
:10DE68001268137040F25402C2F200021268137072
:10DE780040F25802C2F200021268137040F25C02CB
:10DE8800C2F200021268137040F26002C2F200028D
:10DE98001268137040F26402C2F200021268137032
:10DEA80040F26802C2F200021268137040F26C027B
:10DEB800C2F200021268137040F27002C2F200024D
:10DEC8001268137040F27402C2F2000212681370F2
:10DED80040F27802C2F200021268137040F27C022B
:10DEE800C2F200021268137040F28002C2F200020D
:10DEF8001268137040F28402C2F2000212681370B2
:10DF080040F28802C2F200021268137040F28C02DA
:10DF1800C2F200021268137040F29002C2F20002CC
:10DF28001268137040F29402C2F200021268137071
:10DF380040F29802C2F200021268137040F29C028A
:10DF4800C2F200021268137040F2A002C2F200028C
:10DF58001268137040F2A402C2F200021268137031
:10DF680040F2A802C2F200021268137040F2AC023A
:10DF7800C2F200021268137040F2B002C2F200024C
:10DF88001268137040F2B402C2F2000212681370F1
:10DF980040F2B802C2F200021268137040F2BC02EA
:10DFA800C2F2000212681370704700BF10B54FF438
:10DFB800C050C4F201004FF48041F9F73DFD00382C
:10DFC80018BF012040F29813C2F200031B78002BFF
:10DFD80047D000283CD040F29813C2F200031B78C7
:10DFE8000C2B07D940F29813C2F200034FF000043B
:10DFF8001C70B5E140F29813C2F200035B78EBB1F4
:10E0080040F29813C2F200034FF000045C7041F62E
:10E018001A32C2F2000210884FEA40004FF6FE7131
:10E0280000EA010111805988128892B20A405A8088
:10E038001A7802F10102D2B21A7091E140F29813F3
:10E04800C2F200034FF001025A704FF0000487E15A
:10E0580040F29813C2F200031C784FF000021A70C5
:10E068007EE198B141F61A32C2F200024FF6FE7311
:10E07800138040F29813C2F200035988128892B2B2
:10E088000A405A804FF001021A7062E140F21C0304
:10E09800C2F200031B681B784BB140F29813C2F21E
:10E0A80000035A8892B242F001025A800BE040F213
:10E0B8009812C2F20002538823F001034FEA034387
:10E0C8004FEA1343538040F21803C2F200031B685F
:10E0D8001B784BB140F29813C2F200035A8892B2EF
:10E0E80042F002025A800BE040F29812C2F200029B
:10E0F800538823F002034FEA03434FEA1343538044
:10E1080040F21403C2F200031B681B784BB140F2C3
:10E118009813C2F200035A8892B242F004025A805D
:10E128000BE040F29812C2F20002538823F0040375
:10E138004FEA03434FEA1343538040F21003C2F2FD
:10E1480000031B681B784BB140F29813C2F200031E
:10E158005A8892B242F008025A800BE040F29812B4
:10E16800C2F20002538823F008034FEA03434FEA40
:10E178001343538040F20C03C2F200031B681B7860
:10E188004BB140F29813C2F200035A8892B242F09F
:10E1980010025A800BE040F29812C2F20002538833
:10E1A80023F010034FEA03434FEA1343538040F22E
:10E1B8000803C2F200031B681B784BB140F29813A6
:10E1C800C2F200035A8892B242F020025A800BE051
:10E1D80040F29812C2F20002538823F020034FEA5B
:10E1E80003434FEA1343538040F20403C2F200038F
:10E1F8001B681B784BB140F29813C2F200035A888F
:10E2080092B242F040025A800BE040F29812C2F2F9
:10E218000002538823F040034FEA03434FEA1343B5
:10E22800538040F20003C2F200031B681B784BB115
:10E2380040F29813C2F200035A8892B242F0800268
:10E248005A800BE040F29812C2F20002538823F081
:10E2580080034FEA03434FEA1343538040F22003FD
:10E26800C2F200031B681B784BB140F29813C2F24C
:10E2780000035A8892B242F480725A800BE040F24E
:10E288009812C2F20002538823F480734FEA0343C2
:10E298004FEA1343538040F22403C2F200031B6881
:10E2A8001B784BB140F29813C2F200035A8892B21D
:10E2B80042F400725A800BE040F29812C2F2000257
:10E2C800538823F400734FEA03434FEA1343538000
:10E2D80040F22803C2F200031B681B784BB140F2DE
:10E2E8009813C2F200035A8892B242F480625A80AC
:10E2F8000BE040F29812C2F20002538823F48063C4
:10E308004FEA03434FEA1343538040F22C03C2F20F
:10E3180000031B681B784BB140F29813C2F200034C
:10E328005A8892B242F400625A800BE040F2981286
:10E33800C2F20002538823F400634FEA03434FEA12
:10E348001343538040F29813C2F200034FF00002C7
:10E358001A7040F29813C2F200034FF000045C7088
:10E3680040F29813C2F200035A88D2B21A715B883D
:10E3780013F4807F08D04FF4C050C4F201004FF46A
:10E388008061F9F787FB07E04FF4C050C4F2010041
:10E398004FF48061F9F78CFB40F29813C2F2000346
:10E3A8005B8813F4007F08D04FF4C050C4F201001A
:10E3B8004FF40061F9F76EFB07E04FF4C050C4F268
:10E3C80001004FF40061F9F773FB40F29813C2F2B1
:10E3D80000035B8813F4806F08D04FF4C050C4F278
:10E3E80001004FF48051F9F755FB07E04FF4C05096
:10E3F800C4F201004FF48051F9F75AFB40F2981328
:10E40800C2F200035B8813F4006F08D04FF4C050C9
:10E41800C4F201004FF40051F9F73CFB07E04FF458
:10E42800C050C4F201004FF40051F9F741FB9CB110
:10E43800FFF798FC40F29813C2F200034FF0000275
:10E448005A801A71082C9CBFC4F10904E4B240F246
:10E458009813C2F200035C7140F23003C2F2000369
:10E468001B681B784BB140F29813C2F20003DA889C
:10E4780092B242F00102DA800BE040F29812C2F246
:10E488000002D38823F001034FEA03434FEA134302
:10E49800D38040F23403C2F200031B681B784BB1EF
:10E4A80040F29813C2F20003DA8892B242F00202F4
:10E4B800DA800BE040F29812C2F20002D38823F00F
:10E4C80002034FEA03434FEA1343D38040F2380371
:10E4D800C2F200031B681B784BB140F29813C2F2DA
:10E4E8000003DA8892B242F00402DA800BE040F2CC
:10E4F8009812C2F20002D38823F004034FEA0343C0
:10E508004FEA1343D38040F23C03C2F200031B6876
:10E518001B784BB140F29813C2F20003DA8892B22A
:10E5280042F00802DA800BE040F29812C2F20002D0
:10E53800D38823F008034FEA03434FEA1343D380F9
:10E5480040F24003C2F200031B681B784BB140F253
:10E558009813C2F20003DA8892B242F01002DA800D
:10E568000BE040F29812C2F20002D38823F01003A5
:10E578004FEA03434FEA1343D38040F24403C2F205
:10E5880000031B681B784BB140F29813C2F20003DA
:10E59800DA8892B242F02002DA800BE040F2981258
:10E5A800C2F20002D38823F020034FEA03434FEA64
:10E5B8001343D38040F24803C2F200031B681B7860
:10E5C8004BB140F29813C2F20003DA8892B242F0DB
:10E5D8004002DA800BE040F29812C2F20002D388BF
:10E5E80023F040034FEA03434FEA1343D38040F23A
:10E5F8004C03C2F200031B681B784BB140F298131E
:10E60800C2F20003DA8892B242F08002DA800BE0AC
:10E6180040F29812C2F20002D38823F080034FEA36
:10E6280003434FEA1343D38040F29813C2F2000326
:10E63800DB8813F0010F08D04FF48050C4F20100BA
:10E648004FF00401F9F726FA07E04FF48050C4F2BE
:10E6580001004FF00401F9F72BFA40F29813C2F2C7
:10E668000003DB8813F0020F08D04FF48050C4F287
:10E6780001004FF00801F9F70DFA07E04FF4805058
:10E68800C4F201004FF00801F9F712FA40F29813AA
:10E69800C2F20003DB8813F0040F08D04FF40060C7
:10E6A800C4F201004FF00801F9F7F4F907E04FF45C
:10E6B8000060C4F201004FF00801F9F7F9F940F2DF
:10E6C8009813C2F20003DB8813F0080F08D04FF448
:10E6D8000060C4F201004FF01001F9F7DBF907E020
:10E6E8004FF40060C4F201004FF01001F9F7E0F9AF
:10E6F80040F29813C2F20003DB8813F0100F08D021
:10E708004FF40060C4F201004FF02001F9F7C2F99C
:10E7180007E04FF40060C4F201004FF02001F9F760
:10E72800C7F940F29813C2F20003DB8813F0200FF8
:10E7380008D04FF44060C4F201004FF00401F9F72B
:10E74800A9F907E04FF44060C4F201004FF004015A
:10E75800F9F7AEF940F29813C2F20003DB8813F020
:10E76800400F08D04FF4C050C4F201004FF480713C
:10E77800F9F790F907E04FF4C050C4F201004FF4E4
:10E788008071F9F795F940F29813C2F20003DB881B
:10E7980013F0800F08D04FF4C050C4F201004FF4BA
:10E7A8000071F9F777F910BD4FF4C050C4F20100B9
:10E7B8004FF40071F9F77CF910BD00BF00B583B0C4
:10E7C80040F29813C2F200031B7A13F0800F20D096
:10E7D80041F6F623C2F200031A7802F10102D2B21E
:10E7E8001A701B78052B32D941F61133C2F2000397
:10E7F8004FF000021A7041F6F623C2F200031A70B5
:10E8080040F2C003C2F200031B684FF001021A7005
:10E818001DE041F61133C2F200031A7802F1010239
:10E82800D2B21A701B78052B11D941F61132C2F2F7
:10E8380000024FF00003137041F6F622C2F2000204
:10E84800137040F2C002C2F200021268137040F264
:10E858009813C2F200031B7A13F0400F20D041F640
:10E868002833C2F200031A7802F10102D2B21A70F8
:10E878001B78052B32D941F60933C2F200034FF059
:10E8880000021A7041F62833C2F200031A7040F2EF
:10E89800C403C2F200031B684FF001021A701DE0A6
:10E8A80041F60933C2F200031A7802F10102D2B22A
:10E8B8001A701B78052B11D941F60932C2F20002F1
:10E8C8004FF00003137041F62832C2F200021370B1
:10E8D80040F2C402C2F200021268137040F29813A8
:10E8E800C2F200031B7A13F0200F20D041F6163332
:10E8F800C2F200031A7802F10102D2B21A701B7830
:10E90800052B32D941F61833C2F200034FF000024A
:10E918001A7041F61633C2F200031A7040F2C803A7
:10E92800C2F200031B684FF001021A701DE041F6A5
:10E938001833C2F200031A7802F10102D2B21A7037
:10E948001B78052B11D941F61832C2F200024FF09C
:10E958000003137041F61632C2F20002137040F23F
:10E96800C802C2F200021268137040F29813C2F291
:10E9780000031B7A13F0100F20D041F62E33C2F299
:10E9880000031A7802F10102D2B21A701B78052B23
:10E9980032D941F61233C2F200034FF000021A7066
:10E9A80041F62E33C2F200031A7040F2CC03C2F2D1
:10E9B80000031B684FF001021A701DE041F6123384
:10E9C800C2F200031A7802F10102D2B21A701B785F
:10E9D800032B11D941F61232C2F200024FF00003A4
:10E9E800137041F62E32C2F20002137040F2CC02CC
:10E9F800C2F200021268137040F29813C2F20003C8
:10EA08001B7A13F0080F20D041F6F923C2F2000355
:10EA18001A7802F10102D2B21A701B78052B32D98A
:10EA280041F6FE23C2F200034FF000021A7041F6CD
:10EA3800F923C2F200031A7040F2D003C2F20003B5
:10EA48001B684FF001021A701DE041F6FE23C2F266
:10EA580000031A7802F10102D2B21A701B78052B52
:10EA680011D941F6FE22C2F200024FF000031370E2
:10EA780041F6F922C2F20002137040F2D002C2F24B
:10EA880000021268137040F29813C2F200031B7A56
:10EA980013F0040F20D041F62633C2F200031A788F
:10EAA80002F10102D2B21A701B78052B32D941F655
:10EAB8002A33C2F200034FF000021A7041F62633DF
:10EAC800C2F200031A7040F2D403C2F200031B68BA
:10EAD8004FF001021A701DE041F62A33C2F200031A
:10EAE8001A7802F10102D2B21A701B78052B11D9DB
:10EAF80041F62A32C2F200024FF00003137041F6C9
:10EB08002632C2F20002137040F2D402C2F20002AE
:10EB18001268137040F29813C2F200031B7A13F0C4
:10EB2800020F20D041F62933C2F200031A7802F10D
:10EB38000102D2B21A701B78052B32D941F608337C
:10EB4800C2F200034FF000021A7041F62933C2F2F4
:10EB580000031A7040F2D803C2F200031B684FF09A
:10EB680001021A701DE041F60833C2F200031A7858
:10EB780002F10102D2B21A701B78052B11D941F6A5
:10EB88000832C2F200024FF00003137041F6293236
:10EB9800C2F20002137040F2D802C2F200021268F8
:10EBA800137040F29813C2F200031B7A13F0010F9E
:10EBB80020D041F61333C2F200031A7802F10102A1
:10EBC800D2B21A701B78052B32D941F6F523C2F25E
:10EBD80000034FF000021A7041F61333C2F200032B
:10EBE8001A7040F2DC03C2F200031B684FF0010206
:10EBF8001A701DE041F6F523C2F200031A7802F1FB
:10EC08000102D2B21A701B78052B11D941F6F522F0
:10EC1800C2F200024FF00003137041F61332C2F241
:10EC28000002137040F2DC02C2F200021268137094
:10EC38004FF40060C4F20100F8F71EFFADF80600BB
:10EC4800BDF8063013F0010F20D041F6F723C2F2C9
:10EC580000031A7802F10102D2B21A701B78052B50
:10EC680032D941F62733C2F200034FF000021A707E
:10EC780041F6F723C2F200031A7040F2E003C2F231
:10EC880000031B684FF001021A701DE041F627339C
:10EC9800C2F200031A7802F10102D2B21A701B788C
:10ECA800052B11D941F62732C2F200024FF00003BA
:10ECB800137041F6F722C2F20002137040F2E0022C
:10ECC800C2F2000212681370BDF8063013F0020F8A
:10ECD80020D041F6EE23C2F200031A7802F10102B5
:10ECE800D2B21A701B78052B32D941F62D33C2F2F5
:10ECF80000034FF000021A7041F6EE23C2F200033F
:10ED08001A7040F2E403C2F200031B684FF00102DC
:10ED18001A701DE041F62D33C2F200031A7802F191
:10ED28000102D2B21A701B78052B11D941F62D3287
:10ED3800C2F200024FF00003137041F6EE22C2F255
:10ED48000002137040F2E402C2F20002126813706B
:10ED5800BDF8063013F0800F20D041F6EC23C2F244
:10ED680000031A7802F10102D2B21A701B78052B3F
:10ED780032D941F6FA23C2F200034FF000021A70AA
:10ED880041F6EC23C2F200031A7040F2F803C2F213
:10ED980000031B684FF001021A701DE041F6FA23C8
:10EDA800C2F200031A7802F10102D2B21A701B787B
:10EDB800052B11D941F6FA22C2F200024FF00003E6
:10EDC800137041F6EC22C2F20002137040F2F8020E
:10EDD800C2F2000212681370BDF8063013F0400F3B
:10EDE80020D041F6FD23C2F200031A7802F1010295
:10EDF800D2B21A701B78052B32D941F61D33C2F2F4
:10EE080000034FF000021A7041F6FD23C2F200031E
:10EE18001A7040F2FC03C2F200031B684FF00102B3
:10EE28001A701DE041F61D33C2F200031A7802F190
:10EE38000102D2B21A701B78052B11D941F61D3286
:10EE4800C2F200024FF00003137041F6FD22C2F235
:10EE58000002137040F2FC02C2F200021268137042
:10EE68004FF44060C4F20100F8F706FEADF8060062
:10EE7800BDF8063013F0020F20D041F6FF23C2F28E
:10EE880000031A7802F10102D2B21A701B78052B1E
:10EE980032D941F6FC23C2F200034FF000021A7087
:10EEA80041F6FF23C2F200031A7040F2E803C2F2EF
:10EEB80000031B684FF001021A701DE041F6FC23A5
:10EEC800C2F200031A7802F10102D2B21A701B785A
:10EED800052B11D941F6FC22C2F200024FF00003C3
:10EEE800137041F6FF22C2F20002137040F2E802EA
:10EEF800C2F2000212681370BDF8063013F0010F59
:10EF080020D041F62433C2F200031A7802F101023C
:10EF1800D2B21A701B78052B32D941F60A33C2F2E5
:10EF280000034FF000021A7041F62433C2F20003C6
:10EF38001A7040F2EC03C2F200031B684FF00102A2
:10EF48001A701DE041F60A33C2F200031A7802F182
:10EF58000102D2B21A701B78052B11D941F60A3278
:10EF6800C2F200024FF00003137041F62432C2F2DD
:10EF78000002137040F2EC02C2F200021268137031
:10EF880003B000BD10B446F6B843C4F200031888B5
:10EF980080B246F6B043C4F20003198889B246F637
:10EFA800B443C4F200031B889BB246F6AC42C4F2D9
:10EFB8000002148804F10104A4B21480128892B2E9
:10EFC800062A81BF46F6AC42C4F20002002414802F
:10EFD800032B14BF00220122012B08BF42F00102BB
:10EFE8009AB9072B14BF00220122052B08BF42F053
:10EFF800010252B90A2B14BF00220122082B08BFB4
:10F0080042F001020AB90C2B0FD11E299CBF013115
:10F0180089B253D90C2B1DBF01339BB2012101309A
:10F0280002BF80B201210B4648E0062B14BF002224
:10F038000122042B08BF42F0010242B90B2B14BF76
:10F0480000220122092B08BF42F0010242B11D290A
:10F0580099BF013189B201339BB288BF01212DE0EC
:10F06800022B2BD11B299CBF013189B226D91C291F
:10F0780018D110F0030F1CBF012103231ED14FF03C
:10F088006402B0FBF2F102FB110292B23AB94FF4FA
:10F09800C872B0FBF2F102FB110292B22AB94FF02A
:10F0A8001D010BE01D2909D104E04FF001014FF0CB
:10F0B800030303E04FF001014FF0030346F6B042AB
:10F0C800C4F20002118046F6B442C4F20002138072
:10F0D80046F6B843C4F20003188010BC704700BF5E
:10F0E80010B504464FF080404FF001014FF0000288
:10F0F800FAF7DEF84FF400604FF00001F9F7F0FA84
:10F10800FEF754FC2046FEF7CBFCFEF75FFC4FF001
:10F118005000FBF78BFC4FF400604FF00101F9F74A
:10F12800DFFA4FF080404FF001010A46FAF7C0F8C5
:10F1380010BD00BFF0B583B007460E4614461D4605
:10F1480001F0E8FAFEF732FC4FF03500FEF748FC14
:10F15800ADB1F61923788DF8043063788DF8053051
:10F16800BDF80410304689B2FEF77CFC06F10206B1
:10F1780005F1FF35ADB204F10204002DEAD1FEF726
:10F1880025FC01F0BFFA03B0F0BD00BF10B483B096
:10F198001C46B3B1081802F1020304F1FF34A4B20B
:10F1A80003EB440450F8023B9BB2ADF804309DF8E1
:10F1B800043013709DF80530537002F10202944236
:10F1C800F0D103B010BC704710B541F6F023C2F27D
:10F1D80000031B6883B141F6F023C2F200031A68EA
:10F1E80002F1FF321A601B6833B941F61433C2F2D8
:10F1F80000034FF000021A7041F63033C2F20003E8
:10F208004FF000021A704FF4A050C4F201004FF4FE
:10F218008061F8F711FC38B141F63033C2F20003CF
:10F228001A7842F008021A704FF4A050C4F2010094
:10F238004FF40061F8F700FC38B141F63033C2F200
:10F2480000031A7842F010021A704FF4A050C4F26A
:10F2580001004FF48051F8F7EFFB38B141F6303335
:10F26800C2F200031A7842F020021A704FF4A0503C
:10F27800C4F201004FF40051F8F7DEFB38B141F653
:10F288003033C2F200031A7842F040021A7041F695
:10F298003033C2F200031B78002B77D041F62033BD
:10F2A800C2F200034FF000021A7041F60033C2F2B6
:10F2B80000031B78002B00F0888041F63033C2F23F
:10F2C80000031A7841F60133C2F200031B7843EABF
:10F2D800020241F6ED23C2F200031B78934248D1A3
:10F2E80041F62133C2F200031A7802F10102D2B2C8
:10F2F8001A701B78052B68D97F4A4FF0000341F636
:10F30800ED24C2F20004217812F8010F88421ED1C0
:10F3180041F6EF22C2F20002137040F64312C2F225
:10F328000002127822B141F62232C2F200021370B2
:10F3380041F6F023C2F2000342F210721A6041F65D
:10F348001433C2F200034FF001021A7004E003F113
:10F358000103DBB2142BD6D141F62133C2F20003EC
:10F368004FF000021A7041F60033C2F200031A701F
:10F378002BE041F6ED23C2F200031A7041F6213367
:10F38800C2F200034FF000021A701EE041F620336B
:10F39800C2F200031A7802F10102D2B21A701B7885
:10F3A800142B12D941F60033C2F200034FF00102C8
:10F3B8001A7041F62033C2F200034FF000021A70AF
:10F3C80041F62133C2F200031A7041F60133C2F24A
:10F3D80000031B78042B76D8DFE803F0031B3147C2
:10F3E8005F004FF4A050C4F201004FF48041F8F7D9
:10F3F8005FFB4FF48050C4F201004FF48071F8F7BE
:10F4080049FB41F60133C2F200034FF001021A70C2
:10F4180010BD4FF48054C4F2010420464FF48071AB
:10F42800F8F746FB20464FF08001F8F733FB41F62A
:10F438000133C2F200034FF002021A7010BD4FF4FC
:10F448008054C4F2010420464FF08001F8F730FBE5
:10F4580020464FF04001F8F71DFB41F60133C2F298
:10F4680000034FF003021A7010BD4FF48050C4F22D
:10F4780001004FF04001F8F71BFB4FF4A050C4F215
:10F4880001004FF40041F8F705FB41F60133C2F2E1
:10F4980000034FF004021A7010BD4FF4A054C4F2D8
:10F4A800010420464FF40041F8F702FB20464FF4D0
:10F4B8008041F8F7EFFA41F60133C2F200034FF04A
:10F4C80000021A7010BD4FF48050C4F201004FF4CE
:10F4D800E071F8F7EDFA4FF4A050C4F201004FF4D0
:10F4E8004041F8F7E5FA41F60133C2F200034FF064
:10F4F80000021A7010BD00BFE31D01082DE9F00FCE
:10F5080086B045B24FEAD57433EA250328BFFF23F6
:10F5180038299CBF0126039605D93F299CBF0025A1
:10F52800039500F2C6811BB1012B40F0CD81F2E0BA
:10F5380011F00709CDF8049036D14FEAD1034FEA0C
:10F54800C313C31802EB820240F29C21C2F20001ED
:10F558008F6803F1050C1FFA8CFC41F6F856C0F6CB
:10F56800010640F26845C2F20005012F0EBFB15CEA
:10F57800B11891F8F814E95403F101039BB200F1B2
:10F588000100C0B2802805D8634505D002F1010208
:10F5980092B2EAE74FF0010440F26842C2F2000278
:10F5A8004FF00001D1548FE14FEAD1014FEAC11564
:10F5B800451902EB820240F29C23C2F20003D3F801
:10F5C80008904FF0000841F6F85CC0F6010C019F66
:10F5D80040F26841C2F20001C7F10803DBB20293AE
:10F5E8000494B9F1010F0EBF1CF802300CEB0203B2
:10F5F80093F8F8343E46019C03FA04FB2C4611F8B4
:10F6080005A04AEA0B0A5FFA8AFA01F805A09346B0
:10F618003A46DA464FEA4303DBB243F0010302F10C
:10F62800FF32D2B2002AF5D1524611F804A003EAFB
:10F638000A030B55039B002B39D0B9F1010F01BF09
:10F648001CF802B0CDF814B0C6F1080A4BFA0AFB50
:10F658001FBF0CEB020393F8F8340593C6F1080BAF
:10F6680018BF43FA0BFB04F1800411F804A04AEA1E
:10F678000B0A5FFA8AFA01F804A0DDF808A05346DD
:10F6880073B1059B93465246DA464FEA530343F05B
:10F69800800302F1FF32D2B2002AF6D10593524616
:10F6A80011F804A0DDF814B00BEA0A030B5505F1B4
:10F6B8000105ADB200F10100C0B2802800F2FC8063
:10F6C80008F101085FFA88F8B8F1050F03D002F1D4
:10F6D800010292B285E7049C40F26843C2F200033B
:10F6E800595DC6F108024FF0FF0040FA02F201EA44
:10F6F80002025A55039B002B00F0E68005F18005B5
:10F7080040F26843C2F20003595D00FA06F201EACA
:10F7180002025A55D8E011F0070B38D14FEAD1034D
:10F728004FEAC313C3184FEAC2024FF0000641F66E
:10F73800F85CC0F6010C40F26845C2F200050CEB1B
:10F748004201B1F8F019CFB2EF5403F18007C1F3C9
:10F758000721E95503F101039BB202F1010292B2BC
:10F7680000F10100C0B210F0800F40F0A88006F14F
:10F778000106F6B2082EE2D140F26842C2F2000257
:10F788004FF00001D15403F18003D1549CE04FEABB
:10F79800D1014FEAC11141184FEAC2074FF0000CDE
:10F7A80041F6F855C0F601050195D84640F2684281
:10F7B800C2F20002CBF108060296F3B20493059454
:10F7C800019C04EB4703B3F8F059EBB2C24603FAC5
:10F7D8000BF60C4612F8019049EA0606F6B25654A2
:10F7E80046464FEA4303DBB243F0010306F1FF3616
:10F7F800F6B2002EF5D1165D33401355039E0EB3B5
:10F8080004F18003DDF8089045FA09F6D6544FEA6A
:10F81800152343FA09F304F58074165D46EA0303D9
:10F82800DBB213554FEA1525049B43B14FEA550542
:10F8380045F0800503F1FF33DBB2002BF6D1135DF1
:10F848001D40155501F1010189B200F10100C0B256
:10F8580010F0800F36D10CF1010C5FFA8CFCBCF172
:10F86800080F03D007F10107BFB2A9E7059C40F2D2
:10F878006843C2F20003585CCAF108024FF0FF0562
:10F8880045FA02F200EA02025A54039BE3B101F17D
:10F89800800240F26843C2F200034FF0000098541F
:10F8A80001F58071585C05FA0AF200EA02025A541E
:10F8B8000AE04FF0010407E04FF0010404E04FF0C4
:10F8C800010401E04FF00104204606B0BDE8F00F46
:10F8D800704700BF2DE9F047064688461F463F2976
:10F8E80088BF002403D880288CBF00240124154633
:10F8F8004FF000094FF0010A1BE0D2B217B1012FF7
:10F9080017D10BE0304641464B46FFF7F7FD00287C
:10F9180018BF002406F10606F6B20AE03046414652
:10F928005346FFF7EBFD002818BF002406F109062F
:10F93800F6B215F8012B51B2231E18BF0123002976
:10F948000CBF002303F00103002BD6D140F2A8130B
:10F95800C2F200031A7802F10102D2B21A70BDE8AD
:10F96800F08700BF38B51C469DF810509DF814303C
:10F97800302A19D17CB915F0010F04D0FFF7BEFD6C
:10F988004FF0010416E04FF02002FFF7B7FD002802
:10F9980018BF80240EE04FF03002FFF7AFFD0028BB
:10F9A80014BF8124012405E0FFF7A8FD002814BF37
:10F9B80081240124204638BD2DE9F04F83B0074645
:10F9C8008B4616461C469DF8309003F1FF3303F032
:10F9D800FF03092B88BF0A246FEA00023F298CBF66
:10F9E8000023012313EAD21300F0A380C9F34008CF
:10F9F80009F0F003202B0BD0302B11D0102B1BD18A
:10FA0800F3B213F0800F1CBF5B42DEB214D072E079
:10FA1800B3B213F4004F1CBF5B429EB20CD06AE035
:10FA2800002EB8BF764207DA65E007F10907FFB292
:10FA380002E007F10607FFB204F1FF33092B24D8CF
:10FA4800DFE803F0201D1A17140F0A056C6749F246
:10FA58008065C0F2980565E044F24025C0F20F05C4
:10FA680060E048F2A065C0F201055BE042F2107563
:10FA780058E04FF47A7555E04FF0640552E04FF0C6
:10FA88000A054FE04FF001054CE054B34AE0B6FBDD
:10FA9800F5F202F13002CDF80090CDF80480384636
:10FAA8005946D2B2FFF75EFF034642B234EA220457
:10FAB80028BF0124B8F1000F03D007F10907FFB2EE
:10FAC80002E007F10607FFB204F1FF34E4B244B1E3
:10FAD800B6FBF5F205FB1266AAFB05254FEAD5052C
:10FAE800D5E740F2A813C2F200031A7802F1010226
:10FAF800D2B21A701DE0384659464FF02D024346DF
:10FB0800FFF7FCFC002818BF0024B8F1000F90D0C4
:10FB18008BE74FF44A45C3F69A3503E04FF4614545
:10FB2800C0F2F5554FF000034CF6CD4ACCF6CC4A5E
:10FB3800ADE703B0BDE8F08F2DE9F04F83B005467F
:10FB48008A4690461C469DF830609DF8349003F133
:10FB5800FF3303F0FF03092B88BF0A246FEA000272
:10FB68003F298CBF0023012313EAD21300F0AE8093
:10FB7800B8F1000F13DAC8F100084FF02D024B4618
:10FB8800FFF7BCFC002818BF0024B9F1000F03D10F
:10FB980005F10605EDB202E005F10905EDB246B141
:10FBA800B44282BFC6F10106361906F0FF0605D831
:10FBB80002E04FF0FF0601E04FF0FF0604F1FF33CB
:10FBC800092B24D8DFE803F0201D1A17140F0A05A3
:10FBD8007D7849F28067C0F298071AE044F240271E
:10FBE800C0F20F0715E048F2A067C0F2010710E065
:10FBF80042F210770DE04FF47A770AE04FF064078D
:10FC080007E04FF00A0704E04FF0010701E0002C7D
:10FC180048D04CF6CD4BCCF6CC4B06F1FF36F6B2BD
:10FC2800A6B9284651464FF02E024B46FFF766FC10
:10FC3800002818BF0024B9F1000F03D105F106050B
:10FC4800EDB22DE005F10905EDB229E0B8FBF7F2B8
:10FC580002F130024FF000030093CDF804902846DB
:10FC68005146D2B24FF00103FFF77CFE40B234EAAE
:10FC7800200428BF0124B8FBF7F307FB1388ABFB6C
:10FC880007274FEAD707B9F1000F03D105F1060599
:10FC9800EDB202E005F10905EDB204F1FF34E4B27A
:10FCA800002CBAD140F2A813C2F200031A7802F16C
:10FCB8000102D2B21A7009E04FF44A47C3F69A37E4
:10FCC800A7E74FF46147C0F2F557A2E703B0BDE8D4
:10FCD800F08F00BF10B540F2A813C2F200034FF036
:10FCE80000025A70F1F7A2F94FF014004FF0010129
:10FCF800F4F7BCFE4FF4A054C4F2010420464FF0C0
:10FD08001001F7F7D5FE4FF014004FF00101F4F79A
:10FD1800ADFE20464FF01001F7F7BCFE4FF014007F
:10FD28004FF00101F4F7A2FE20464FF00801F7F763
:10FD3800BFFE20464FF48071F7F7BAFE4FF46050CB
:10FD4800C4F200004FF0A301F9F740F84FF0C803E0
:10FD5800013BFDD14FF4A054C4F2010420464FF4F6
:10FD68008071F7F797FE4FF002004FF00101F4F7AA
:10FD78007DFE20464FF48071F7F79AFE4FF46050ED
:10FD8800C4F200004FF0A101F9F720F84FF0C803C2
:10FD9800013BFDD14FF4A054C4F2010420464FF4B6
:10FDA8008071F7F777FE4FF002004FF00101F4F78A
:10FDB8005DFE20464FF48071F7F77AFE4FF46050ED
:10FDC800C4F200004FF0C001F9F700F84FF0C80383
:10FDD800013BFDD14FF4A054C4F2010420464FF476
:10FDE8008071F7F757FE4FF002004FF00101F4F76A
:10FDF8003DFE20464FF48071F7F75AFE4FF46050ED
:10FE0800C4F200004FF0A601F8F7E0FF4FF0C80376
:10FE1800013BFDD14FF4A054C4F2010420464FF435
:10FE28008071F7F737FE4FF002004FF00101F4F749
:10FE38001DFE20464FF48071F7F73AFE4FF46050EC
:10FE4800C4F200004FF02F01F8F7C0FF4FF0C803CD
:10FE5800013BFDD14FF4A054C4F2010420464FF4F5
:10FE68008071F7F717FE4FF002004FF00101F4F729
:10FE7800FDFD20464FF48071F7F71AFE4FF46050ED
:10FE8800C4F200004FF0F801F8F7A0FF4FF0C803E4
:10FE9800013BFDD14FF4A054C4F2010420464FF4B5
:10FEA8008071F7F7F7FD4FF002004FF00101F4F70A
:10FEB800DDFD20464FF48071F7F7FAFD4FF46050EE
:10FEC800C4F200004FF00001F8F780FF4FF0C803BC
:10FED800013BFDD14FF4A054C4F2010420464FF475
:10FEE8008071F7F7D7FD4FF002004FF00101F4F7EA
:10FEF800BDFD20464FF48071F7F7DAFD4FF46050EE
:10FF0800C4F200004FF02601F8F760FF4FF0C80375
:10FF1800013BFDD14FF4A054C4F2010420464FF434
:10FF28008071F7F7B7FD4FF002004FF00101F4F7C9
:10FF38009DFD20464FF48071F7F7BAFD4FF46050ED
:10FF4800C4F200004FF08101F8F740FF4FF0C803FA
:10FF5800013BFDD14FF4A054C4F2010420464FF4F4
:10FF68008071F7F797FD4FF002004FF00101F4F7A9
:10FF78007DFD20464FF48071F7F79AFD4FF46050ED
:10FF8800C4F200004FF01001F8F720FF4FF0C8034B
:10FF9800013BFDD14FF4A054C4F2010420464FF4B4
:10FFA8008071F7F777FD4FF002004FF00101F4F789
:10FFB8005DFD20464FF48071F7F77AFD4FF46050ED
:10FFC800C4F200004FF0AC01F8F700FF4FF0C8038F
:10FFD800013BFDD14FF4A054C4F2010420464FF474
:10FFE8008071F7F757FD4FF002004FF00101F4F769
:08FFF8003DFD20464FF480712D
:020000040801F1
:10000000F7F75AFD4FF46050C4F200004FF00001C2
:10001000F8F7E0FE4FF0C803013BFDD14FF4A054C8
:10002000C4F2010420464FF48071F7F737FD4FF01A
:1000300002004FF00101F4F71DFD20464FF48071DE
:10004000F7F73AFD4FF46050C4F200004FF0AF01F3
:10005000F8F7C0FE4FF0C803013BFDD14FF4A054A8
:10006000C4F2010420464FF48071F7F717FD4FF0FA
:1000700002004FF00101F4F7FDFC20464FF48071BF
:10008000F7F71AFD4FF46050C4F200004FF0400142
:10009000F8F7A0FE4FF0C803013BFDD14FF4A05488
:1000A000C4F2010420464FF48071F7F7F7FC4FF0DB
:1000B00002004FF00101F4F7DDFC20464FF400711F
:1000C000F7F7ECFC40F2A813C2F200034FF0010274
:1000D0005A704FF000029A7010BD00BF10B540F288
:1000E000A813C2F200035B78072B00F20781DFE858
:1000F00013F00C010800320071009500B900DA001D
:10010000F3004FF4A054C4F2010420464FF008015C
:10011000F7F7D2FC20464FF48071F7F7CDFC4FF48F
:100120006050C4F200004FF04001F8F753FE4FF06A
:10013000C803013BFDD14FF4A050C4F201004FF4BD
:100140008071F7F7ABFC40F2A813C2F200034FF046
:1001500002025A7010BD4FF4A050C4F201004FF4D7
:100160008071F7F7A9FC40F2A813C2F20003997856
:100170004FF46050C4F2000041F0B001F8F72AFEDD
:100180004FF0C803013BFDD14FF4A050C4F2010071
:100190004FF48071F7F782FC40F2A813C2F200031B
:1001A0009A784FEAC2129A809A7802F10102D2B28A
:1001B0009A709B78072B81BF40F2A813C2F200030C
:1001C00000229A7040F2A813C2F200034FF003021B
:1001D0005A7010BD4FF4A050C4F201004FF480716A
:1001E000F7F76AFC4FF46050C4F200004FF01001C2
:1001F000F8F7F0FD4FF0C803013BFDD14FF4A050DC
:10020000C4F201004FF48071F7F748FC40F2A813E4
:10021000C2F200034FF004025A7010BD4FF4A05018
:10022000C4F201004FF48071F7F746FC4FF46050C0
:10023000C4F200004FF00001F8F7CCFD4FF0C80306
:10024000013BFDD14FF4A050C4F201004FF4807186
:10025000F7F724FC40F2A813C2F200034FF00502A6
:100260005A7010BD4FF4A054C4F2010420464FF060
:100270000801F7F713FC20464FF48071F7F71CFCD8
:1002800040F2A814C2F20004A08880B240F2684391
:10029000C2F2000318184FF08001F0F7FFFE4FF094
:1002A0000603637010BD4FF40030F8F743FF60B3EE
:1002B0004FF02000F8F76EFF4FF4A050C4F2010099
:1002C0004FF48071F7F7EAFB40F2A813C2F2000383
:1002D0004FF007025A7010BD40F2A813C2F200039B
:1002E0004FF001025A709B797BB140F2A813C2F221
:1002F00000034FF000029A715A7010BD40F2A8132B
:10030000C2F200034FF001025A7010BD2DE9F00F48
:1003100084B09DF83050904282BF04461046224679
:10032000994282BF0C461946234644B230EA240063
:1003300028BF7F203F2928BF3F21C9B254B232EAEB
:10034000240228BF7F223F2B34BF9A464FF03F0A3A
:100350005FFA8AFA904214BF4FF000084FF001088C
:10036000514514BF4FF0000B4FF0010B01F0070394
:1003700001934FF0010707FA03F7FFB215B16FEAD7
:100380000707FFB24FEAD101029103904FEAC1196A
:1003900081441FFA89F9C0F101069619F6B2DEB15F
:1003A0004B46314640F26844C2F2000435B114F8BD
:1003B00003C00CEA070C04F803C005E014F803C0FE
:1003C0004CEA070C04F803C001F1FF31C9B219B1BE
:1003D00003F101039BB2E9E708EB0B033BBB0AF017
:1003E00007034FF0010404FA03F4E4B215B16FEA15
:1003F0000404E4B2DEB14FEADA034FEAC313DDF8D6
:100400000CC063449BB240F26841C2F200011DB1CE
:10041000CF5C2740CF5402E0CF5C2743CF5406F196
:10042000FF36F6B21EB103F101039BB2EFE7BBF159
:10043000000F40F03A810299C1EBDA06F6B2002EC5
:1004400000F0F2804FF0FF01019B01FA03F1C9B205
:10045000D5B16FEA0101C9B240F26843C2F20003AC
:1004600013F809400C4003F80940B8F1000F22D1FD
:10047000C0EB0904A41840F26843C2F200031F5DF8
:1004800007EA0101195516E040F26843C2F2000381
:1004900013F809400C4303F80940B8F1000F0AD1E2
:1004A000C0EB0904A41840F26843C2F200031F5DC8
:1004B00047EA01011955012E40F2828006F1FF3111
:1004C000C9B2002937D04B4640F26844C2F200045A
:1004D0004FF0FF07C0EB020CCDF804C04FF0000B4B
:1004E000029094464246E04603F180039BB245B138
:1004F00004F803B062B9019800EB030C04F80CB0E7
:1005000006E0E75422B9019800EB030C04F80C70E4
:1005100001F1FF31C9B20029E6D102984346904665
:100520001A46A6F10203DBB24FEAC31303F18003BC
:1005300099441FFA89F96FEA0A0A0AF0070A4FF08C
:10054000FF0141FA0AF1C9B209F180091FFA89F9DC
:10055000E5B16FEA0101C9B240F26843C2F200039B
:1005600013F809400C4003F80940B8F1000F40F0BF
:100570009C80121A914440F26843C2F2000313F8BF
:10058000092002EA010103F809108EE040F26843F5
:10059000C2F2000313F809400C4303F80940B8F114
:1005A000000F40F08280121A914440F26843C2F278
:1005B000000313F8092042EA010103F8091074E06E
:1005C0006FEA0A0303F007034FF0FF0444FA03F451
:1005D000E4B209F180039BB2A5B16FEA0404E4B26E
:1005E00040F26841C2F20001CD5C2540CD54B8F123
:1005F000000F5AD11B1A9A180B46895C01EA0404B1
:100600009C5452E040F26841C2F20001CD5C2543A7
:10061000CD54B8F1000F48D11B1A9A180B46895CCB
:1006200041EA04049C5440E04FF0FF03019C03FAAC
:1006300004F1C9B26FEA0A0A0AF0070A43FA0AF398
:1006400001EA0303D5B16FEA0303D9B240F268436C
:10065000C2F2000313F809400C4003F80940B8F156
:10066000000F22D1C0EB0900821840F26843C2F2A9
:100670000003985C00EA0101995416E040F26841D9
:10068000C2F2000111F809401C4301F80940B8F119
:10069000000F0AD1C0EB0900821840F26841C2F293
:1006A0000001885C40EA03038B5440F2A813C2F2B5
:1006B00000031A7802F10102D2B21A7004B0BDE848
:1006C000F00F704730B44FF00005294640F26844FF
:1006D000C2F200040AE01A18A15403F10103DBB2CC
:1006E000802BF8D105F10105082D03D00B464FEA08
:1006F000C510F0E740F2A813C2F200031A7802F125
:100700000102D2B21A7030BC704700BF40F2A81389
:10071000C2F200034FF001025A70704740F2A81372
:10072000C2F200034FF001029A711A465378002B6F
:10073000FCD17047446F6261206F746576F8656E16
:10074000ED2074E1686C612E200020202020202004
:1007500020202020202020202020202020202000B9
:100760002020202020202020202020202020202089
:10077000202020202000736563000000000000009E
:100780000000000000000000000000004C300000ED
:100790000000000000000000000000000000000059
:1007A0000000320000000000000000000000000017
:1007B0000000000000000000446F62612063686F69
:1007C00064752062696F20666978752E200020208C
:1007D0002020202020202020202020202020202019
:1007E0002020200020202020202020202020202029
:1007F000202020202020202020006D696E00000095
:1008000000000000000000000000000000000000E8
:100810004C3000000000000000000000000000005C
:100820000000000000003200000000000000000096
:100830000000000000000000000000004D61782072
:10084000646F62612063686F64752020202020201F
:10085000200070726F6772616D75206B726D656ECE
:10086000ED2E2020202020002020202020202020CD
:100870002020202020202020202020202000736500
:100880006300000000000000000000000000000005
:10089000000000004C3000000000000000000000DC
:1008A0000000000000000000000034000000000014
:1008B0000000000000000000000000000000000038
:1008C0004D696E20646F62612063686F64752020DB
:1008D00020202020200070726F6772616D75206B80
:1008E000726D656EED202020202020002020202029
:1008F00020202020202020202020202020202020F8
:10090000200073656300000000000000000000008C
:1009100000000000000000004C300000000000005B
:100920000000000000000000000000000000330094
:1009300000000000000000000000000000000000B7
:10094000000000005472616E73706F72742E20206C
:1009500020202020202020202000506FE8657420D7
:10096000696D702F6D696E2020000000000000008E
:100970002020202020202020202020202020202077
:10098000202020202000692F6D00000000000000C2
:100990000000000000000000000000004C300000DB
:1009A0000000000000000000000000000000000047
:1009B0000000340000000000000000000000000003
:1009C0000000000000000000527963686C6F7374CF
:1009D000207265616B6365206E61202020006B6F63
:1009E0006E636F76E9207370ED6E61E865202020FC
:1009F0002020200053312C53322C53332C53342ECF
:100A0000202020202020202020007365630000008B
:100A100000000000000000000000000000000000D6
:100A20004C3000000000000000000000000000004A
:100A30000000000000003200000000000000000084
:100A40000000000000000000000000005A61206B60
:100A5000647920646F7379706520706F2020202086
:100A60002000726F7A65706E7574ED20736EED6D97
:100A700061E8F920202020005332206E65626F204B
:100A80005333206E65626F2053342E2020006D6931
:100A90006E000000000000000000000000000000E8
:100AA000000000004C3000000000000000000000CA
:100AB0000000000000000000000032000000000004
:100AC0000000000000000000000000000000000026
:100AD0004D61782E20646F62612063686F647520B9
:100AE0002020202020006D6F746F72752070F869CF
:100AF00020646F737970E176E16EED004E65646F8E
:100B0000E86B616C2073652053322C332C342E201B
:100B100020006D696E000000000000000000000071
:100B200000000000000000004C3000000000000049
:100B30000000000000000000000000000000320083
:100B400000000000000000000000000000000000A5
:100B5000000000005672656D71206F746B726976CB
:100B6000616E6965202020202000747167692E2045
:100B70002020202020202020202020202020200095
:100B80002020202020202020202020202020202065
:100B9000202020202000736563000000000000007A
:100BA0000000000000000000000000004C300000C9
:100BB0000000000000000000000000000000000035
:100BC00000003200000000000000000000000000F3
:100BD00000000000000000005672656D7120786F03
:100BE00064612062696F206669782E2020002020D1
:100BF00020202020202020202020202020202020F5
:100C00002020200020202020202020202020202004
:100C1000202020202020202020006D696E00000070
:100C200000000000000000000000000000000000C4
:100C30004C30000000000000000000000000000038
:100C40000000000000003200000000000000000072
:100C50000000000000000000000000004D6178204E
:100C60007672656D7120786F6461202020202020CD
:100C7000200070726F6772616D6D61206B6F726DB5
:100C80006C656E69652E2000202020202020202009
:100C900020202020202020202020202020007365DC
:100CA00063000000000000000000000000000000E1
:100CB000000000004C3000000000000000000000B8
:100CC00000000000000000000000340000000000F0
:100CD0000000000000000000000000000000000014
:100CE0004D696E207672656D7120786F6461202089
:100CF00020202020200070726F6772616D6D61206E
:100D00006B6F726D6C656E69652E2000202020204F
:100D100020202020202020202020202020202020D3
:100D20002000736563000000000000000000000068
:100D300000000000000000004C3000000000000037
:100D40000000000000000000000000000000330070
:100D50000000000000000000000000000000000093
:100D6000000000005472616E73706F72742E202048
:100D7000202020202020202020004E6F6D65722032
:100D8000696D702F6D696E202020202020202000AA
:100D90002020202020202020202020202020202053
:100DA000202020202000692F6D000000000000009E
:100DB0000000000000000000000000004C300000B7
:100DC0000000000000000000000000000000000023
:100DD00000003400000000000000000000000000DF
:100DE0000000000000000000536B6F726F7374E925
:100DF000207265616B636971206E612020007065EF
:100E000072656B6C68E86174656CE92E20202020A7
:100E10002020200053312C53322C53332C53342EAA
:100E20002020202020202020200073656300000067
:100E300000000000000000000000000000000000B2
:100E40004C30000000000000000000000000000026
:100E50000000000000003200000000000000000060
:100E60000000000000000000000000005672656DE8
:100E70007120737970616E69652020706F736C6585
:100E8000200076796B6C75E8656E69652E202020F0
:100E90002020202020202000533220696C6920204F
:100EA00053332020696C692053342E2020006D6953
:100EB0006E000000000000000000000000000000C4
:100EC000000000004C3000000000000000000000A6
:100ED00000000000000000000000320000000000E0
:100EE0000000000000000000000000000000000002
:100EF0004D61782E207672656D7120786F64612067
:100F0000202020202000646269676174656C612084
:100F10007072692073797061742E20008E64616C28
:100F20002053322C332C342E20202020202020202F
:100F300020006D696E00000000000000000000004D
:100F400000000000000000004C3000000000000025
:100F5000000000000000000000000000000032005F
:100F60000000000000000000000000000000000081
:100F700000000000437A6173206F747761726369C7
:100F80006120636965676C612E002020202020208D
:100F90002020202020202020202020202020200071
:100FA0002020202020202020202020202020202041
:100FB00020202020200073656B000000000000004E
:100FC0000000000000000000000000004C300000A5
:100FD0000000000000000000000000000000000011
:100FE00000003200000000000000000000000000CF
:100FF0000000000000000000437A61732062696510
:101000006775202020202020202020202000424919
:101010004F204649585520202020202020202020E5
:1010200020202000202020202020202020202020E0
:10103000202020202020202020006D696E0000004C
:1010400000000000000000000000000000000000A0
:101050004C30000000000000000000000000000014
:10106000000000000000320000000000000000004E
:101070000000000000000000000000004D616B73E4
:1010800020637A6173206269656720202020202018
:1010900020006D61737A796E792E20202020202027
:1010A0002020202020202000202020202020202060
:1010B00020202020202020202020202020007365B8
:1010C00063000000000000000000000000000000BD
:1010D000000000004C300000000000000000000094
:1010E00000000000000000000000340000000000CC
:1010F00000000000000000000000000000000000F0
:101100004D696E2E637A61732062696567202020C5
:101110002020202020006D61737A796E792E2020A6
:1011200020202020202020202020200020202020DF
:1011300020202020202020202020202020202020AF
:101140002000736563000000000000000000000044
:1011500000000000000000004C3000000000000013
:10116000000000000000000000000000000033004C
:10117000000000000000000000000000000000006F
:10118000000000005472616E73706F72742E202024
:10119000202020202020202020004C69637A6261DA
:1011A00020696D702F6D696E202020202020200086
:1011B000202020202020202020202020202020202F
:1011C000202020202000692F6D000000000000007A
:1011D0000000000000000000000000004C30000093
:1011E00000000000000000000000000000000000FF
:1011F00000003400000000000000000000000000BB
:1012000000000000000000005265616B636A61200D
:10121000646F2020202020202020202020007072B9
:101220007A656C61637A79E82020202020202020D4
:101230002020200053312C53322C53332C53342E86
:101240002020202020202020200073656B0000003B
:10125000000000000000000000000000000000008E
:101260004C30000000000000000000000000000002
:10127000000000000000320000000000000000003C
:101280000000000000000000000000005A61206A19
:10129000616B20646C75672E646F737970652020B4
:1012A000200020202020202020202020202020205E
:1012B00020202020202020005332206E65626F20E5
:1012C0005333206E65626F2053342E2020006D69E9
:1012D0006E000000000000000000000000000000A0
:1012E000000000004C300000000000000000000082
:1012F00000000000000000000000320000000000BC
:1013000000000000000000000000000000000000DD
:101310004D616B7320637A61732062696567202079
:1013200020202020200073696C6E696B612077207B
:10133000646F7379702E20202020200050727A79FB
:10134000737A6C79202053322C332C342E202020B9
:1013500020006D696E000000000000000000000029
:1013600000000000000000004C3000000000000001
:10137000000000000000000000000000000032003B
:10138000000000000000000000000000000000005D
:10139000000000005A61626C6F6B6F7661742068A8
:1013A00065736C656D3F0000000020202020202028
:1013B00020202020202020202020202000000000AD
:1013C000202020202020202020202020202020201D
:1013D00020200000000020000000000000000000AD
:1013E000000000000000000000000000423030005B
:1013F00000000000000000000000000000000000ED
:1014000000003100000000000000000000000000AB
:101410000000000000000000202020205A766F6CA1
:10142000206A617A796B2E202020000000002020A5
:1014300020202020202020202020202020202020AC
:10144000000000002020202020202020202020201C
:1014500020202020202000000000200000000000AC
:10146000000000000000000000000000000000007C
:1014700042303100000000000000000000000000C9
:10148000000000000000310000000000000000002B
:1014900000000000000000000000000020536C6508
:1014A000646F7661742076FD7061646B7920000052
:1014B000000020202020202073ED74EC203F20200D
:1014C000202020200000000020202020202020209C
:1014D00020202020202020202020000000002000AC
:1014E00000000000000000000000000000000000FC
:1014F000000000004230300000000000000000004A
:1015000000000000000000000000310000000000AA
:1015100000000000000000000000000000000000CB
:101520004E61206A616B6F75207465706C6F7475A5
:101530002020000000002020767968F8ED766174A4
:10154000205453312E202020000000002020202095
:1015500020202020202020202020202020200000CB
:101560000000430000000000000000000000000038
:1015700000000000000000004C30000000000000EF
:101580000000000000000000000000000000320029
:10159000000000000000000000000000000000004B
:1015A000000000002046756E6B6365207370ED6E61
:1015B00061E8F920202000000000202053312C3267
:1015C0002C332C342E20202020202020000000004E
:1015D000202020202020202020202020202020200B
:1015E000202000000000200000000000000000009B
:1015F0000000000000000000000000004230330046
:1016000000000000000000000000000000000000DA
:101610000000310000000000000000000000000099
:101620000000000000000000426C6F6B69726F7672
:101630006174E9207061726F6C6F6D3F0000202053
:10164000202020202020202020202020202020209A
:1016500020200000202020202020202020202020CA
:10166000202020202020202000002000000000005A
:10167000000000000000000000000000000000006A
:1016800042303000000000000000000000000000B8
:101690000000000000003100000000000000000019
:1016A0000000000000000000000000002020205684
:1016B00079626572697465206A617A796B2E20207F
:1016C000000020202020202020202020202020205A
:1016D000202020202020000020202020202020204A
:1016E000202020202020202020202020000020005A
:1016F00000000000000000000000000000000000EA
:101700000000000042303100000000000000000036
:101710000000000000000000000031000000000098
:1017200000000000000000000000000000000000B9
:10173000536D6F74726574E9206F746B6C68E86543
:101740006E696A20000020202020202070697461CA
:101750006E6965203F2020202020000020202020CE
:101760002020202020202020202020202020202079
:101770000000200000000000000000000000000049
:1017800000000000000000004230300000000000B7
:101790000000000000000000000000000000310018
:1017A0000000000000000000000000000000000039
:1017B00000000000507269206B616B6F6A2020206E
:1017C0002020202020200000000074656D706572CC
:1017D0006174757265202054533120200000000090
:1017E00020202020202020202020202020202020F9
:1017F0002020000000004300000000000000000066
:101800000000000000000000000000004C3000005C
:1018100000000000000000000000000000000000C8
:101820000000320000000000000000000000000086
:1018300000000000000000002046756E6B6365200C
:1018400076796B6C75E869742E200000000020200A
:1018500053312C322C332C342E20202020202020D9
:1018600000000000202020202020202020202020F8
:101870002020202020200000000020000000000088
:101880000000000000000000000000000000000058
:1018900042303300000000000000000000000000A3
:1018A0000000000000003100000000000000000007
:1018B000000000000000000000000000426C6F6BA0
:1018C0006F7661E8206861736C656D3F20200000D1
:1018D0000000202020202020202020202020202048
:1018E0002020202000000000202020202020202078
:1018F0002020202020202020202000000000200088
:1019000000000000000000000000000000000000D7
:101910000000000042303000000000000000000025
:101920000000000000000000000031000000000086
:1019300000000000000000000000000000000000A7
:10194000202020205779626F72206A657A796B6156
:101950002E200000000020202020202020202020F9
:1019600020202020202020200000000020202020F7
:1019700020202020202020202020202020200000A7
:101980000000200000000000000000000000000037
:1019900000000000000000004230310000000000A4
:1019A0000000000000000000000000000000310006
:1019B0000000000000000000000000000000000027
:1019C000000000004F62736572776F7761E8207ADC
:1019D000616E696B6920000000002020202020201B
:1019E0006D6F6369203F2020202020200000000030
:1019F00020202020202020202020202020202020E7
:101A00002020000000002000000000000000000076
:101A10000000000000000000000000004230300024
:101A200000000000000000000000000000000000B6
:101A30000000310000000000000000000000000075
:101A4000000000000000000050727A79206B616B8A
:101A500069656A2020202020202000000000746595
:101A60006D706172617475727A65205453312E20E5
:101A700000000000202020202020202020202020E6
:101A80002020202020200000000043000000000053
:101A90000000000000000000000000000000000046
:101AA0004C300000000000000000000000000000BA
:101AB00000000000000032000000000000000000F4
:101AC0000000000000000000000000002046756ECD
:101AD0006B6365207370ED6E61E8F92020200000D3
:101AE0000000202053312C322C332C342E20202087
:101AF0002020202000000000202020202020202066
:101B00002020202020202020202000000000200075
:101B100000000000000000000000000000000000C5
:101B20000000000042303300000000000000000010
:101B30000000000000000000000031000000000074
:101B40000000000000000000000000000000000095
:101B50004B616C696272616365207465706C6F744F
:101B6000792E000000007A76EC749A6F76E16EEDC3
:101B70006D20E8ED736C6120000000007A6F622038
:101B8000542E736E699E756A692E353D314300008F
:101B90000000200000000000000000000000000025
:101BA00000000000000000004C30000000000000B9
:101BB00000000000000000000000000000003200F3
:101BC0000000000000000000000000000000000015
:101BD000000000002020204B6F72656B636520526F
:101BE00054432E2020200000000050F869E874695A
:101BF000206E65626F206F6465E874690000000004
